:100000000C94FA1C0C942B1D0C942B1D0C942B1D82
:100010000C942B1D0C942B1D0C942B1D0C942B1D40
:100020000C942B1D0C942B1D0C942B1D0C942B1D30
:100030000C942B1D0D94FF080C942B1D0C942B1D60
:100040000C942B1D0C944FDB0C942B1D0C942B1D2E
:100050000C942B1D0C94FBDC0C94F2DB0D94BF0371
:100060000C942B1D0C9453DD0C947DDD0C942B1DF6
:100070000C942B1D0C942B1D0C942B1D0C942B1DE0
:100080000C942B1D0C942B1D0C942B1D0C942B1DD0
:100090000C942B1D0C942B1D0C942B1D0D94CD0139
:1000A0000C942B1D0C942B1D0C942B1D0C942B1DB0
:1000B0000C942B1D0C942B1D0C942B1D0C942B1DA0
:1000C0000C942B1D0C942B1D0C942B1D0C942B1D90
:1000D0000C942B1D0C942B1D0C942B1D0C942B1D80
:1000E0000C942B1DDF95F795F795F795F795F795F8
:1000F000F795F795F795F795F795F795F795F795A0
:10010000F795F795F795F795F795F795F795F7958F
:10011000F795F795F795F795CE9580958A9504957F
:10012000F795B095BA95F795F7951595F294F795DB
:10013000A695F795C4959C959495F795F795F795A1
:1001400062956C957695F795F795F795F795F795F0
:10015000F795F795F795F795CE9580958A9504953F
:10016000F795B095BA95F795F7951595F294F7959B
:10017000A695F795C4959C959495F795F795F79561
:1001800062956C95769507B398B32BB47CB517C47C
:1001900017C417C417C417C417C417C417C417C487
:1001A000C4B400B53EB517C417C417C417C417C4E8
:1001B00017C417C417C417C417C417C4A3B805B904
:1001C00065B9C5B925BA85BAE5BA17C461BF69BBB7
:1001D000DFBB52BCC4BC36BDA8BD1ABE87BEF4BED0
:1001E00017C417C417C417C417C426B7F3B749B741
:1001F000A9BF16C082C0EFC010C152C184C1B6C130
:100200000FC26AC2C3C21CC33DC331C117C417C4E5
:1002100017C417C417C417C417C417C417C417C406
:1002200017C417C4C6B6F5B617C417C417C417C485
:1002300017C417C417C417C4BFC317C4C2B717C4A1
:1002400017C417C467C395C317C417C417C417C40A
:10025000FAB217C417C4BFB562B6A6B64BB8BC0194
:100260008401BE019801B201C8017A01A201940182
:1002700092019001B6018601C401C801AA01A6013C
:100280009A019C01C601B401C001880196019E013A
:100290008201AE01A401BA0176017E018E019601B0
:1002A000A001AC01C20107634236B79BD8A71A3937
:1002B000685618AEBAAB558C1D3CB7CC5763BD6DB4
:1002C000EDFD753EF6177231BF000000803F05A8B6
:1002D0004CCDB2D44EB93836A9020C50B9918688AB
:1002E000083CA6AAAA2ABE000000803F0D94010582
:1002F0000D944D000D9447030D942B000D940505AE
:100300000D943E000D94ED040D9424030D9484038C
:100310000D94DE040D944E000D94B3050D94090563
:100320000D946B030D9461030D9457030D941C05FC
:100330000D9433030D94AC030D94E2040D94E90481
:100340000D940F050D944F030D94F7040D94A20323
:100350000D9423000D9498030D9413050D94F3044C
:100360000D947A000D943D030D94D4040D947503FF
:100370000D94EE000D94FB040D941F030D942903BE
:100380000D94D8040D9417050D948E030D94E50477
:100390000D94B603436F6C6420657874727573694D
:1003A0006F6E20646973616C6C6F77656400436F76
:1003B0006C6420657874727573696F6E20616C6C03
:1003C0006F776564004175746F72657472616374F0
:1003D0003A0053657474696E67206D6F746F722094
:1003E00063757272656E742E2E2E00536574204DE7
:1003F0006963726F7374657070696E6700547269B7
:1004000067676572696E67207761746368646F6798
:100410002E204966206163746976617465642C20BE
:10042000746865207072696E7465722077696C6C8F
:100430002072657365742E0053657474696E67204D
:100440005468726573686F6C6420546F3A00494E4B
:10045000542050494E3A20004D323531200020744E
:100460006F200053657420766F6C756D65747269CA
:100470006320657874727573696F6E20666F722081
:100480006578747275646572200044697361626C8A
:10049000656420766F6C756D65747269632065782C
:1004A00074727573696F6E20666F722065787472EE
:1004B0007564657220004D313134200048656174E7
:1004C000696E67204265640048656174696E6720E3
:1004D00045787472756465720050696E2063616E50
:1004E000206E6F7420626520736574206279204DE0
:1004F00034322C206D617920696E20696E76616CD2
:100500006964206F7220696E207573652E20004922
:100510006C6C6567616C20532076616C7565206634
:100520006F72204D3432005A2028432920746F778F
:10053000657220666C6F6F722073657420746F3AF9
:100540002000592028422920746F77657220666C3C
:100550006F6F722073657420746F3A2000582028E2
:10056000412920746F77657220666C6F6F722073FB
:10057000657420746F3A2000526F64205261646980
:1005800075732073657420746F3A200047313334DB
:100590002000506F7346726F6D53746570733A002C
:1005A000436F6D7044656C74613A0043616C6962BD
:1005B000726174696F6E206D6F76656D656E742003
:1005C0006973206C696D6974656420746F203130C3
:1005D0006D6D2E004669727374206D6F76652074A0
:1005E0006F20746F75636820617420782C793D30BA
:1005F0002C3020746F206175746F2D7365742072B8
:1006000061646975732E0043616C6962726174691B
:100610006F6E206D6F76656D656E74206973206CEA
:10062000696D6974656420746F2031306D6D2E00C2
:1006300043616E6E6F7420736574207261646975B6
:100640007320616E6420666C6F6F7220617420731A
:10065000616D652074696D652E0043616C6962721D
:100660006174696F6E20636F6465206973206C69C3
:100670006D6974656420746F20626F74746F6D208F
:10068000313025206F66205A2068656967687400DC
:1006900052656C617469766520706F736974696FF7
:1006A0006E696E67004162736F6C75746520706F60
:1006B000736974696F6E696E670047363920005A36
:1006C0003A2000593A2000583A20004F46465345F8
:1006D0005453204F464620425920544F4F204D55E9
:1006E0004348205F20545259494E472041474149D1
:1006F0004E3A200053657474696E672050726F62C1
:10070000652053656E736974697669747920546FD6
:100710003A005A2070726F6265206661696C656488
:10072000206F6E2073656E73697469766974793AA7
:10073000200053657474696E672050726F62652083
:1007400053656E736974697669747920546F3A00E1
:100750005A2070726F6265206661696C6564206FF3
:100760006E2073656E73697469766974793A2000D6
:1007700053657474696E672050726F6265205365AB
:100780006E736974697669747920546F3A005A20DF
:1007900070726F6265206661696C6564206F6E209F
:1007A00073656E73697469766974793A2000686557
:1007B0006865004E6577205261646975733A200060
:1007C0004F6C64205261646975733A200043616C18
:1007D00063756C6174656420526164697573206926
:1007E0007320626164203A0053657474696E6720F7
:1007F00050726F62652053656E73697469766974AF
:100800007920546F3A005A2070726F6265206661D9
:10081000696C6564206F6E2073656E7369746976A8
:100820006974793A200053657474696E6720507258
:100830006F62652053656E73697469766974792097
:10084000546F3A005A2070726F6265206661696C5D
:100850006564206F6E2073656E7369746976697460
:10086000793A2000473332200050524F42452D5AEA
:100870004F46465345543A0047333000536574742D
:10088000696E672050726F62652053656E7369747C
:10089000697669747920546F3A0050726F6265739B
:1008A00020646F206E6F74206D617463682E204F1A
:1008B0006666206279200047333020004D313137A1
:1008C0002043414C4942524154494F4E20434F4DE1
:1008D000504C4554450068656865004E6577204872
:1008E0006F72697A6F6E74616C205261646975739E
:1008F0003A20004F6C6420486F72697A6F6E7461A1
:100900006C205261646975733A200043616C6375B1
:100910006C61746564205261646975732069732029
:100920006261643A20004D3131372043414C4942E5
:10093000524154494F4E204641494C454400436181
:100940006C6962726174696F6E204661696C65647E
:100950000053657474696E672050726F626520532E
:10096000656E736974697669747920546F3A005AB8
:100970002070726F626520284852202D205A207402
:100980006F77657229206661696C6564206F6E20DF
:1009900073656E73697469766974793A20004E657F
:1009A00077205A204865696768743A004F6C642064
:1009B0005A204865696768743A004D3131372043E1
:1009C000414C4942524154494F4E204641494C45C1
:1009D000440043616C6962726174696F6E204661A4
:1009E000696C65640053657474696E672050726F3A
:1009F00062652053656E73697469766974792054F1
:100A00006F3A005A2070726F626520284852202D7C
:100A10002043656E74657220506F696E742920667C
:100A200061696C6564206F6E2073656E73697469AB
:100A3000766974793A200047363920005A3A200006
:100A4000593A2000583A20004D31313720456E6424
:100A500073746F70204F6666736574204572726F91
:100A600072004F464653455453204F464620425944
:100A700020544F4F204D5543482E2041626F7274D1
:100A8000696E672E2053656E73697469766974792F
:100A90003A20004D3131372043414C4942524154B4
:100AA000494F4E204641494C45440043616C6962C0
:100AB000726174696F6E204661696C65640053658C
:100AC0007474696E672050726F62652053656E732F
:100AD0006974697669747920546F3A005A2070728B
:100AE0006F626520285A20546F77657229206661ED
:100AF000696C6564206F6E2073656E7369746976C6
:100B00006974793A20004D3131372043414C4942D4
:100B1000524154494F4E204641494C45440043619F
:100B20006C6962726174696F6E204661696C65649C
:100B30000053657474696E672050726F626520534C
:100B4000656E736974697669747920546F3A005AD6
:100B50002070726F626520285920546F7765722962
:100B6000206661696C6564206F6E2073656E7369C1
:100B70007469766974793A20004D313137204341E8
:100B80004C4942524154494F4E204641494C4544FC
:100B90000043616C6962726174696F6E20466169BD
:100BA0006C65640053657474696E672050726F627F
:100BB000652053656E736974697669747920546F22
:100BC0003A005A2070726F626520285820546F775F
:100BD000657229206661696C6564206F6E2073659B
:100BE0006E73697469766974793A2000456E64732E
:100BF000746F70287329206E6F7420776F726B6921
:100C00006E672070726F7065726C79005A2000599F
:100C100020005820004572726F723A20004D313129
:100C20003720454E4453544F50204552524F5200A6
:100C30004D3130342053300A4D3134302053300A96
:100C40004D313037004D3131372049324320457224
:100C5000726F722E2041626F7274696E6700493242
:100C600043204572726F72202D2043616C6962725D
:100C70006174696F6E2041626F7274656400456EC5
:100C80006473746F70287329206E6F7420776F728D
:100C90006B696E672070726F7065726C79005A2094
:100CA000005920005820004572726F723A20004DA2
:100CB00031313720454E4453544F50204552524F06
:100CC00052006578656375746547436F6465202FCE
:100CD00020717565756544656C74614D6F7665202E
:100CE00072657475726E73206572726F72006969D5
:100CF0007332646820616363656C65726F6D6574DF
:100D0000657220696E697469616C697A696E672EB3
:100D10002E2E00616363656C65726F6D657465721C
:100D2000206932632072656376206661696C656450
:100D30002E00616363656C65726F6D65746572200A
:100D4000777269746520693263206661696C6564D5
:100D50002E00616363656C65726F6D6574657220EA
:100D600073656E6420693263206661696C65642E08
:100D70000000000100250030001D000C00180024B8
:100D80000031001C000B00170023002F001B000A7D
:100D9000001E000D00FFFF0900030022002B001AB7
:100DA0000041004200000002003500206465672E0B
:100DB000204300206D656173757265642000457283
:100DC000726F723A436F756C64206E6F7420686F37
:100DD0006C642074656D7065726174757265200055
:100DE000206D730020616674657220004572726F19
:100DF000723A54656D702E20726169736564207457
:100E00006F20736C6F772E2052697365203D200030
:100E10004739310A4731452D313830463630303088
:100E20000A473930004D3131372045787472756486
:100E3000657220300A54300A4D38342050340A4745
:100E400039310A47314531373246363030300A477A
:100E5000314535463530300A473930001C151C14F1
:100E60000000002243141F1F70121C12AC115C11F1
:100E7000000000000000D410C80F780FFC0E800E98
:100E80000400081D900058091C01B007A801C806FD
:100E900034023006C002C0054C036805D8031805AB
:100EA0006404D004F00498047C056004080630044F
:100EB000940600042007D003AC07A8033808800379
:100EC000C408580350093003DC090803680AD80233
:100ED000F40AB002800B88020C0C6002980C3002FD
:100EE000240DF801B00DC0013C0E8001C80E300188
:100EF000540FB800B40F2800E00F00000400401D9C
:100F0000900060091C01B007A801D0063402380621
:100F1000C002C8054C036805D80318056404D8044A
:100F2000F00498047C05600408063004940600046C
:100F30002007D003AC07A80338088003C40858036F
:100F400050093003DC090803680AE002F40AB80219
:100F5000800B88020C0C6002980C3002240DF80102
:100F6000B00DC0013C0E8001C80E3001540FB80016
:100F7000B40F2800E00F000004000016D800C006DF
:100F8000AC0178058002C004540348042804E80337
:100F9000FC049803D0055003A40618037807D80270
:100FA0004C08A80220097002F4093802C80A080295
:100FB0009C0BD001700C9001440D5001180EF800EC
:100FC000EC0E8800C00F00000400681D4C00500BA0
:100FD00094005809DC0050082401A8076C01280778
:100FE000B401C006FC017006440228068C02F0051C
:100FF000D402B8051C03880564035805AC0330050A
:10100000F40310053C04E8048404C804CC04A804D8
:10101000140590045C057004A4055804EC0538041C
:10102000340620047C060804C406F0030C07D80329
:101030005407C8039C07B003E40798032C088003F7
:1010400074087003BC085803040948034C093003B2
:1010500094091803DC090803240AF0026C0AE00270
:10106000B40AC802FC0AB002440BA0028C0B88022E
:10107000D40B70021C0C5802640C4002AC0C280209
:10108000F40C10023C0DF001840DD801CC0DB80118
:10109000140E98015C0E7001A40E4801EC0E1801AC
:1010A000340FD8007C0F8800C40F0800FC0F00002C
:1010B0000000000000000000000000000000000030
:1010C0000000000000000000000000000000000020
:1010D000000000000000401F450060094F0010099B
:1010E0005C00C0086B0070087D0020089200D007EB
:1010F000AC008007CC003007DE00E006230190063C
:101100005E014006A601F005FF01A0056D02500535
:10111000F30200059603B0045A046004400510046D
:101120004806C0036E077003A8082003EB09D0022D
:10113000230B8002410C3002390DE001040E9001B6
:10114000A20E4001170FF000690FA000A20F50007F
:10115000C60F0000DD0FB0FFEB0F60FF0400700D45
:10116000D8004804AC0158038002D802540380021E
:1011700028043802FC040002D005C801A406980126
:10118000780770014C08480120091801F409F000A3
:10119000C80AC8009C0BA000700C7000440D3800F9
:1011A000180E0000EC0EA8FFC00FE8FE0400001BA4
:1011B00054006009640010097400C00884007008BD
:1011C0009C002008B800D007D80080070001300735
:1011D0002C01E00668019006AC0140060002F00513
:1011E0006802A005E0025005740300052404B00461
:1011F000F0046004DC051004E406C0030408700376
:1012000030092003780B8002600DE001A80E400138
:10121000680FA000C00F0000E80F60FF0400801AF4
:10122000D8009808AC012007800250065403C80576
:1012300028045805FC040005D005B004A406680481
:10124000780728044C08E8032009B003F409700368
:10125000C80A38039C0BF802700CB002440D6802F7
:10126000180E0802EC0E8801C00F8800F00F000075
:101270000000A00F5C006009690010097900C00837
:101280008C007008A2002008BD00D007DE00800797
:10129000050130073401E0066D019006B2014006F9
:1012A0000702F0056D02A005E80250057B0300056A
:1012B0002B04B004F8046004EB06C00335092003D6
:1012C0007F0B8002650DE001B00E40011D0FF000A4
:1012D000480FC8006C0FA000ED0F60FFFE0F48FE26
:1012E000000200002110422063308440A550C660F7
:1012F000E770088129914AA16BB18CC1ADD1CEE1D3
:10130000EFF13112100273325222B5529442F77249
:10131000D662399318837BB35AA3BDD39CC3FFF322
:10132000DEE36224433420040114E664C774A44459
:1013300085546AA54BB528850995EEE5CFF5ACC572
:101340008DD55336722611163006D776F666955629
:10135000B4465BB77AA719973887DFF7FEE79DD7C2
:10136000BCC7C448E5588668A778400861180228B9
:101370002338CCC9EDD98EE9AFF9488969990AA912
:101380002BB9F55AD44AB77A966A711A500A333A89
:10139000122AFDDBDCCBBFFB9EEB799B588B3BBB62
:1013A0001AABA66C877CE44CC55C222C033C600C19
:1013B000411CAEED8FFDECCDCDDD2AAD0BBD688DB2
:1013C000499D977EB66ED55EF44E133E322E511E69
:1013D000700E9FFFBEEFDDDFFCCF1BBF3AAF599F02
:1013E000788F8891A981CAB1EBA10CD12DC14EF1A2
:1013F0006FE18010A100C230E32004502540467008
:101400006760B9839893FBA3DAB33DC31CD37FE332
:101410005EF3B1029012F322D23235421452776257
:101420005672EAB5CBA5A89589856EF54FE52CD502
:101430000DC5E234C324A0148104667447642454A7
:101440000544DBA7FAB79987B8975FE77EF71DC712
:101450003CD7D326F2369106B016576676761546F7
:1014600034564CD96DC90EF92FE9C899E9898AB962
:10147000ABA94458654806782768C018E108823847
:10148000A3287DCB5CDB3FEB1EFBF98BD89BBBAB72
:101490009ABB754A545A376A167AF10AD01AB32A97
:1014A000923A2EFD0FED6CDD4DCDAABD8BADE89DC2
:1014B000C98D267C076C645C454CA23C832CE01CE7
:1014C000C10C1FEF3EFF5DCF7CDF9BAFBABFD98F52
:1014D000F89F176E367E554E745E932EB23ED10E37
:1014E000F01E7C3C3E5E2B3D3F2F5B5D3B2C2A2259
:1014F0005C004D617854656D703A004469616D65BA
:101500007465723A00416363656C65726174696FFA
:101510006E3A004D617853706565643A004A6572B1
:101520006B3A004D617842656454656D703A0050C5
:1015300072696E746572547970653A44656C746151
:10154000005A54726176656C416363656C3A005968
:1015500054726176656C416363656C3A00585472ED
:101560006176656C416363656C3A005A5072696ECE
:1015700074416363656C3A00595072696E744163DB
:1015800063656C3A00585072696E74416363656CB0
:101590003A005A53697A653A005953697A653A00B4
:1015A0005853697A653A005A4D61783A00594D614D
:1015B000783A00584D61783A005A4D696E3A0059B0
:1015C0004D696E3A00584D696E3A004A65726B5823
:1015D000593A005072696E746C696E654361636854
:1015E000653A00454550524F4D3A004175746F6C55
:1015F0006576656C3A005A50726F62653A004361D5
:1016000073654C69676874733A00537570706F72D4
:10161000744C6F63616C46696C616D656E74636870
:10162000616E67653A00537570706F727447313040
:101630004731313A005A486F6D654469723A005932
:10164000486F6D654469723A0058486F6D6544692A
:10165000723A00536F667477617265506F77657286
:101660005377697463683A004C43443A0046616EAC
:101670003A005344436172643A004865617465649A
:101680004265643A004D6978696E67457874727591
:101690006465723A004E756D457874727564657252
:1016A0003A00496E7075744275666665723A00421A
:1016B000617564726174653A004E6F206361736591
:1016C000206C6967687473004D31313420006465A3
:1016D0006C6179203130306D732E00686F6D65411B
:1016E0007869732000686F6D6541786973202F20D9
:1016F000717565756544656C74614D6F76652072B2
:10170000657475726E73206572726F7200486F6DCA
:10171000652044656C7461005072696E7465723A3C
:101720003A736574757020006D6F7665546F5265FD
:10173000616C202F20717565756544656C74614D11
:101740006F76652072657475726E73206572726F44
:1017500072006D6F7665546F202F20717565756509
:1017600044656C74614D6F76652072657475726E38
:1017700073206572726F72005374657070657220A9
:1017800044697361626C6564004B696C6C656400EC
:101790006973506F736974696F6E416C6C6F7765B4
:1017A0006420005344206572726F72206669786508
:1017B00064005344206572726F7220646964206E05
:1017C0006F74207265636F766572210053442052F6
:1017D000656164204572726F720055706C6F616450
:1017E000696E672E2E2E00005344207072696E744D
:1017F0002073746F707065642062792075736572F0
:101800002E005344206361726420696E73657274A4
:101810006564005344204361726420696E7365728D
:1018200074656400534420436172642072656D6F77
:1018300076656400534420636172642072656D6F45
:1018400076656400457874722E00436F6E66696732
:101850003A004F6E65206865617465722073656536
:101860006D73206465636F75706C65642066726F5C
:101870006D20746865726D6973746F72202D2064B9
:10188000697361626C696E6720616C6C20666F724F
:101890002073616665747921004865617465722002
:1018A0006465636F75706C6564004372656174692B
:1018B0006F6E206661696C6564004469726563746B
:1018C0006F727920637265617465640044656C654C
:1018D00074696F6E206661696C65640046696C6549
:1018E0002064656C6574656400446F6E6520736187
:1018F00076696E672066696C652E00577269746937
:101900006E6720746F2066696C653A20006F7065A1
:101910006E206661696C65642C2046696C653A20AE
:10192000004E6F74205344207072696E74696E6744
:10193000005344207072696E74696E672062797416
:1019400065200066696C652E6F70656E2066616942
:101950006C65640046696C652073656C65637465CD
:1019600064002053697A653A0046696C65206F709F
:10197000656E65643A00456E642066696C65206C2E
:1019800069737400426567696E2066696C65206CD6
:10199000697374006572726F722077726974696E10
:1019A0006720746F2066696C6500534420696E6916
:1019B00074206661696C00616476616E6365204CB9
:1019C000205B303D6F66665D006578747275646596
:1019D0007220636F6F6C6572207370656564205B45
:1019E000302D3235355D0064697374616E63652036
:1019F000746F2072657472616374207768656E20FD
:101A000068656174696E67205B6D6D5D0074656DFE
:101A1000702E20666F722072657472616374696FD4
:101A20006E207768656E2068656174696E67205BFB
:101A3000435D0074656D702E2073746162696C691A
:101A40007A652074696D65205B735D00592D6F6642
:101A500066736574205B73746570735D00582D6FD9
:101A60006666736574205B73746570735D005049BE
:101A700044206D61782076616C7565205B302D3275
:101A800035355D0050494420442D6761696E005032
:101A9000494420492D6761696E0050494420502D0A
:101AA0006761696E2F646561642D74696D650050AE
:101AB0004944206472697665206D696E005049441E
:101AC000206472697665206D6178006865617420B4
:101AD0006D616E61676572205B302D335D006163FF
:101AE00063656C65726174696F6E205B6D6D2F73D9
:101AF0005E325D0073746172742066656564726144
:101B00007465205B6D6D2F735D006D61782E2066AE
:101B100065656472617465205B6D6D2F735D007324
:101B20007465707320706572206D6D00426564206D
:101B3000504944206D61782076616C7565205B307A
:101B40002D3235355D004265642050494420442DD6
:101B50006761696E004265642050494420492D67E1
:101B600061696E004265642050494420502D6761D0
:101B7000696E00426564205049442064726976654C
:101B8000206D696E0042656420504944206472698A
:101B90007665206D61780042656420486561742037
:101BA0004D616E61676572205B302D335D00436F60
:101BB00072722E20646961676F6E616C2043205BD6
:101BC0006D6D5D00436F72722E20646961676F6E88
:101BD000616C2042205B6D6D5D00436F72722E2040
:101BE000646961676F6E616C2041205B6D6D5D00A3
:101BF0004D6178207072696E7461626C65207261EB
:101C000064697573205B6D6D5D00546F776572203C
:101C10005A20656E6473746F70206F6666736574A6
:101C2000205B73746570735D00546F776572205923
:101C300020656E6473746F70206F666673657420C0
:101C40005B73746570735D00546F77657220582004
:101C5000656E6473746F70206F6666736574205B65
:101C600073746570735D005365676D656E74732F73
:101C70007320666F722074726176656C00536567BD
:101C80006D656E74732F7320666F72207072696E4B
:101C900074696E6700486F72697A6F6E74616C2048
:101CA000726F642072616469757320617420302CD6
:101CB00030205B6D6D5D00446961676F6E616C2003
:101CC000726F64206C656E677468205B6D6D5D007B
:101CD000486F6D696E672066656564726174652022
:101CE0005B6D6D2F735D004D61782E2066656564B8
:101CF00072617465205B6D6D2F735D005374657048
:101D00007320706572206D6D0054726176656C2071
:101D1000616363656C65726174696F6E205B6D6D84
:101D20002F735E325D00416363656C657261746937
:101D30006F6E205B6D6D2F735E325D004D61782E8E
:101D4000206A65726B205B6D6D2F735D005A206D8C
:101D50006178206C656E677468205B6D6D5D0059FD
:101D6000206D6178206C656E677468205B6D6D5DB9
:101D70000058206D6178206C656E677468205B6D1B
:101D80006D5D005A20686F6D6520706F73205B6D0C
:101D90006D5D005920686F6D6520706F73205B6DFD
:101DA0006D5D005820686F6D6520706F73205B6DEE
:101DB0006D5D0053746F7020737465707065722070
:101DC000616674657220696E61637469766974799D
:101DD000205B6D732C303D6F66665D004D61782E23
:101DE00020696E6163746976652074696D65205B36
:101DF0006D732C303D6F66665D005072696E746560
:101E00007220616374697665205B735D0046696C5E
:101E1000616D656E74207072696E746564205B6DAF
:101E20005D00416476616E63656420557365720080
:101E30004261756472617465004550523A33200006
:101E40004550523A3220004550523A312000455018
:101E5000523A30200050726F746F636F6C20766559
:101E60007273696F6E206368616E6765642C20759C
:101E70007067726164696E6700436F6E666967754B
:101E8000726174696F6E20726573657420746F205F
:101E900064656661756C74732E00436F6E66696766
:101EA00075726174696F6E206C6F61646564206621
:101EB000726F6D20454550524F4D2E00436F6E6638
:101EC000696775726174696F6E2073746F7265648F
:101ED00020746F20454550524F4D2E004175746F50
:101EE0006C6576656C206163746976652028312F96
:101EF0003029005A2D70726F6265205933005A2DB7
:101F000070726F6265205833005A2D70726F62656F
:101F1000205932005A2D70726F6265205832005A73
:101F20002D70726F6265205931005A2D70726F6288
:101F300065205831005A2D70726F626520782D79B6
:101F40002D7370656564205B6D6D2F735D005A2D78
:101F500070726F6265207370656564205B6D6D2FB4
:101F6000735D005A2D70726F6265206F66667365CF
:101F7000742079205B6D6D5D005A2D70726F626503
:101F8000206F66667365742078205B6D6D5D004D13
:101F900061782E207A2D70726F6265202D20626527
:101FA0006420646973742E205B6D6D5D005A2D7022
:101FB000726F626520686569676874205B6D6D5D2E
:101FC0000077616974005072696E7465722068658B
:101FD000696768743A005A2D70726F626520666195
:101FE000696C6564005472616E73666F726D6174C2
:101FF000696F6E206D61747269783A004175746F13
:102000006C6576656C696E672064697361626C6586
:1020100064004175746F6C6576656C696E672065E8
:102020006E61626C6564004175746F6C6576656C99
:10203000206D617472697820726573657400004761
:1020400032382F6E47315A32352F6E005A2D70724A
:102050006F62652073746174653A005265736574CC
:10206000205A20686569676874005A2D70726F6223
:102070006520617665726167652068656967687467
:102080003A00205374657020566172696174696FFB
:102090006E2066726F6D2050726F626520746F20C3
:1020A0006265642044697374616E63653A005A2DF9
:1020B00070726F62653A005072696E746572207357
:1020C000657420696E746F206472792072756E2059
:1020D0006D6F646520756E74696C207265737461D0
:1020E000727421003A20776F726B696E67003A2034
:1020F00074656D702073656E736F722064656665BC
:102100006374006578747275646572200068656137
:1021100074656420626564004D54454D503A00502A
:102120004944204175746F74756E652066696E69E7
:1021300073686564202120506C6163652074686554
:10214000204B702C204B6920616E64204B6420630F
:102150006F6E7374616E747320696E20746865208D
:10216000436F6E66696775726174696F6E2E682061
:102170006F7220454550524F4D00504944204175E3
:10218000746F74756E65206661696C656421207476
:10219000696D656F757400504944204175746F74A2
:1021A000756E65206661696C6564212054656D708B
:1021B0006572617475726520746F20686967680064
:1021C000204B643A2000204B693A2000204B703AA3
:1021D000200020436C6173736963205049440020E0
:1021E00054753A2000204B753A2000206D61783AF2
:1021F0002000206D696E3A200020643A20002062A1
:102200006961733A2000504944204175746F7475B8
:102210006E652073746172740054617267657442F4
:1022200065643A0054617267657445787472004E53
:102230006F206D6F766520696E2064656C74612017
:102240007365676D656E742077697468203E203110
:10225000207365676D656E742E20546869732073F2
:10226000686F756C64206E65766572206861707049
:10227000656E20616E64206D6179206361757365A0
:1022800020612070726F626C656D210044656C7412
:10229000612052616469757320432830293A0044F3
:1022A000656C74612052616469757320422830291D
:1022B0003A0044656C746120526164697573204111
:1022C0002830293A00416C70686120432839302950
:1022D0003A00416C706861204228333330293A005B
:1022E000416C706861204128323130293A00546FC6
:1022F00077657220333A00546F77657220323A0066
:10230000546F77657220313A00496E76616C69646A
:102310002064656C746120636F6F7264696E6174B0
:1023200065202D206D6F76652069676E6F7265641C
:10233000006C696E656172204C3A00454550524F01
:102340004D2075706461746564002C207370656540
:10235000643D00206C696E656172207374657073F2
:102360003A004A65726B3A007A5F6D61783A00799B
:102370005F6D61783A00785F6D61783A004C2000BB
:10238000482000206973200020746F20005365747A
:10239000206F75747075743A20004D53312C4D5375
:1023A000322050696E730045313A0045303A005A88
:1023B0003A00593A0020002C00206D696E00206818
:1023C0006F7572732000206461797320006D2000A6
:1023D0005072696E74696E672074696D653A005059
:1023E00072696E7465642066696C616D656E743ABD
:1023F0000046616E73706565643A00482E20526134
:10240000646975733A00466C6F774D756C746970CA
:102410006C793A0053706565644D756C7469706CC5
:10242000793A00202F002F003A0020524157002017
:1024300042403A0020403A0020423A00543A0020FC
:10244000453A00205A3A0020593A0020583A00589C
:102450003A00467265652052414D3A00556E6B6EEA
:102460006F776E20636F6D6D616E643A00536F66B7
:102470007477617265205265736574005761746387
:1024800068646F672052657365740042726F776E7F
:10249000206F757420526573657400457874657299
:1024A0006E616C20526573657400506F776572556C
:1024B0007000737461727400424C4B2000736B693E
:1024C00070200020676F7420004572726F723A6549
:1024D00078706563746564206C696E652000534490
:1024E0002072656164206572726F72002052002054
:1024F0004A0020490020500020530020460020457B
:1025000000205A00205900205800446F6E6520704A
:1025100072696E74696E672066696C6500466F72D9
:102520006D6174206572726F720057726F6E6720F2
:10253000636865636B73756D004563686F3A00523D
:102540006573656E643A005761726E696E673A0032
:10255000496E666F3A004572726F723A00494E4694
:10256000004E414E006F6B004649524D5741524557
:102570005F4E414D453A52657065746965725F30D2
:102580002E39322E32204649524D574152455F4432
:102590004154453A3230313731313133204D4143A6
:1025A00048494E455F545950453A526F73746F63B2
:1025B0006B204D415820763320005265717565734C
:1025C0007450617573653A004D31313720494E536F
:1025D0004552542053442043415244004D31313739
:1025E0002053442043415244204552524F520055FB
:1025F000495F414354494F4E5F5345545F4D4541F8
:1026000053555245445F4F524947494E20004E6F43
:1026100020534420436172640053687574204F66F0
:102620006620414C4C2048656174730050726568A7
:102630006561742041425300507265686561742081
:10264000504C410055495F414354494F4E5F484FFC
:102650004D455F5A200055495F414354494F4E5FF5
:10266000484F4D455F59200055495F414354494FFC
:102670004E5F484F4D455F58200055495F414354D8
:10268000494F4E5F484F4D45414C4C200055495FE6
:10269000414354494F4E5F5A504F534954494F4E4E
:1026A0005F464153545F4E4F5445535420005549A3
:1026B0005F414354494F4E5F5A504F534954494F1D
:1026C0004E5F4E4F54455354200055495F4143548B
:1026D000494F4E5F45504F534954494F4E20005586
:1026E000495F414354494F4E5F5A504F53495449F3
:1026F0004F4E5F46415354200055495F4143544972
:102700004F4E5F59504F534954494F4E5F464153C6
:1027100054200055495F414354494F4E5F58504F34
:10272000534954494F4E5F46415354200055495F29
:10273000414354494F4E5F5A504F534954494F4EAD
:10274000200055495F414354494F4E5F59504F5304
:102750004954494F4E200055495F414354494F4E1B
:102760005F58504F534954494F4E200042616E67A5
:1027700042616E6700536C6F7742616E670044651B
:1027800061642054696D650050494400003A00209E
:1027900064617973200050657263656E74205072B5
:1027A000696E7465643A00206465662000465720AF
:1027B0004461746520323031373131313300526F2A
:1027C00073746F636B4D41587633005365654D6587
:1027D000434E4300526F73746F636B204D4158201A
:1027E00076330064341A34AD335033416374696F07
:1027F0006E3A256C6100040003004E6F005965734A
:10280000004E2F41004F6666004F6E000000003FF3
:10281000CDCC4C3D0AD7A33B6F12033A526570658D
:1028200074696572207620302E39322E32000040D5
:1028300014548025000040380000004B00008070D8
:10284000000000960000C0DA000000E10000002C4B
:10285000010008B2010000C2010000F40100008480
:10286000030090D0030000E803000008070020A147
:10287000070000100E0040420F0060E31600000049
:102880000000110A0411040A1111001C1F11111F6C
:102890000000040A0A0A0E1F1F0E001F1111111F4B
:1028A0000000001F1F1F1F1F0000040A040000007B
:1028B0000000040E15041C0000000200000600C108
:1028C00028D7302729A82DFA28FB2D6929020000D6
:1028D0000700D428D730E228A82DFA28FB2D332D65
:1028E0000E29E92802A92E00005072696E746572E3
:1028F0002053657474696E6773000129027B2F0091
:102900000041646A7573742054656D7073001529F5
:10291000023F290000416476616E6365642053655F
:102920007474696E6773002E2902C02E0000507205
:10293000696E7465722053657474696E6773000202
:10294000000009004629D730542A402A302A202A7C
:102950005829092AF12969295F2902D62C00004447
:102960006562756767696E6700702902B82F00009D
:1029700043616C6962726174696F6E204D656E753A
:10298000000310270200882993298C299A29000026
:10299000000000AB2900000000006C6F61646564FA
:1029A00020662E20454550524F4D00436F6E66699C
:1029B0006775726174696F6E000310270200C02989
:1029C000CB29C429D2290000000000E3290000001F
:1029D000000073746F72656420696E204545505223
:1029E0004F4D00436F6E66696775726174696F6EF3
:1029F00000F82903070400004C6F61642066726FC1
:102A00006D20454550524F4D00102A03060400002A
:102A100053746F726520746F20454550524F4D00BE
:102A2000272A02632A000045787472756465720073
:102A3000372A026A2C00004665656472617465007D
:102A4000472A02962C0000416363656C65726174CD
:102A5000696F6E005B2A02B62B000047656E6572D7
:102A6000616C0002000010006A2AD730A22B8E2B66
:102A70007C2B6B2B562B272B3F2B102BFD2AE92A67
:102A8000D82AC72AB22A9D2A8A2A912A042F04000A
:102A900000504944204D61783A25584400A42A0446
:102AA000260400004472697665204D61783A255805
:102AB0004D00B92A04250400004472697665204D52
:102AC000696E3A25586D00CE2A042404000050494E
:102AD0004420443A25586400DF2A042304000050AF
:102AE000494420493A25586900F02A04220400008C
:102AF00044542F50494420503A25587000042B0468
:102B00002D040000436F6E74726F6C3A2558680094
:102B1000172B0446040000416476616E6365206CE7
:102B2000696E3A25586C002E2B044D040000576145
:102B3000697420556E6974733A2558556D6D004659
:102B40002B044C040000576169742054656D702E8D
:102B50002558540243005D2B042E04000053746179
:102B6000622E54696D653A25587700722B042A0449
:102B70000000416363656C3A25584100832B042BA8
:102B80000400004D61782046523A25584600952BA6
:102B9000042C04000053746172742046523A255884
:102BA0006600A92B042904000053746570732F4D2F
:102BB0004D3A255365000200000400BD2BD730F2CA
:102BC0002BDA2BC52BCC2B02062C00004D61782E66
:102BD00020496E61637469766500E12B02382C0030
:102BE000005374657070657220496E616374697614
:102BF0006500F92B04100400004261756472617471
:102C0000653A256F630003580402000D2C182C113F
:102C10002C1F2C0000000000292C00000000005B8D
:102C2000735D20303D4F6666004469732E20416617
:102C30007465723A2569700003200402003F2C4A33
:102C40002C432C512C00000000005B2C00000000E5
:102C5000005B735D20303D4F6666004469732E2033
:102C600041667465723A25697300020000030071C1
:102C70002CD730872C772C7E2C0413040000486F4F
:102C80006D653A25665A008E2C04160400004D61CD
:102C9000783A25667A0002000004009D2CD730C5E2
:102CA0002CB52CA52CAC2C040E0400004A65726BCC
:102CB0003A25616A00BC2C040D0400004D6F766556
:102CC0003A25615A00CC2C040A0400005072696E47
:102CD000743A25617A000200000500DD2CD730200F
:102CE0002D0D2DFA2CE72CEE2C0335040000447238
:102CF000792072756E3A25646400012D0334040056
:102D0000004572726F7273203A25646500142D03BA
:102D100033040000496E666F2020203A2564690064
:102D2000272D03320400004563686F2020203A25D8
:102D3000646F003A2D02472D000053442043617216
:102D400064204D656E750002000006004E2DD730E0
:102D5000A82D952D7F2D6D2D5A2D612D03F4030186
:102D60000244656C6574652066696C6500742D02AB
:102D7000C72D020053746F70205072696E74008604
:102D80002D03F7030400436F6E74696E7565205060
:102D900072696E74009C2D03F60302045061757312
:102DA00065205072696E7400AF2D03F50301025364
:102DB000656C6563742053442046696C65000100AE
:102DC000000100C52DD7300200000300CE2DE92DF3
:102DD000DF2DD42DDB2D035424020059657300E64A
:102DE0002D03E80300004E6F00F02D0100000000ED
:102DF00053746F70205072696E7400022E02132E8D
:102E0000000041646A7573742046616E20737065BA
:102E100065640002000007001A2ED730912E7D2E27
:102E2000682E532E3E2E282E2F2E031E04000053F4
:102E300065742046616E2031303025252500452EF1
:102E4000031D0400005365742046616E203735254C
:102E50002525005A2E031C0400005365742046618A
:102E60006E203530252525006F2E031B04000053EE
:102E700065742046616E20323525252500842E0399
:102E80001A0408005475726E2046616E204F666603
:102E900000982E045204000046616E207370656530
:102EA000643A254673252525000200000900B02E4E
:102EB000D7300A2FF12E682F552F3B2FC330232FE9
:102EC0000200000900C72ED7300A2FF12E682F55B7
:102ED0002F3B2FC330D92E232FE02E03B20F00003B
:102EE000556E6C6F636B2046756C6C204D656E750E
:102EF00000F82E0448040000466C6F7720205261D1
:102F000074653A256F6625252500112F041F0400DE
:102F100000537065656420526174653A256F6D25B4
:102F20002525002A2F034204001044697361626C56
:102F30006520537465707065727300422F03380406
:102F4000000053687574204F666620414C4C204841
:102F500065617473005C2F0347040000507265685C
:102F600065617420414253006F2F03370400005005
:102F700072656865617420504C41000200000400D5
:102F8000822FD730A02F882F8F2F043C04000042BF
:102F900045442054656D703A202025456202430067
:102FA000A72F043D0400004E4F5A2054656D703A1F
:102FB00020202545300243000200000600BF2FD725
:102FC00030F52FCB2FC3308D30E12FD22F042104C9
:102FD0000000482E20526164697573203A256F689D
:102FE00000E82F03AC0F0000536574205A204F7285
:102FF0006967696E00FC2F020D30000046756C6C2D
:103000002043616C6962726174696F6E0002000036
:1030100004001430D7304A3035301C30233003B12F
:103020000F0000426567696E2043616C69627261DE
:1030300074696F6E003C3003B50F000042454420B8
:1030400041524520434C45414E00513003B40F00DE
:10305000004D414B452053555245204E4F5A5A4C36
:103060004520260002000006006B30D730C330B187
:10307000309F308D3077307E3002F0300000457860
:1030800074722E20706F736974696F6E00943002D1
:10309000513200005A20506F736974696F6E00A638
:1030A0003002A63200005920506F736974696F6E48
:1030B00000B83002FB3200005820506F7369746909
:1030C0006F6E00CA3003FD030000486F6D6520502D
:1030D00072696E74657200DE3003E803000050729E
:1030E0006576696F75732053637265656E200100A4
:1030F00003F0030400F73014310D310631FF301BAB
:10310000310000000000293100000000003A3100C9
:103110000000000049310000000000255566206DC8
:10312000207072696E7465640020453A2565632FCE
:1031300025456302437E256F43003120636C69633C
:103140006B203D2031206D6D00453A257833206D90
:103150006D0003FC030400593176316F3168316131
:10316000317D3100000000007E3100000000008E43
:103170003100000000009E310000000000004D61A1
:103180007820656E6473746F703A25735A004D69C8
:103190006E20656E6473746F703A25737A005A3AC4
:1031A000257832206D6D0003FB030400AE31CB3176
:1031B000C431BD31B631D2310000000000D331003E
:1031C00000000000E3310000000000F331000000C7
:1031D0000000004D617820656E6473746F703A254D
:1031E0007359004D696E20656E6473746F703A2573
:1031F000737900593A257831206D6D0003FA030484
:103200000003322032193212320B32273200000012
:1032100000002832000000000038320000000000EA
:1032200048320000000000004D617820656E647334
:10323000746F703A257358004D696E20656E647323
:10324000746F703A25737800583A257830206D6D88
:103250000003EF030400583275326E326732603279
:103260007C3200000000007D3200000000008D3242
:1032700000000000009D320000000000004D617859
:1032800020656E6473746F703A25735A004D696ED1
:1032900020656E6473746F703A25737A005A3A250C
:1032A0007832206D6D0003EE030400AD32CA32C3E4
:1032B00032BC32B532D1320000000000D232000000
:1032C000000000E2320000000000F23200000000C6
:1032D00000004D617820656E6473746F703A2573D9
:1032E00059004D696E20656E6473746F703A257372
:1032F0007900593A257831206D6D0003ED03040003
:1033000002331F33183311330A3326330000000011
:1033100000273300000000003733000000000047A2
:10332000330000000000004D617820656E64737406
:103330006F703A257358004D696E20656E64737422
:103340006F703A25737800583A257830206D6D00FB
:103350000000000400573374336D3366335F337BF2
:1033600033000000000081330000000000953300AE
:103370000000000099330000000000255566206D14
:1033800000546F74616C2046696C616D656E7420C9
:10339000557365640025557400546F74616C20503A
:1033A00072696E74696E672054696D650000000073
:1033B0000400B433D133CA33C333BC33D833000031
:1033C000000000E7330000000000F53300000000BB
:1033D0000007340000000000526F73746F636B20AD
:1033E0004D4158207633005072696E746572204DDD
:1033F0006F64656C00465720446174653A20323032
:103400003137313131330046572056657273696F59
:103410006E3A20302E39322E320000000004002196
:10342000343E343734303429344534000000000051
:1034300049340000000000523400000000005B34FA
:103440000000000000256F73005A3A257832206D85
:103450006D00593A257831206D6D00583A25783045
:10346000206D6D0000000004006B34883481347AD4
:103470003473348F340000000000933400000000E7
:1034800000AC340000000000BF3400000000002544
:103490006F730053706565643A256F6D252525208F
:1034A000466C6F773A256F66252525004245443ADC
:1034B000256562205461726765743A254562004E45
:1034C0004F5A3A256563205461726765743A254501
:1034D00063000000000000000000000000FF00008A
:1034E00001000000000000000000000000000000DB
:1034F000000024F403D950C38EB1C2A23D96828B42
:103500003582127AE372816CCB66A861015DC7587F
:10351000EB546151204E1E4B5648C14559431A4148
:10352000013F093D2F3B7139CD374036C9346533F2
:103530001432D430A32F802E6B2D632C672B752A69
:103540008E29B028DC2710274B268F25D9242B2441
:103550008223E0224322AC211A218D200420801FE7
:10356000001F841E0C1E971D261DB81C4E1CE61B3A
:10357000821B201BC11A641A0A1AB2195D190A1992
:10358000B9186A181C18D11788174017FA16B516FB
:1035900073163116F115B31576153A150015C714C3
:1035A0008F1458142214EE13BA13881356132513CC
:1035B000F612C71299126C1240121512EB11C111BA
:1035C0009811701148112111FB10D610B1108D10F7
:1035D0006910461024100210E10FC00FA00F800FD9
:1035E000610F420F230F060FE80ECB0EAF0E930EA6
:1035F000770E5C0E410E270E0D0EF30DDA0DC10D88
:10360000A80D900D780D600D490D320D1B0D050DA7
:10361000EF0CD90CC30CAE0C990C850C700C5C0C27
:10362000480C350C210C0E0CFB0BE80BD60BC40B15
:10363000B20BA00B8E0B7D0B6B0B5A0B4A0B390B8D
:10364000290B180B080BF80AE90AD90ACA0ABB0A9F
:10365000AC0A9D0A8E0A800A710A630A550A470A53
:10366000390A2C0A1E0A110A040AF709EA09DD09B7
:10367000D009C409B709AB099F09920987097B09D9
:103680006F09630958094C09410936092B092009BA
:1036900015090A090009F508EB08E008D608CC0866
:1036A000C208B808AE08A4089A08900887087D08E0
:1036B00074086B08610858084F0846083D0834082C
:1036C0002C0823081A08120809080108F807F0074F
:1036D000E807E007D807D007C807C007B807B00752
:1036E000A807A1070000420FA1071605D0030D038C
:1036F0008B022E02E801B2018601630145012C0113
:1037000017010401F400526F73746F636B4D4158DD
:1037100020526561647900526F73746F636B4D4121
:103720005820526561647900526F73746F636B4DFA
:10373000415820526561647900207A3A0020793A34
:103740000020783A00696E20717565756544656C76
:1037500074614D6F766520746F2063616C63756C66
:1037600061746544656C74615375625365676D651A
:103770006E74732072657475726E73206572726FE9
:10378000722E00432068697420666C6F6F7200436C
:10379000706F7320782073717561726520004370BB
:1037A0006F732078207374657073200043706F739B
:1037B000207920737175617265200043706F7320EA
:1037C00079207374657073200042206869742066E4
:1037D0006C6F6F720042706F732078207371756127
:1037E0007265200042706F73207820737465707367
:1037F000200042706F7320792073717561726520AB
:103800000042706F732079207374657073200041DB
:103810002068697420666C6F6F720041706F73204E
:103820007820737175617265200041706F73207824
:10383000207374657073200041706F73207920735A
:103840007175617265200041706F73207920737407
:1038500065707320006D6F766552656C6174697672
:103860006544697374616E6365496E537465707302
:10387000202F20717565756544656C74614D6F7698
:10388000652072657475726E73206572726F720056
:1038900000000A0B02090C0D0E08070304010000CA
:1038A0000000000000000000000000000000000018
:1038B00000000000000000000000000012111000D5
:1038C00000000000000000000000000000000000F8
:1038D0000000000000000102102020080810204015
:1038E00010204080020102010804020101020408C4
:1038F0001020408080402010080402018004020152
:10390000804020100804020108040201010204089A
:1039100010204080010204081020408005050505A4
:10392000070508080808020202020A0A0808040437
:103930000404010101010101010103030303030365
:103940000303040707070C0C0C0C0C0C0C0C0202F4
:10395000020206060606060606060B0B0B0B0B0BF1
:103960000B0B000020002300260029002C002F0054
:1039700032000001000003010601090100002200DD
:10398000250028002B002E00310034000201000029
:10399000050108010B0100002100240027002A0076
:1039A0002D003000330001010000040107010A016D
:1039B000024E414E494E495459494E46CDCCCC3D1C
:1039C0000AD7233C17B7D13877CC2B329595E6240C
:1039D0001FB14F0A000020410000C84200401C46B1
:1039E00020BCBE4CCA1B0E5AAEC59D744790809F2A
:1039F0002DDEB80111241FBECFEFD1E2DEBFCDBF57
:103A000000E00CBF13E0A0E0B2E0E4EFF4E202E07B
:103A10000BBF02C007900D92A039B107D9F72EE174
:103A2000A0E9B3E001C01D92A938B207E1F719E39C
:103A3000C4EFD9E300E006C022970109FE010BBFE5
:103A40000F94F30DCC3ED10780E00807A9F70F943F
:103A50005F090D9478120C940000CF93DF9300D08F
:103A60001F92CDB7DEB744E050E0BC01CE01019615
:103A70000F94341269817A818B819C810F900F9011
:103A80000F900F90DF91CF91089522E090E02817DA
:103A900028F4963019F0220F9F5FF9CF209A289AC8
:103AA000219A229A2398809164008B7F80936400EE
:103AB000892F806A86958CBD90FD03C081E0963089
:103AC00009F480E08DBD08958091EA0283FB882788
:103AD00080F90895179A0895169A0895159A0895E9
:103AE00080B182FB882780F9089580B18695817026
:103AF000089588E493E0B1CFCF92DF92EF92FF92E6
:103B0000CF93DF9300D01F921F92CDB7DEB76B012A
:103B10007C0160937707709378078093790790937F
:103B20007A070E94E774C982DA82EB82FC8244E061
:103B300050E065E773E0CE0101960F94561223E042
:103B4000B701A60188E795E00E949BA10E9444CF9F
:103B5000682F88E690E06D830F9444126D8168179A
:103B600021F088E690E00F945F120F900F900F9075
:103B70000F900F90DF91CF91FF90EF90DF90CF905B
:103B80000895CF93DF931F92CDB7DEB7BC018DE7C9
:103B900093E00F9472120E9444CF682F88E690E061
:103BA00069830F9444126981681739F088E690E0C0
:103BB0000F90DF91CF910D945F120F90DF91CF9115
:103BC0000895CF93DF931F92CDB7DEB7BC018FE787
:103BD00093E00F9472120E9444CF682F88E690E021
:103BE00069830F9444126981681739F088E690E080
:103BF0000F90DF91CF910D945F120F90DF91CF91D5
:103C00000895CF93DF931F92CDB7DEB7BC0181E853
:103C100093E00F9472120E9444CF682F88E690E0E0
:103C200069830F9444126981681739F088E690E03F
:103C30000F90DF91CF910D945F120F90DF91CF9194
:103C40000895CF93C82F8091A6048823D1F01092B5
:103C5000A6040E942C5A9091DF0291509093DF02AB
:103C6000911109C08091E002833010F40E94B9598B
:103C700085E08093DF026C2F86E79AE0CF910C9469
:103C800079CACF91089580912C0C882349F00E9425
:103C9000649880E0D6DF86E79AE00E9478CAF3CF86
:103CA00008954F925F926F927F928F929F92AF9200
:103CB000BF92CF92DF92EF92FF920F931F93CF9319
:103CC000DF9300D01F92CDB7DEB78C018091F10752
:103CD0009091F207A091F307B091F40789839A833A
:103CE000AB83BC83C090F507D090F607E090F70750
:103CF000F090F8078090F9079090FA07A090FB07E2
:103D0000B090FC079C01AD01BC01CD010F94250DC5
:103D100081110FC149805A806B807C80E89477F8CC
:103D20002FEF3FEF4FE75FE7C301B2010F94250D7F
:103D300081110BC02FEF3FEF4FE75FE7C301B201E7
:103D40000F94D20918160CF4F4C0A7019601C7010C
:103D5000B6010F94250D8111ECC026013701E894BE
:103D600077F82FEF3FEF4FE75FE7C301B2010F9402
:103D7000250D81110BC02FEF3FEF4FE75FE7C30128
:103D8000B2010F94D20918160CF4D3C0A501940106
:103D9000C501B4010F94250D8111CBC0240135015B
:103DA000E89477F82FEF3FEF4FE75FE7C301B201E9
:103DB0000F94250D81110BC02FEF3FEF4FE75FE709
:103DC000C301B2010F94D20918160CF4B2C02091AD
:103DD000C9073091CA074091CB075091CC07698140
:103DE0007A818B819C810F946E092B013C0120917B
:103DF000CD073091CE074091CF075091D007C70132
:103E0000B6010F946E096B017C012091D1073091AE
:103E1000D2074091D3075091D407C501B4010F9444
:103E20006E094B015C0180915108882329F020E73D
:103E300032E441E25DE304C020E030E040E85FE3CB
:103E4000C301B2010F947A0CAB01BC0122E08FE4F4
:103E500094E20E94D8A180915108882329F020E79C
:103E600032E441E25DE304C020E030E040E85FE39B
:103E7000C701B6010F947A0CAB01BC0122E087E4C4
:103E800094E20E94D8A180915108882329F020E76C
:103E900032E441E25DE304C020E030E040E85FE36B
:103EA000C501B4010F947A0CAB01BC0123E083E49B
:103EB00094E20E94D8A16091090870910A0880914B
:103EC0000B0890910C080F94A50A20914D08309191
:103ED0004E0840914F08509150080F947A0C209151
:103EE0005108222329F020E732E441E25DE304C0D7
:103EF00020E030E040E85FE30F947A0CAB01BC01B6
:103F000024E08FE394E20F900F900F900F90DF91D9
:103F1000CF911F910F91FF90EF90DF90CF90BF90C6
:103F2000AF909F908F907F906F905F904F900C9488
:103F30009BA1C8010E94BD9F4ACFCF92DF92EF9212
:103F4000FF92CF93DF93EC01893191053CF0C53F9F
:103F500081E0D8072CF0C4EFD1E002C0C9E1D0E085
:103F6000BE01882777FD8095982F0F94A50A6B01D5
:103F70007C016091010770910207882777FD809589
:103F8000982F0F94A50A9B01AC01C701B6010F94AD
:103F9000D9099B01AC0160910307709104078091DE
:103FA0000507909106070F947A0C609303077093AE
:103FB00004078093050790930607D0930207C093E8
:103FC0000107BE0184E194E2DF91CF91FF90EF9071
:103FD000DF90CF900C9481A0CF92DF92EF92FF926E
:103FE0006B017C0120E030E040E752E40F94D209FD
:103FF00087FD11C020E030E046E153E4C701B6017F
:104000000F94060C18166CF4C12CD12C86E1E82E06
:1040100083E4F82E06C0C12CD12C90E7E92E92E45F
:10402000F92EC0927707D0927807E0927907F09244
:104030007A0722E0B701A6018BEF93E2FF90EF90A1
:10404000DF90CF900C949BA18F929F92AF92BF92E2
:10405000CF92DF92EF92FF92CF93DF93EC01893101
:10406000910534F0893C91052CF0C8ECD0E002C0F9
:10407000C9E1D0E0D0930007C093FF06E091900320
:10408000F0919103E258FF4FC080D180E280F3802D
:1040900020E030E0A901C701B6010F94D209AE01BA
:1040A000662757FD6095762F18165CF0CB01BA0194
:1040B0000F94A50A2AE037ED43E25CE30F947A0CF3
:1040C00024C0CB01BA010F94A50A2AE037ED43E2E0
:1040D0005CE30F947A0C20E030E040E850E40F9469
:1040E0007A0C4B015C01A7019601C701B6010F9440
:1040F0007A0C2BED3FE049E450E40F947A0C9B01DD
:10410000AC01C501B4010F94D9096093E502709325
:10411000E6028093E7029093E802BE0186E094E213
:10412000DF91CF91FF90EF90DF90CF90BF90AF9055
:104130009F908F900C9481A0CF93DF932091C5071F
:1041400097FD0DC0EC018F3F910519F014F0CFEFF2
:10415000D0E0209721F028602093C50705C0277F75
:104160002093C507C0E0D0E061118DDD8091851DF1
:1041700090E0C817D90729F0BE0181EF93E20E94B1
:1041800081A0C093851DDF91CF9108954F925F92DA
:104190006F927F928F929F92AF92BF92CF92DF9257
:1041A000EF92FF92CF93DF9300D01F92CDB7DEB78F
:1041B0002FE632E143E85AE36091E9067091EA069E
:1041C0008091EB069091EC060F947A0C6B017C01C8
:1041D00081E890E042DC9B01AC01C701B6010F947D
:1041E0006E09AB01BC0122E08FED93E20E94D8A1E1
:1041F0008DEC93E20E94839FE0910A02F0910B0202
:1042000020E030E040E751E463857485858596853C
:104210000F94060C18160CF46BC020E030E0A901D6
:104220008DE790E029833A834B835C830F944C1293
:104230004B015C0129813A814B815C81820E931E86
:10424000A41EB51EC501B40120E831E541E050E0EF
:104250000F94A60D60E87EEA8EEF9FEF0F94410D5C
:104260006B017C01C80CD91CEA1CFB1CBA01A9011A
:1042700080ED93E20E94A7A0C701B60120E13EE0D5
:1042800040E050E00F94A60D49015A01BA01A9017E
:1042900086EC93E20E94A7A0A0EFB1EFA5019401E4
:1042A0000F94EF0D6C0D7D1D8E1D9F1D2CE330E0D6
:1042B00040E050E00F94A60DBA01A9018EEB93E205
:1042C0000E94A7A089EB93E20F900F900F900F90A0
:1042D000DF91CF91FF90EF90DF90CF90BF90AF90A4
:1042E0009F908F907F906F905F904F900C949C9FC9
:1042F0000F940904C090ED06D090EE06E090EF0612
:10430000F090F0066C197D098E099F0928EE33E0C4
:1043100040E050E00F94840D83CF5F988EBD0DB4C4
:1043200007FEFDCF6EBD0DB407FEFDCF5F9A089569
:10433000CF93DF9300D01F921F92CDB7DEB795E0E9
:10434000E7E4F3E0DE01119601900D929A95E1F712
:10435000E1E0F0E0EC0FFD1FE80FF11D808190E03F
:104360000F900F900F900F900F90DF91CF91D5CFBE
:10437000FF920F931F93CF93DF9300D01F921F9252
:10438000CDB7DEB785E0ECE4F3E0DE0111960190F5
:104390000D928A95E1F780E078DB579A8E010F5FE6
:1043A0001F4FF12CF80161918F0170E08F2DC0DF5C
:1043B000F394F5E0FF12F6CF0F900F900F900F904F
:1043C0000F90DF91CF911F910F91FF90089567FD9E
:1043D00043C08230E9F028F4882341F0813061F055
:1043E0003BC0833009F1843059F136C0662311F0A7
:1043F000A19A67C0A19865C080910801662311F059
:10440000806801C08F778093080147FF3AC05DC084
:1044100080910801662311F0806401C08F7B809336
:10442000080147FF34C053C080910801662311F092
:10443000886001C0877F8093080147FF32C044C075
:1044400080910801662311F0826001C08D7F809306
:10445000080147FF2EC03AC047FD39C08230B9F08D
:1044600028F4882341F0813061F008958330C9F049
:104470008430F9F00895442311F0A09A0895A0988B
:104480000895442311F0A29A0895A2980895809166
:104490000801442311F0806201C08F7D80930801E0
:1044A000089580910801442311F08061F7CF8F7E39
:1044B000F5CF80910801442311F08460EFCF8B7F0A
:1044C000EDCF47FFD8CF0895089508950895089532
:1044D000643079F028F4613041F0623041F00895A1
:1044E000683051F0603141F0089540E003C040E091
:1044F00004C041E060E002C041E061E068CFCF93DA
:10450000DF938AE993E20E949C9F62B36695617093
:1045100070E08FE494E20E9475A062B3617070E075
:1045200087EB93E20E9481A0C6E0D1E088819927C1
:1045300087FD9095692F661F6627661F70E082EBE6
:1045400093E20E9475A062B362FB662760F970E097
:1045500087EB93E20E9481A0688166FB662760F981
:1045600070E08FEA93E20E9475A0688165FB662780
:1045700060F970E087EB93E20E9481A0688163FBA1
:10458000662760F970E08BEA93E20E9475A068816B
:104590006295617070E087EB93E20E9481A0688170
:1045A0006695617070E087EA93E20E9475A0688169
:1045B00062FB662760F970E087EB93E2DF91CF91B1
:1045C0000C9481A0FF920F931F93CF93DF9300D0A1
:1045D0001F921F92CDB7DEB785E0E1E5F3E0DE0183
:1045E000119601900D928A95E1F7989A9A9A809186
:1045F00007018062809307018091070180618093A9
:104600000701809107018460809307018E010F5F8D
:104610001F4FF12CF80161918F018F2D59DFF39419
:10462000F5E0FF12F7CF0F900F900F900F900F90C3
:10463000DF91CF911F910F91FF9008950C94DDDAD7
:104640000E94C8DA2091080230910902821793076C
:1046500024F490930902809308020895609108025F
:1046600070910902809106029091070268177907FC
:1046700044F4709307026093060282E594E20C947E
:1046800081A00895CF93C82F69E170E080E99DE192
:104690000F94D9006C2F80E99DE10F947A0060E0BF
:1046A00080E99DE10F94DA00882329F082E59DE0FE
:1046B000CF910C949C9FCF910895CF93DF93D82FE7
:1046C000C62F69E170E080E99DE10F94D9006D2F5C
:1046D00080E99DE10F947A006C2F80E99DE10F94B1
:1046E0007A0080E99DE10F94EC00882331F082E3A9
:1046F0009DE0DF91CF910C949C9FDF91CF91089525
:10470000C1DF41E050E069E170E080E99DE10F9494
:10471000CD0080E99DE10F942300892B31F080E9E1
:104720009DE10F942B0081E0089583E19DE00E94BC
:104730009C9F80E008958EEE9CE00E949C9F80E903
:104740009DE10F94B8008FE0DBDF81E3D9DF80E2E9
:10475000D7DF6CE980E2B1DF80E2D2DF82E2D0DF36
:1047600060E482E2AADF82E2CBDF85E2C9DF60E0BB
:1047700085E2A3DF85E2C4DF83E2C2DF60E383E298
:104780009CDF83E2BDDF84E2BBDF6AE484E295DF85
:1047900084E2B6DF80E3B4DF60E280E38EDF80E3B3
:1047A000AFDF81E3ADDF82E3ABDF64E182E385DF8E
:1047B00082E3A6DF83E3A4DF60E083E37EDF83E3BD
:1047C0009FDF84E39DDF60E084E377DF84E398DFAD
:1047D00086E396DF62E386E370DF86E391DF87E3BB
:1047E0008FDF60E087E369DF87E38ADF88E388DFC4
:1047F00060E188E362DF88E383DF89E381DF8AE3C6
:104800007FDF62E38AE359DF8AE37ACFCF9381E3E4
:1048100077DFC82F85E374DF811101C0C0E089E331
:104820006FDF811101C0C0E08DE26ADF811101C03C
:10483000C0E08C2FCF9108956DE08AE39BE00E9449
:104840007CD96AE08AE39BE00C947CD9CF93C82F93
:10485000E0919003F091910342A953A964A975A92D
:1048600022E08CE394E20E94D8A1E0919003F091C1
:10487000910346A957A960AD71AD20E083E294E2AF
:104880000E94D8A10E94BD51AB01BC0122E088E387
:1048900094E20E94D8A14091190250911A026091AD
:1048A0001B0270911C0220E083E294E20E94D8A1D6
:1048B000CC2391F061E070E08AE294E20E9475A05E
:1048C0006CEF7FE08091110290911202681B790BCE
:1048D00088E294E20E9475A0E0910E02F0E0EE57AB
:1048E000F24E608170E08FE294E20E9475A0E09148
:1048F000DE02EF3F29F4E0919003F0919103E08113
:10490000F0E0EE57F24E608170E084E394E20E94A2
:1049100075A0CF9191CF2F923F924F925F926F925D
:104920007F928F929F92AF92BF92CF92DF92EF923F
:10493000FF920F931F93CF93DF93CDB7DEB72997E5
:104940000FB6F894DEBF0FBECDBF5C01DC0116963A
:104950008D919C9117978C38910509F469C608F0E0
:10496000DBC08235910509F40EC408F07EC08A319F
:10497000910509F4C5C208F03FC08531910509F4DD
:104980003DC278F48231910509F417C28431910552
:1049900009F418C2419711F00C946D3517981698C8
:1049A000AFC58731910509F461C208F443C288316B
:1049B000910509F489C2499711F00C946D3560E0B6
:1049C00082E299E029960FB6F894DEBF0FBECDBF04
:1049D000DF91CF911F910F91FF90EF90DF90CF90DB
:1049E000BF90AF909F908F907F906F905F904F900F
:1049F0003F902F900C94559B8E31910509F4DDC2A8
:104A000018F58C31910509F4B0C210F00C94A6355C
:104A100082E299E029960FB6F894DEBF0FBECDBFB3
:104A2000DF91CF911F910F91FF90EF90DF90CF908A
:104A3000BF90AF909F908F907F906F905F904F90BE
:104A40003F902F900C949C9E8A32910509F40FC3DD
:104A500028F4809709F4DEC20C946D3580359105F9
:104A600010F00C94A6350C946D358B36910511F42D
:104A70000C949B2E38F58C35910509F48FC460F4A5
:104A80008435910509F488C308F481C385359105FF
:104A900009F460C40C946D358836910509F433C56A
:104AA00030F48336910509F4DDC40C946D358936F4
:104AB000910509F410C68A36910511F40C948A2EDA
:104AC0000C946D358337910511F40C94EC2E80F421
:104AD0008F36910511F40C94BC2E8237910511F498
:104AE0000C940A2F8D36910511F00C946D3515C676
:104AF0008537910511F40C940D2F10F40C94142E9D
:104B00008737910511F40C94382F8837910511F4EB
:104B10000C947F2F0C946D358530B1E09B0711F418
:104B20000C948D3208F0B0C08F3C910511F40C94B8
:104B3000273108F041C08A3C910511F40C9456309D
:104B400070F4883C910511F40C94A52F10F00C948E
:104B5000F82F8E3B910509F4B6C70C946D358C3C4B
:104B6000910511F40C94AD3010F40C949B308D3CF5
:104B7000910511F40C940D318E3C910511F00C94BB
:104B80006D35C50129960FB6F894DEBF0FBECDBFB7
:104B9000DF91CF911F910F91FF90EF90DF90CF9019
:104BA000BF90AF909F908F907F906F905F904F904D
:104BB0003F902F900C94E5D58F3D910511F40C9406
:104BC000E23188F48C3D910511F40C948F318D3DC8
:104BD000910511F40C94B731813D910511F00C94BD
:104BE0006D350C946F31893E910511F40C94F731B9
:104BF00040F5883E910511F00C946D3560918A1D49
:104C000070918B1D83E593E20E9475A04091861DF3
:104C10005091871D6091881D7091891D22E08AE462
:104C200093E20E949BA110928B1D10928A1D1092FC
:104C3000861D1092871D1092881D1092891D0C945C
:104C4000A6358B3F910511F40C943032843091409D
:104C500011F00C946D3529960FB6F894DEBF0FBE97
:104C6000CDBFDF91CF911F910F91FF90EF90DF901B
:104C7000CF90BF90AF909F908F907F906F905F90FC
:104C80004F903F902F9057CD8E3521E0920711F431
:104C90000C94E533C0F58E3241E0940711F40C9486
:104CA000303398F48931A1E09A0711F40C94E5327D
:104CB0008C32B1E09B0711F40C94F53286309140B0
:104CC00011F00C946D350C94AF328034F1E09F07F5
:104CD00011F40C94A33338F48F32914011F40C94F6
:104CE0006F330C946D35813441E0940711F40C94CA
:104CF000A7338234914011F00C946D3580E00E940E
:104D0000198C0C94BC338239A1E09A0711F40C94ED
:104D1000D03498F58836E1E09E0711F40C949C3469
:104D200038F48336914011F40C9456340C946D355C
:104D3000803931E0930711F40C94B63481399140F5
:104D400011F00C946D3529960FB6F894DEBF0FBEA6
:104D5000CDBFDF91CF911F910F91FF90EF90DF902A
:104D6000CF90BF90AF909F908F907F906F905F900B
:104D70004F903F902F900C949386853F51E095077C
:104D800011F40C94003560F4843F914011F00C94C0
:104D90006D3580E00E945BCF8CEB9EE10C940B356F
:104DA000863FE1E09E0711F40C9425358C38934042
:104DB00011F40C943F350C946D350E946A1D0E94CD
:104DC0006C1D77C282E299E029960FB6F894DEBF97
:104DD0000FBECDBFDF91CF911F910F91FF90EF904C
:104DE000DF90CF90BF90AF909F908F907F906F900B
:104DF0005F904F903F902F900C94E59D82E299E058
:104E000029960FB6F894DEBF0FBECDBFDF91CF91CC
:104E10001F910F91FF90EF90DF90CF90BF90AF90D8
:104E20009F908F907F906F905F904F903F902F90CA
:104E30000C94DA9A82E299E029960FB6F894DEBFD4
:104E40000FBECDBFDF91CF911F910F91FF90EF90DB
:104E5000DF90CF90BF90AF909F908F907F906F909A
:104E60005F904F903F902F900C94DF9AD5018D91D9
:104E70009C9197FD02C00C94A63560E082E299E017
:104E80000E943167F501EE5AFF4F6081718140E069
:104E900082E299E029960FB6F894DEBF0FBECDBF2F
:104EA000DF91CF911F910F91FF90EF90DF90CF9006
:104EB000BF90AF909F908F907F906F905F904F903A
:104EC0003F902F900C94169E82E299E029960FB69F
:104ED000F894DEBF0FBECDBFDF91CF911F910F9130
:104EE000FF90EF90DF90CF90BF90AF909F908F900A
:104EF0007F906F905F904F903F902F900C94449BC9
:104F0000F5018081918192FD02C00C94A635468DF9
:104F1000578D60A171A180918C09882311F40C94A4
:104F2000A635409383095093840960938509709353
:104F3000860982E699E029960FB6F894DEBF0FBE87
:104F4000CDBFDF91CF911F910F91FF90EF90DF9038
:104F5000CF90BF90AF909F908F907F906F905F9019
:104F60004F903F902F900C947765D5018D919C9137
:104F700097FD02C00C94A635F501EE5AFF4F6081F3
:104F8000718182E299E029960FB6F894DEBF0FBED8
:104F9000CDBFDF91CF911F910F91FF90EF90DF90E8
:104FA000CF90BF90AF909F908F907F906F905F90C9
:104FB0004F903F902F900C94BD9EF5018081918180
:104FC00097FD02C00C94A63560E082E299E00E9451
:104FD0003167F501EE5AFF4F6081718182E299E0FD
:104FE00029960FB6F894DEBF0FBECDBFDF91CF91EB
:104FF0001F910F91FF90EF90DF90CF90BF90AF90F7
:105000009F908F907F906F905F904F903F902F90E8
:105010000C941F9FD5018D919C9197FD02C00C941B
:10502000A63560E082E299E00E943167F501EE5A10
:10503000FF4F6081718182E299E029960FB6F89462
:10504000DEBF0FBECDBFDF91CF911F910F91FF90BB
:10505000EF90DF90CF90BF90AF909F908F907F9018
:105060006F905F904F903F902F900C944D9FF50163
:105070002081318133FD02C00C94A63512A1E12EAE
:10508000F3A0E1E7FDE0449150E04E155F0509F41F
:105090005EC032964DE0E53EF407A9F7F7FC57C035
:1050A00032FF2CC0D5015E964D915D916D917C9142
:1050B00091974F3F51056105710509F0E0F461E0FA
:1050C000812F0F941D05F501668D812F0F945605D4
:1050D000D5015E966D917C915F97812F0F94FB02B5
:1050E000B7018DE893E20E9475A0F501668D778D7A
:1050F00088E893E212C08FE095E02BC062E0812F38
:105100000F941D05B70188E893E20E9475A0812FD6
:105110000F948B05BC0183E893E229960FB6F894AF
:10512000DEBF0FBECDBFDF91CF911F910F91FF90DA
:10513000EF90DF90CF90BF90AF909F908F907F9037
:105140006F905F904F903F902F900C9481A089EDCD
:1051500094E029960FB6F894DEBF0FBECDBFDF9165
:10516000CF911F910F91FF90EF90DF90CF90BF9064
:10517000AF909F908F907F906F905F904F903F90F7
:105180002F900C94BD9F10920D080C94A63581E0D1
:1051900080930D080C94A635D5018D919C911197A3
:1051A00092FF14C05E962D913D914D915C91919727
:1051B000A8EEB3E00F94E30D60933E0370933F03BA
:1051C00080934003909341030C94A63593FFA5C0B0
:1051D000F50182A193A1A4A1B5A182309105A105F9
:1051E000B10509F466C02CF50097A105B10509F4D5
:1051F00046C00197A105B10511F00C94A63529967A
:105200000FB6F894DEBF0FBECDBFDF91CF911F91D7
:105210000F91FF90EF90DF90CF90BF90AF909F9055
:105220008F907F906F905F904F903F902F900C9455
:105230006C1D83309105A105B10509F454C0049794
:10524000A105B10511F00C94A63529960FB6F89476
:10525000DEBF0FBECDBFDF91CF911F910F91FF90A9
:10526000EF90DF90CF90BF90AF909F908F907F9006
:105270006F905F904F903F902F900C94D45129964F
:105280000FB6F894DEBF0FBECDBFDF91CF911F9157
:105290000F91FF90EF90DF90CF90BF90AF909F90D5
:1052A0008F907F906F905F904F903F902F900C94D5
:1052B0006A1D29960FB6F894DEBF0FBECDBFDF91F1
:1052C000CF911F910F91FF90EF90DF90CF90BF9003
:1052D000AF909F908F907F906F905F904F903F9096
:1052E0002F900C946E1D29960FB6F894DEBF0FBE5A
:1052F000CDBFDF91CF911F910F91FF90EF90DF9085
:10530000CF90BF90AF909F908F907F906F905F9065
:105310004F903F902F900C94C6510E94431E81E005
:1053200029960FB6F894DEBF0FBECDBFDF91CF91A7
:105330001F910F91FF90EF90DF90CF90BF90AF90B3
:105340009F908F907F906F905F904F903F902F90A5
:105350000C947B74D5018D919C91119792FF14C090
:105360005E962D913D914D915C919197A8EEB3E0A1
:105370000F94E30D609342037093430380934403BF
:10538000909345030C94A635109242031092430368
:1053900010924403109245030C94A635F5018081C8
:1053A00083FF0CC082859385A485B58580932703F0
:1053B00090932803A0932903B0932A03D5018C91DD
:1053C00084FF0EC01E968D919D910D90BC91A02DD5
:1053D00080932B0390932C03A0932D03B0932E0363
:1053E000F501808185FF0CC082899389A489B589E4
:1053F00080932F0390933003A0933103B093320333
:105400000E94E774D5018C9186FD02C00C94A635EC
:10541000209190033091910356968D919D910D901E
:10542000BC91A02DF90181879287A387B4878081E1
:1054300029960FB6F894DEBF0FBECDBFDF91CF9196
:105440001F910F91FF90EF90DF90CF90BF90AF90A2
:105450009F908F907F906F905F904F903F902F9094
:105460000C940350D501ED91FC911197F2FF0DC002
:105470005E962D913D914D915C919197A8EEB3E090
:105480000F94E30D6B017C0106C040E1C42E47E29E
:10549000D42EE12CF12CE3FD0E946A1DF5018081E0
:1054A00084FD0E946C1DD5018C9185FD0E946E1DAE
:1054B0000F9409042B013C014C0C5D1C6E1C7F1CDD
:1054C0000F940904A3019201261B370B480B590BBB
:1054D000DA01C901803A9648A140B10518F40E944A
:1054E000DD79EECFD5018C9183FD1798F501808190
:1054F00084FD1698D5018C9185FD02C00C94A635CB
:1055000015980C94A6350E94EA5981110C94A63581
:105510000F94090460938C1D70938D1D80938E1DD4
:1055200090938F1D0E94641D81110C94A635F50186
:105530008081918193FF02C00C94903592FF0AC044
:10554000868D978DA0A1B1A1892B8A2B8B2B11F46D
:105550000C949035D5018D919C91119792FD02C0CC
:105560000C94A6359C012227317091FF23C0232B78
:1055700089F011E020E030E0A9015A966D917D910B
:105580008D919C915D970F94060C18160CF010E00D
:10559000212F01C020E085010C5A1F4FF501668DB7
:1055A000778D80A191A129870F94A50A2985D8011B
:1055B0004C9124C0232B81F011E020E030E0A901C0
:1055C000F501628D738D848D958D0F94060C1816E0
:1055D0000CF010E0212F01C020E000919003109109
:1055E0009103D5015E966D917D918D919C919197DE
:1055F00029870F94A50A2985F801408129960FB6BD
:10560000F894DEBF0FBECDBFDF91CF911F910F91F8
:10561000FF90EF90DF90CF90BF90AF909F908F90D2
:105620007F906F905F904F903F902F900C943A55E1
:105630000E94EA5981110C94A6350F9409046093D5
:105640008C1D70938D1D80938E1D90938F1D0E94D5
:10565000641D81110C94A635D5018D919C911197F3
:1056600092FD02C00C94A63590FF11C011E020E01D
:1056700030E0A9015A966D917D918D919C915D9735
:105680000F94060C18160CF010E0412F01C040E0FA
:10569000F501668D778D80A191A149870F94A50AA8
:1056A000498529960FB6F894DEBF0FBECDBFDF91B6
:1056B000CF911F910F91FF90EF90DF90CF90BF900F
:1056C000AF909F908F907F906F905F904F903F90A2
:1056D0002F900C940356D5018D919C9133E09695B3
:1056E00087953A95E1F7817029960FB6F894DEBF59
:1056F0000FBECDBFDF91CF911F910F91FF90EF9023
:10570000DF90CF90BF90AF909F908F907F906F90E1
:105710005F904F903F902F9099C80E94EA59811155
:105720000C94A6350F94090460938C1D70938D1D05
:1057300080938E1D90938F1D0E94641D81110C9487
:10574000A63540E068EC74E086E79AE00E94A6ABDC
:1057500086E79AE00E94FAAE0E94431E20909003D2
:1057600030909103F5018081918191FF09C0EC5A3D
:10577000FF4F2081211104C02BE5222E22E0322E82
:1057800092FF1EC090FF0FC011E020E030E0A901A1
:10579000D5015A966D917D918D919C915D970F9455
:1057A000060C18160CF010E0F501668D778D80A1BF
:1057B00091A10F94A50A212FD1014C910E943A5535
:1057C000F10126A937A940AD51AD62A973A984A9F9
:1057D00095A90F946D092B013C0120E030E0A9014F
:1057E0000F94060C181664F420E030E040EA50E410
:1057F000C301B2010F94D20987FF0EC00C94A635E5
:1058000020E030E040EA50ECC301B2010F94060CF6
:10581000181614F40C94A63599249394D101D096BB
:105820002D913C91D1979E968D919C919F97821737
:1058300093070CF0912C0F9409046D837E838F8362
:10584000988710E0412C512C32010F940904698390
:105850007A838B839C8360938C1D70938D1D8093C2
:105860008E1D90938F1DDC01CB012D813E814F81D8
:105870005885821B930BA40BB50B893E9340A10561
:10588000B10558F080E00E94262489819A81AB817D
:10589000BC818D839E83AF83B88781E00E94211EE7
:1058A00080919003909191032816390609F064C005
:1058B000D1019396ED90FC9094971E141F040CF068
:1058C0005BC0111158C0992009F477C091966D9171
:1058D0007C919297882777FD8095982F0F94A50A41
:1058E0009B01AC01F10162A973A984A995A90F9448
:1058F000060C181614F00C949D35662777276E1940
:105900007F09882777FD8095982F0F94A50A20910D
:1059100033033091340340913503509136030F9493
:105920007A0C0F94720A1F921F92D10152962C91F9
:1059300052972F9351962C9151972F9350962C91CB
:1059400050972F931F962C912F935B016C01E12CA4
:10595000F12C870120E030E0A90160E070E0CB018C
:105960000E942CF80F900F900F900F900F900F90B7
:1059700011E00C949D3511E041145104610471044F
:1059800009F050C09920F1F020E030E040E85FE3FA
:10599000F10166A977A980AD91AD0F946D099B01C6
:1059A000AC01D101D2966D917D918D919C91D5974D
:1059B0000F94060C87FF1FC045CF411451046104AA
:1059C000710481F520E030E040E85FE3F10166A971
:1059D00077A980AD91AD0F946E099B01AC01D10107
:1059E000D2966D917D918D919C91D5970F94D2090E
:1059F00018160CF427CFF101A78DB0A128EE33E0E3
:105A00000F94DD0D2B013C0129813A814B815C8192
:105A1000420E531E641E751E41145104610471042C
:105A200009F413CFD301C20129813A814B815C81F2
:105A3000821B930BA40BB50B81159449A543B74763
:105A400008F403CF112309F4E2C0809190039091F0
:105A500091032816390609F0DAC0D10193966D91A9
:105A60007C919497882777FD8095982F0F94A50AAD
:105A70002091330330913403409135035091360324
:105A80000F947A0C0F94720A1F921F92F1012289CF
:105A90002F9321892F9320892F9327852F935B01A3
:105AA0006C01E12CF12C870120E030E0A90160E0DD
:105AB00070E0CB010E942CF80F900F900F900F9088
:105AC0000F900F90A4C00E94641D81110C94A63504
:105AD00040E06CEB74E086E79AE00E94A6AB86E7B4
:105AE0009AE00E94FAAE0E94431ED5018D919C91CE
:105AF000119792FF1FC090FF11C011E020E030E02D
:105B0000A9015A966D917D918D919C915D970F940D
:105B1000060C18160CF010E0412F01C040E0F50112
:105B2000668D778D80A191A149870F94A50A49853B
:105B30000E9403562091190230911A0240911B02D3
:105B400050911C026091150270911602809117020B
:105B5000909118020F946D092B013C0120E030E078
:105B6000A9010F94060C18165CF420E030E040EA1E
:105B700050E4C301B2010F94D20987FF0CC0E6C7FD
:105B800020E030E040EA50ECC301B2010F94060C73
:105B900018160CF4DBC70F9409042B013C0120E01C
:105BA00030E040E05FE36091150270911602809151
:105BB0001702909118020F946E09209119023091EA
:105BC0001A0240911B0250911C020F94D20987FFC8
:105BD0001EC00F9409046419750986099709693E66
:105BE00073408105910578F080E00E9426240F948F
:105BF00009042B013C0160938C1D70938D1D8093D3
:105C00008E1D90938F1D81E00E94211EC8CF10929F
:105C1000DF0A0F94090460938C1D70938D1D80938F
:105C20008E1D90938F1D92C70E94641D81118EC797
:105C30000F9409042B013C010F94090464197509A0
:105C400086099709693E73408105910538F080E027
:105C50000E9426240F9409042B013C0181E00E943C
:105C6000211E00910A0210910B02D8011B968D9003
:105C70009D90AD90BC901E9720E030E040EF51E445
:105C8000C501B4010F94060C1816BCF4F801278165
:105C9000308541855285C501B4010F946D099F7708
:105CA00001E020E030E040E85FE30F94060C1816B6
:105CB0000CF000E011E0102701C011E0E0900C02B0
:105CC000F0900D02D7011B968D909D90AD90BC90E9
:105CD0001E9720E030E040EF51E4C501B4010F947D
:105CE000060C18169CF4F7012781308541855285F2
:105CF000C501B4010F946D099F7720E030E040E8C2
:105D00005FE30F94060C18160CF496CF112309F4D8
:105D100093CF1CC7D5018D919C91119793FB66275A
:105D200060F992FF05C05E968D919C915F970AC0C5
:105D30008FEF90E007C0F501618163FB662760F992
:105D400080E090E029960FB6F894DEBF0FBECDBF7D
:105D5000DF91CF911F910F91FF90EF90DF90CF9047
:105D6000BF90AF909F908F907F906F905F904F907B
:105D70003F902F900C949C20D5018D919C91119770
:105D800092FF04C05E962C912093EA0293FF12C00A
:105D9000F50182A193A1A4A1B5A12091EA02181650
:105DA00019061A061B0614F4822B02C081508223A6
:105DB0008093EA020E94641D882309F4C7C620E08C
:105DC00040E060E070E0CB010E943A5520E040E006
:105DD00060E070E0CB0112CC88E695E20E949C9FC7
:105DE00029960FB6F894DEBF0FBECDBFDF91CF91DD
:105DF0001F910F91FF90EF90DF90CF90BF90AF90E9
:105E00009F908F907F906F905F904F903F902F90DA
:105E10000C94C62086EB94E066C3D5018D919C91CD
:105E200097FF94C6F501EE5AFF4F6081718140E003
:105E300086E79AE00E941FAC86E79AE029960FB6A3
:105E4000F894DEBF0FBECDBFDF91CF911F910F91B0
:105E5000FF90EF90DF90CF90BF90AF909F908F908A
:105E60007F906F905F904F903F902F900C94FAAE80
:105E70000E94431E86E793E20E94839F0E94701D4A
:105E8000882319F080E893E202C08DE793E20E9434
:105E9000839F8FE693E20E94839F0E94751D882353
:105EA00019F080E893E202C08DE793E20E94839F9D
:105EB00088E693E20E94839F379903C08DE793E2BF
:105EC00002C080E893E20E94839F29960FB6F8945F
:105ED000DEBF0FBECDBFDF91CF911F910F91FF901D
:105EE000EF90DF90CF90BF90AF909F908F907F907A
:105EF0006F905F904F903F902F900C941C24F50171
:105F00008081918188279C7081159C4009F01EC674
:105F1000F50162A1868D29960FB6F894DEBF0FBEFB
:105F2000CDBFDF91CF911F910F91FF90EF90DF9048
:105F3000CF90BF90AF909F908F907F906F905F9029
:105F40004F903F902F900C94A4A2E0919003F09179
:105F500091032081D5018D919C9191FF06C0F5019F
:105F6000EC5AFF4F8081882311F0822F01C080E01E
:105F7000F501928192FF05C046A457A460A871A8BC
:105F800003C0412C512C320193FF07C0D501D2969A
:105F90004D905D906D907C90D597082F10E0B3E800
:105FA0008B9FF0011124E752FD4F408251826282A3
:105FB0007382821306C08091FF06909100070E94B1
:105FC000242020E030E0A901C301B2010F94D209DE
:105FD000B801811103C08AE894E09FC883E694E089
:105FE0000E9475A022E0B301A2018EE594E05DC19C
:105FF000F501808183FF0CC082859385A485B585DA
:106000008093FB029093FC02A093FD02B093FE02EA
:10601000D5018C9184FF0EC01E968D919D910D909F
:10602000BC91A02D8093FF0290930003A0930103E5
:10603000B0930203F501808185FF0CC082899389AA
:10604000A489B5898093030390930403A093050367
:10605000B0930603D5018C9186FF0EC056968D91A4
:106060009D910D90BC91A02D809307039093080300
:10607000A0930903B0930A0329960FB6F894DEBFE4
:106080000FBECDBFDF91CF911F910F91FF90EF9089
:10609000DF90CF90BF90AF909F908F907F906F9048
:1060A0005F904F903F902F900C94E774F5018081A2
:1060B00083FF0CC082859385A485B5858093EB0210
:1060C0009093EC02A093ED02B093EE02D5018C9177
:1060D00084FF0EC01E968D919D910D90BC91A02DB8
:1060E0008093EF029093F002A093F102B093F2023A
:1060F000F501808185FF0CC082899389A489B589C7
:106100008093F3029093F402A093F502B093F60209
:10611000D5018C9186FFB0CF56968D919D910D90B3
:10612000BC91A02D8093F7029093F802A093F902FE
:10613000B093FA02A1CFF5018081918192FF06C54B
:10614000868D978DA0A1B1A1181619061A061B06F7
:106150000CF481E08093E002F9C4E0919003F091A7
:106160009103BB96D5012D913C91119732FF11C03F
:106170005E968D919D910D90BC91A02DB7FDE6C4CA
:10618000892B8A2B8B2B19F0EEE0F2E002C0E6E8B7
:10619000F2E023FF0BC0D5011A964D915D916D91F0
:1061A0007C911D97428F538F648F758FD5018C9191
:1061B00084FF0AC01E964D915D916D917C9151971F
:1061C000468F578F60A371A3D5018C9185FF0AC0BC
:1061D00052964D915D916D917C91559742A353A339
:1061E00064A375A3CF0129960FB6F894DEBF0FBE46
:1061F000CDBFDF91CF911F910F91FF90EF90DF9076
:10620000CF90BF90AF909F908F907F906F905F9056
:106210004F903F902F900C94354F29960FB6F894DD
:10622000DEBF0FBECDBFDF91CF911F910F91FF90C9
:10623000EF90DF90CF90BF90AF909F908F907F9026
:106240006F905F904F903F902F900C9492D7F501F4
:10625000208123FF0CC082859385A485B58580931A
:10626000FB069093FC06A093FD06B093FE0626FF66
:1062700011C02091900330919103F501868997898F
:10628000A08DB18DF901878B908FA18FB28F808106
:106290000E9403504091FB065091FC066091FD0660
:1062A0007091FE0622E082E693E229960FB6F894FA
:1062B000DEBF0FBECDBFDF91CF911F910F91FF9039
:1062C000EF90DF90CF90BF90AF909F908F907F9096
:1062D0006F905F904F903F902F900C949BA1D501B1
:1062E0008D919C91119792FF31C461E05E968D91E2
:1062F0009D910D90BC91A02D2091C607892B8A2BD2
:106300008B2B21F460E0822F8D7F02C0822F826070
:106310008093C60770E085EC93E00C948D28F5011E
:106320008081918192FF05C0868D978DA0A1B1A13A
:1063300004C084E690E0A0E0B0E029960FB6F8949F
:10634000DEBF0FBECDBFDF91CF911F910F91FF90A8
:10635000EF90DF90CF90BF90AF909F908F907F9005
:106360006F905F904F903F902F900C949D1FD501A0
:106370008D919C91119792FF07C05E968D919D9192
:106380000D90BC91A02D04C084E690E0A0E0B0E0A8
:1063900029960FB6F894DEBF0FBECDBFDF91CF9127
:1063A0001F910F91FF90EF90DF90CF90BF90AF9033
:1063B0009F908F907F906F905F904F903F902F9025
:1063C0000C942420F5018081918192FFBFC34FB7C7
:1063D000F8948091520890915308268D378D820F42
:1063E000931F90935308809352084FBFAFC3F5019A
:1063F0008081209190033091910384FF09C08685AC
:106400009785A089B189F90185A396A3A7A3B0A711
:10641000D90195964D915D916D917C91989722E06F
:1064200081E393E20E94D8A10E941C2429960FB612
:10643000F894DEBF0FBECDBFDF91CF911F910F91BA
:10644000FF90EF90DF90CF90BF90AF909F908F9094
:106450007F906F905F904F903F902F900C94CD74F1
:106460002091F9073091FA074091FB075091FC0702
:1064700060910B0770910C0780910D0790910E07AA
:106480000F946D0960930B0770930C0780930D07B1
:1064900090930E07109205081092060810920708B4
:1064A000109208080E94E77461E178E08DEF97E0B0
:1064B0000E9418ED80E00E94F08040910B075091FF
:1064C0000C0760910D0770910E0722E086EC9FE1AA
:1064D0000E949BA180E00E945BCF8BE393E20E942D
:1064E0009C9F88E594E029960FB6F894DEBF0FBE16
:1064F000CDBFDF91CF911F910F91FF90EF90DF9073
:10650000CF90BF90AF909F908F907F906F905F9053
:106510004F903F902F900C94511E84E00F948B0568
:10652000BC018EE494E00E9481A029960FB6F894F5
:10653000DEBF0FBECDBFDF91CF911F910F91FF90B6
:10654000EF90DF90CF90BF90AF909F908F907F9013
:106550006F905F904F903F902F900C94062482E3B1
:106560000E948023F5018081918192FFEFC2468DC8
:10657000578D60A171A188E394E00E94BFA0D5016E
:106580005E966C9182E30E945D23F501668D8AE33D
:106590000E945D2382E329960FB6F894DEBF0FBEFA
:1065A000CDBFDF91CF911F910F91FF90EF90DF90C2
:1065B000CF90BF90AF909F908F907F906F905F90A3
:1065C0004F903F902F900C9480238DEF93E00E948A
:1065D000B39F80E00E947B7468EC70E080E090E004
:1065E0000F9438048FB7F894FFCFD5018D919C910B
:1065F000119792FF05C05E966D917C915F9702C0E6
:1066000061E070E093FF04C0F50102A113A102C094
:1066100008EE13E020E030E0A9018FE40F94DB05E1
:10662000B80180E090E00F9438048FE429960FB60B
:10663000F894DEBF0FBECDBFDF91CF911F910F91B8
:10664000FF90EF90DF90CF90BF90AF909F908F9092
:106650007F906F905F904F903F902F900D94EC083B
:10666000D5018D919C91119792FF0EC021E05E960D
:106670008D919D910D90BC91A02D892B8A2B8B2BF8
:1066800009F420E0822F01C081E09091C7078823A0
:1066900011F0906801C09F779093C707882319F085
:1066A0008EEA93E002C084E993E029960FB6F8944D
:1066B000DEBF0FBECDBFDF91CF911F910F91FF9035
:1066C000EF90DF90CF90BF90AF909F908F907F9092
:1066D0006F905F904F903F902F900C949C9FF5018E
:1066E0000081118112FF03C0668D778D02C066E9BB
:1066F00070E013FF0DC0D5019296ED90FC9093973A
:10670000B2E0EB16F10434F082E0E82EF12C02C086
:10671000E12CF12CA3E016950795AA95E1F70170FD
:10672000882777FD8095982F0F94A50AAB01BC01AF
:10673000F701EE0FFF1FE65FFD4F2E2D8081918147
:106740000E94845603C281E00E94C78715C080E082
:106750000E94C787D5018D919C91119792FFF6C138
:106760005E968D919D910D90BC91A02D0097A105F5
:10677000B10509F0D9C1EAC1F5018081918192FF8B
:10678000E5C1868D978DA0A1B1A1892B8A2B8B2B7A
:1067900009F4DCC180E029960FB6F894DEBF0FBE85
:1067A000CDBFDF91CF911F910F91FF90EF90DF90C0
:1067B000CF90BF90AF909F908F907F906F905F90A1
:1067C0004F903F902F900C945BCF8BEE93E00E9404
:1067D0009C9FD5018D919C9192FD0FC0F501808108
:1067E00083FF16C0F50162857385848595850F94B6
:1067F000770A80E00E9468220BC010E0D5015E9607
:106800006C91812F0E9468221F5F1530B9F7E6CF87
:10681000D5018C9184FF0BC01E966D917D918D9159
:106820009C9151970F94770A81E00E946822F501AC
:10683000808185FF09C062897389848995890F9455
:10684000770A82E00E946822D5018C9186FF0BC0F6
:1068500056966D917D918D919C9159970F94770AE1
:1068600083E00E946822F5018081918193FF04C03A
:1068700062A184E00E94682229960FB6F894DEBFD8
:106880000FBECDBFDF91CF911F910F91FF90EF9081
:10689000DF90CF90BF90AF909F908F907F906F9040
:1068A0005F904F903F902F900C947F22D5018D9157
:1068B0009C91119792FF26C081E05E964D915D916B
:1068C0006D917C919197452B462B472B09F480E0E5
:1068D00029960FB6F894DEBF0FBECDBFDF91CF91E2
:1068E0001F910F91FF90EF90DF90CF90BF90AF90EE
:1068F0009F908F907F906F905F904F903F902F90E0
:106900000C94429029960FB6F894DEBF0FBECDBF0F
:10691000DF91CF911F910F91FF90EF90DF90CF907B
:10692000BF90AF909F908F907F906F905F904F90AF
:106930003F902F900C94439029960FB6F894DEBFA9
:106940000FBECDBFDF91CF911F910F91FF90EF90C0
:10695000DF90CF90BF90AF909F908F907F906F907F
:106960005F904F903F902F900C94519029960FB6C6
:10697000F894DEBF0FBECDBFDF91CF911F910F9175
:10698000FF90EF90DF90CF90BF90AF909F908F904F
:106990007F906F905F904F903F902F900C94431E8C
:1069A000F5018081918190FF05C0E28CF38C048D0C
:1069B000158D08C0E0900307F090040700910507CB
:1069C000109106079C0146E0369527954A95E1F718
:1069D0002170AC0165E0569547956A95E1F74170E5
:1069E000BC01E4E076956795EA95E1F76170F3E024
:1069F00096958795FA95E1F781700E94F486A6C076
:106A00000E94B8D1E0919003F091910380810E949F
:106A100003508AE99EE129960FB6F894DEBF0FBEB7
:106A2000CDBFDF91CF911F910F91FF90EF90DF903D
:106A3000CF90BF90AF909F908F907F906F905F901E
:106A40004F903F902F900C94B39F29960FB6F894D7
:106A5000DEBF0FBECDBFDF91CF911F910F91FF9091
:106A6000EF90DF90CF90BF90AF909F908F907F90EE
:106A70006F905F904F903F902F900C9460CD82ED7F
:106A800093E00E949C9FD5018D919C9188279C70DA
:106A900081159C4009F05AC0D5015E966D917C919C
:106AA0005F9792968C9129960FB6F894DEBF0FBE31
:106AB000CDBFDF91CF911F910F91FF90EF90DF90AD
:106AC000CF90BF90AF909F908F907F906F905F908E
:106AD0004F903F902F900C9498218091EA0282FF72
:106AE00035C08CE594E20E94839FC50129960FB6BC
:106AF000F894DEBF0FBECDBFDF91CF911F910F91F4
:106B0000FF90EF90DF90CF90BF90AF909F908F90CD
:106B10007F906F905F904F903F902F900C94719763
:106B20000E94431E0C94AA2A0397A105B10509F0FF
:106B300031CE80E00E94198C2DCE411451046104A5
:106B4000710411F40C94C42C0C94122D29960FB6D8
:106B5000F894DEBF0FBECDBFDF91CF911F910F9193
:106B6000FF90EF90DF90CF90BF90AF909F908F906D
:106B70007F906F905F904F903F902F9008952F924D
:106B80003F924F925F926F927F928F929F92AF92BD
:106B9000BF92CF92DF92EF92FF920F931F93CF930A
:106BA000DF93CDB7DEB7EC970FB6F894DEBF0FBE1C
:106BB000CDBF1C01DC0118968D919C9119978032F4
:106BC000910509F43AC358F58531910509F45EC180
:106BD00098F48430910509F41BC128F4029708F455
:106BE000EBC00C946944449711F00C94694481E023
:106BF000809351080C9474448D31910509F499C126
:106C000028F44C9709F446C10C9469448E319105DF
:106C100009F4F0C14F9709F4FFC20C9469448C3514
:106C2000910511F40C94934040F58534910509F4D5
:106C300063C7B8F48434910511F00C9469448091D1
:106C4000030790910407A0910507B09106078D876F
:106C50009E87AF87B88B44E1442E512C612C712C58
:106C600076C58A35910511F40C9478408B359105E1
:106C700011F40C9484400C9469448438910511F407
:106C80000C942A4308F05DC08436910511F40C94ED
:106C900075418338910511F00C9469446091F107B6
:106CA0007091F2078091F3079091F4072091F50716
:106CB0003091F6074091F7075091F807E090F907F7
:106CC000F090FA070091FB071091FC074090030732
:106CD0005090040760900507709006071092F70621
:106CE0001092F8061092F9061092FA061092F30626
:106CF0001092F4061092F5061092F606E0910E033B
:106D0000EF93E0910D03EF93E0910C03EF93E0918B
:106D10000B03EF93E0EFAE2EE3E2BE2EE4E7CE2EC0
:106D2000E9E4DE2E0E94337E40920307509204076E
:106D3000609205077092060780E00E94F0800C9434
:106D400025438538910511F40C94B9438638910593
:106D500011F00C946944409111085091120860910F
:106D600013087091140880EA95E00E94A7A0409152
:106D7000150850911608609117087091180887EB54
:106D800093E20E94A7A04091190850911A086091BF
:106D90001B0870911C0887EB93E20E94BFA080E063
:106DA0000E94F08082E995E00E94839F8CE895E044
:106DB0000E94511E0C947444F1018081918192FFD4
:106DC00011C0868D978DA0A1B1A12091C707892BF5
:106DD0008A2B8B2B19F0822F806202C0822F8F7D2D
:106DE0008093C707C1010E946782882359F041E060
:106DF00061E081E00E94FCF2811104C082EC9CE021
:106E00000E94A99F61E081E00E94FDEC0C94744413
:106E10000E94431ED1018D919C91119793FF07C051
:106E200092968D909D90AD90BC90959703C0812CCB
:106E3000912C540192FF0BC0F101268D378D40A19A
:106E400051A1A8EEB3E00F94E30D4B015C010F9448
:106E500009046B017C01C80CD91CEA1CFB1C0F94B3
:106E60000904A7019601261B370B480B590BDA01C1
:106E7000C90181159449A543B74710F00C94744497
:106E80000E94649881E00E94211EE9CF109251086F
:106E90000C947444D1018D919C91AC014873552799
:106EA0004115510551F49C0166E0369527956A9588
:106EB000E1F7B1E02B27217001C020E086FF08C078
:106EC0001092090810920A0810920B0810920C08F0
:106ED000211117C0452BD1F0AC0125E056954795FF
:106EE0002A95E1F7BC0134E0769567953A95E1F78C
:106EF00053E0969587955A95E1F7617041708170DE
:106F000003C061E041E081E00E94E18780E00E94EF
:106F1000F0800E94701D81110C9497440E94751D91
:106F200081110C949744379902C00C9474440C94CA
:106F300097440E940624811111C06AEF70E080E03E
:106F400090E00F9438040E940624811107C08EE55A
:106F50009CE00E949C9F85E49CE05AC180E39CE0F9
:106F60000E942A962091030730910407409105075B
:106F700050910607298F3A8F4B8F5C8F80E090E00D
:106F80000E94C11D80E090E00E94E11D80E090E041
:106F90000E94011E80E00E945BCF0E94B8D184E174
:106FA00090E0A0E0B0E0898B9A8BAB8BBC8B86E144
:106FB000482E512C612C712C1DA229893A894B89AC
:106FC0005C892D873E874F87588B41E061E081E0E7
:106FD0000E94E1870E94701D81110C94B4440E94AC
:106FE000751D81110C94B444379902C00C94D84497
:106FF0000C94B444D1012D913C91119732FD02C003
:107000000C94DE495E968D919D910D90BC91A02DC2
:107010000297A105B10511F00C94DE490C94574A72
:1070200081E99BE00E949C9F89E79BE00E942A9651
:1070300086ED9FE10E94BD9FEDA1E1110C94744487
:1070400081E00E94F080298D3A8D4B8D5C8D2093DC
:10705000030730930407409305075093060787E31F
:107060009AE00E94511E8EE390E20E942A96212C03
:10707000312C8091770790917807A0917907B09192
:107080007A07898B9A8BAB8BBC8B80E00E945BCF9D
:107090000E94B8D181E00E94C78741E061E081E0B1
:1070A0000E94E18780E00E94C7878FE390E20E9400
:1070B0002A960E94791D9F938F937F936F93B0EFD1
:1070C000AB2EB3E2BB2EB4E7CB2EB9E4DB2E8601A8
:1070D000750120E030E0A901CA01B9010E949E8536
:1070E00020E041E060E081E00E9470886B017C015B
:1070F00020E041E060E081E00E9470884B015C018B
:107100009B01AC01C701B6010F946D092B013C0135
:107110000F900F900F900F902DEC3CEC4CEC5DE33A
:107120000F94060C181614F00C94EF474D855E85ED
:107130006F85788983E09AE00E94BFA02D853E8507
:107140004F855889283231054105510514F00C94BA
:10715000FB4782E30E9480238D859E85AF85B88999
:107160000296A11DB11D8D879E87AF87B88BAC019C
:10717000BD0185EE99E00E94BFA06D8582E30E946B
:107180005D236D858AE30E945D2382E30E94802354
:10719000B4E02B1631040CF46CCF81E00E94C78759
:1071A00081E00E94F08086ED98E00E94511E8EE3FF
:1071B00090E20E942A96298D3A8D4B8D5C8D20930A
:1071C000030730930407409305075093060741E0F7
:1071D00061E081E00E94E18780E00E945BCF41E0B6
:1071E00066E573E082E299E00E94169E882371F0C2
:1071F00082E299E00E94749B66E573E082E299E086
:107200000E941F9F82E299E00E94AC9A8CEB98E06A
:107210000E942A960C9474448CE490E20E94839F0E
:10722000959902C068E401C06CE48AE39BE00E9487
:107230007CD90E941C240C9474448FE390E20E9439
:107240002A961092D1071092D2071092D30710926B
:10725000D4071092CD071092CE071092CF0710924C
:10726000D0071092C9071092CA071092CB0710924C
:10727000CC0780E00E94C787209103073091040764
:10728000409105075091060729A33AA34BA35CA39D
:107290000E94791D162F072FF82EE92E84E393E024
:1072A0000E942D1D9B01AC0180E393E029AF3AAF12
:1072B0004BAF5CAF0E942D1DEF92FF920F931F9377
:1072C00050EFA52E53E2B52E54E7C52E59E4D52E26
:1072D0008601750129AD3AAD4BAD5CAD0E949E852E
:1072E00020E041E060E081E00E9470882B013C01D9
:1072F0000F900F900F900F9020E030E0A9010F94B5
:10730000D20987FF02C00C9474440E94791D162F85
:10731000072FF82EE92E8CE393E00E942D1D9B0190
:10732000AC0188E393E029AF3AAF4BAF5CAF0E946A
:107330002D1DEF92FF920F931F938601750129ADCA
:107340003AAD4BAD5CAD0E949E8521E041E060E02E
:1073500080E00E9470886D877E878F87988B0F9062
:107360000F900F900F9020E030E0A9010F94D20908
:1073700087FF02C00C9474440E94791D162F072FBA
:10738000F82EE92E84E493E00E942D1D9B01AC01B0
:1073900080E493E029AF3AAF4BAF5CAF0E942D1D64
:1073A000EF92FF920F931F938601750129AD3AADBD
:1073B0004BAD5CAD0E949E8521E041E061E080E044
:1073C0000E9470884B015C010F900F900F900F90FE
:1073D00020E030E0A9010F94D20987FF02C00C948D
:1073E0007444850174012D853E854F855889C301FC
:1073F000B2010E94148E80919D0790919E07A091EA
:107400009F07B091A0078D879E87AF87B88B20918B
:10741000B1073091B2074091B3075091B407298B5F
:107420003A8B4B8B5C8BC090A507D090A607E09061
:10743000A707F090A8078091A9079091AA07A091AB
:10744000AB07B091AC078D8B9E8BAF8BB88F209123
:1074500001083091020840910308509104082DA3BF
:107460003EA34FA358A78091450890914608A0914C
:107470004708B091480889A79AA7ABA7BCA7209155
:10748000AD073091AE074091AF075091B0072D8FF7
:107490003E8F4F8F58A38091A1079091A207A09192
:1074A000A307B091A407898F9A8FAB8FBC8F2091CF
:1074B000FD073091FE074091FF07509100082DA76E
:1074C0003EA74FA758AB8091410890914208A091E8
:1074D0004308B091440889AB9AABABABBCAB1092FC
:1074E0000707109208071092090710920A07D101A6
:1074F0008D919C91119792FFDCC05E968D919D912C
:107500000D90BC91A02DAC01BD0141505109610904
:107510007109423051056105710548F00397A105D5
:10752000B10509F0C6C080E00E945BCFC2C02989C6
:107530003A894B895C896D857E858F8598890F9402
:107540007A0C2B013C012D893E894F89588DC7014A
:10755000B6010F947A0C9B01AC01C301B2010F94E8
:107560006D092B013C016DA17EA18FA198A50F94FF
:10757000A50A9B01AC01C301B2010F947A0C29A5A5
:107580003AA54BA55CA50F947A0C2B013C012D8DDF
:107590003E8D4F8D58A1C701B6010F947A0C6B0137
:1075A0007C0129893A894B895C89698D7A8D8B8D1B
:1075B0009C8D0F947A0C9B01AC01C701B6010F940E
:1075C0006D096B017C016DA57EA58FA598A90F940F
:1075D000A50A9B01AC01C701B6010F947A0C29A939
:1075E0003AA94BA95CA90F947A0C9B01AC01C30189
:1075F000B2010F946E096B017C01F7FAF094F7F871
:10760000F0942D893E894F89588D698D7A8D8B8DA7
:107610009C8D0F947A0C2B013C012D8D3E8D4F8D4E
:1076200058A16D857E858F8598890F947A0C9B0172
:10763000AC01C301B2010F946D099B01AC01C701FC
:10764000B6010F94D9099B01AC01C501B4010F9497
:107650006E092091F9073091FA074091FB0750918C
:10766000FC070F946D0920910B0730910C07409196
:107670000D0750910E070F946E09AB01BC014093AA
:107680000B0750930C0760930D0770930E0722E0D1
:1076900086EC9FE10E949BA181E00E94C787F101D7
:1076A000868D978DA0A1B1A10297A105B10509F41E
:1076B0003ACF81E00E94C7870E94E77481E00E9470
:1076C000F08084E698E00E94511E41E061E081E094
:1076D0000E94E18729A13AA14BA15CA12093030755
:1076E0003093040740930507509306070C947444A5
:1076F0002DEC3CEC4CEC5DEBC701B6010F94D209CC
:1077000087FF85C0B301A20184E498E00E94BFA076
:1077100038E24316510461047104CCF482E30E9400
:10772000802342E0440E511C611C711CB301A20174
:1077300086E298E00E94BFA0642D82E30E945D2350
:10774000642D8AE30E945D2382E30E9480232091BE
:107750007707309178074091790750917A07298F00
:107760003A8F4B8F5C8F80E00E945BCF0E94B8D134
:1077700041E061E081E00E94E1878FE390E20E94B6
:107780002A9680E00E94C7870E94791D9F938F935D
:107790007F936F9330EFA32E33E2B32E34E7C32EE3
:1077A00039E4D32E8601750120E030E0A901CA0139
:1077B000B9010E949E8520E041E060E081E00E94E6
:1077C0007088698B7A8B8B8B9C8B20E041E060E02A
:1077D00081E00E9470886D8B7E8B8F8B988F9B01D0
:1077E000AC0169897A898B899C890F946D096B0139
:1077F0007C010F900F900F900F902DEC3CEC4CEC17
:107800005DE30F94060C18160CF072CF7BCF0E942C
:10781000791D162F072FF82EE92E84E493E00E949D
:107820002D1D9B01AC0180E493E029AF3AAF4BAF33
:107830005CAF0E942D1DEF92FF920F931F9320EFDC
:10784000A22E23E2B22E24E7C22E29E4D22E8601F4
:10785000750129AD3AAD4BAD5CAD0E949E8521E02E
:1078600041E061E080E00E9470884B015C0121E012
:1078700041E061E080E00E9470886B017C019B0127
:10788000AC01C501B4010F946D096D8F7E8F8F8F90
:1078900098A30F900F900F900F902DEC3CEC4CECB8
:1078A0005DE30F94060C181664F02DEC3CEC4CECE8
:1078B0005DEB6D8D7E8D8F8D98A10F94D20987FF22
:1078C00013C0B301A20186E098E00E94BFA082E34A
:1078D0000E94802352E0450E511C611C711CB301B3
:1078E000A20188EE97E026CF29893A894B895C89E5
:1078F0006D897E898F89988D0F946E0920E030E024
:1079000040E05FE30F947A0C698B7A8B8B8B9C8BB6
:1079100020E030E0A9010F94D20987FD18CFA5011E
:107920009401C701B6010F946E0920E030E040E0F9
:107930005FE30F947A0C9B01AC0169897A898B898A
:107940009C890F946D0920E030E040EA52E40F94E6
:107950007A0C6B017C0120E030E0A9010F94D20980
:1079600087FF31C0F7FAF094F7F8F09422E0B701FE
:10797000A6018AE690E20E949BA1209177073091B0
:1079800078074091790750917A07C701B6010F94A3
:10799000D9099B01AC010F946E096B017C0122E0B7
:1079A000AB01BC018AE690E20E949BA1A70196016F
:1079B00060917707709178078091790790917A07A5
:1079C0000F946D0918C08090770790907807A09069
:1079D0007907B0907A07A5019401C701B6010F9409
:1079E000D9099B01AC010F946E099B01AC01C50143
:1079F000B4010F946E0960937707709378078093B2
:107A0000790790937A072EEA37E44FE053E46091C8
:107A10007707709178078091790790917A070F9492
:107A2000D9096B017C012DEC3CEC4CE85FE30F9431
:107A3000060C181654F026E636E646E65FE3C70164
:107A4000B6010F94D20987FF12C08EEA97E4AFE027
:107A5000B3E48093770790937807A0937907B09366
:107A60007A0722E0AC01BD018DEC97E014C022E062
:107A7000498D5A8D6B8D7C8D80EC97E00E949BA187
:107A800040917707509178076091790770917A0754
:107A900022E083EB97E00E949BA18D859E85AF85B8
:107AA000B8898093030790930407A0930507B093C8
:107AB000060781E00E94C78781E00E94F0808EEA7D
:107AC00097E00E94511E8EE390E20E942A962D8537
:107AD0003E854F85588920930307309304074093D0
:107AE00005075093060741E061E081E00E94E187CD
:107AF00080E00E945BCFF8C6809103079091040755
:107B0000A0910507B09106078D8F9E8FAF8FB8A308
:107B100024E130E040E050E02D873E874F87588BCE
:107B2000D1018D919C91119792FF0CC05E968D9121
:107B30009D910D90BC91A02D0297A105B10511F466
:107B40000C94A34B41E061E081E00E94E1878FE368
:107B500090E20E942A9680E00E94C7870E94791DC9
:107B6000162F072FF82EE92E84E393E00E942D1D97
:107B70009B01AC0180E393E029AF3AAF4BAF5CAF20
:107B80000E942D1DEF92FF920F931F9300EFA02EE6
:107B900003E2B02E04E7C02E09E4D02E8601750161
:107BA00029AD3AAD4BAD5CAD0E949E8520E041E031
:107BB00060E081E00E947088698F7A8F8B8F9C8F44
:107BC00020E041E060E081E00E94708869A37AA330
:107BD0008BA39CA39B01AC01698D7A8D8B8D9C8DB1
:107BE0000F946D096B017C010F900F900F900F9017
:107BF0002DEC3CEC4CEC5DE30F94060C181654F0A5
:107C00002DEC3CEC4CEC5DEBC701B6010F94D209B6
:107C100087FF2BC04D855E856F8578898EE897E05C
:107C20000E94BFA02D853E854F8558892832310599
:107C3000410551050CF074CF82E30E948023D101ED
:107C40008D919C9192FF6CCF2D853E854F855889F3
:107C50002E5F3F4F4F4F5F4F2D873E874F87588B8B
:107C6000BA01A90180E797E086C08DE793E00F9401
:107C700051129A8B898B0E94791D162F072FF82E8F
:107C8000E92E8CE393E00E942D1D9B01AC0188E35B
:107C900093E029AF3AAF4BAF5CAF0E942D1DEF923E
:107CA000FF920F931F9310EFA12E13E2B12E14E752
:107CB000C12E19E4D12E8601750129AD3AAD4BAD27
:107CC0005CAD0E949E8521E041E060E080E00E9482
:107CD00070886DA37EA38FA398A721E041E060E0A8
:107CE00080E00E94708869A77AA78BA79CA79B0158
:107CF000AC016DA17EA18FA198A50F946D096B01B8
:107D00007C010F900F900F900F902DEC3CEC4CEC01
:107D10005DE30F94060C181654F02DEC3CEC4CEC83
:107D20005DEBC701B6010F94D20987FF32C04D85C4
:107D30005E856F85788980E597E00E94BFA08D857C
:107D40009E85AF85B8898897A105B1050CF0E8CE6E
:107D500082E30E9480232D853E854F8558892E5FC2
:107D60003F4F4F4F5F4F2D873E874F87588BBA014C
:107D7000A90182E397E00E94BFA06D8582E30E9483
:107D80005D236D858AE30E945D2382E30E94802348
:107D9000C7CE8FE793E00F9451129E8B8D8B0E947C
:107DA000791D162F072FF82EE92E84E493E00E9408
:107DB0002D1D9B01AC0180E493E029AF3AAF4BAF9E
:107DC0005CAF0E942D1DEF92FF920F931F93B0EFB7
:107DD000AB2EB3E2BB2EB4E7CB2EB9E4DB2E86018B
:107DE000750129AD3AAD4BAD5CAD0E949E8521E099
:107DF00041E061E080E00E9470884B015C0121E07D
:107E000041E061E080E00E9470886B017C019B0191
:107E1000AC01C501B4010F946D092B013C010F9019
:107E20000F900F900F902DEC3CEC4CEC5DE30F9419
:107E3000060C181654F02DEC3CEC4CEC5DEBC30139
:107E4000B2010F94D20987FF25C04D855E856F85ED
:107E5000788982E197E00E94BFA08D859E85AF85DD
:107E6000B8898897A105B1050CF05ACE82E30E942B
:107E700080232D853E854F8558892E5F3F4F4F4F7C
:107E80005F4F2D873E874F87588BBA01A90184EF3A
:107E900096E071CFA5019401C701B6010F946E0958
:107EA00020E030E040E05FE30F947A0C6DA77EA7FE
:107EB0008FA798AB81E893E00F9451128C01D10108
:107EC0008D919C91119792FF0CC05E968D919D9122
:107ED0000D90BC91A02D892B8A2B8B2B11F00C942B
:107EE000B64B298D3A8D4B8D5C8D69A17AA18BA102
:107EF0009CA10F946E0920E030E040E05FE30F9416
:107F00007A0C698F7A8F8B8F9C8F2D8D3E8D4F8D44
:107F100058A120930307309304074093050750931B
:107F2000060781E00E94C787D1018D919C9111972E
:107F300092FFABC05E968D919D910D90BC91A02D4E
:107F40000297A105B10509F0A0C020E030E040EAA9
:107F500052E4698D7A8D8B8D9C8D0F947A0C20E084
:107F600030E048EC54E40F946D090F94720A6B01F1
:107F70007C0129893A89442737FD4095542F298B64
:107F80003A8B4B8B5C8B2DA13EA14FA158A569A5C7
:107F90007AA58BA59CA50F946E0920E030E040E007
:107FA0005FE30F947A0C20E030E040EA52E40F9453
:107FB0007A0C20E030E048EC54E40F946D090F9403
:107FC000720A2B013C018D899E89AA2797FDA095F5
:107FD000BA2F8D8B9E8BAF8BB88F20E030E040EABC
:107FE00052E46DA57EA58FA598A90F947A0C20E088
:107FF00030E048EC54E40F946D090F94720A4B0181
:108000005C01222717FD2095322FC414D504E60405
:10801000F70414F00C94CE4BC814D904EA04FB0402
:1080200014F00C94F64B4C185D086E087F088D898F
:108030009E89AF89B88D480E591E6A1E7B1E8C180A
:108040009D08AE08BF08800E911EA21EB31EC2017D
:108050000E94E11DC4010E94011EC12CD12C760199
:10806000A1E94A16A1E05A066104710414F00C94C7
:108070002A4CB1E98B16B1E09B06A104B10414F0BF
:108080000C942A4C80E00E945BCF20E030E0A901F4
:10809000698D7A8D8B8D9C8D0F94D20987FD40CD93
:1080A00020E030E0A9016DA57EA58FA598A90F94C9
:1080B000D20987FD35CD81E00E94F0808AEB96E001
:1080C0000E94511E8EE390E20E942A962D8D3E8DD5
:1080D0004F8D58A120930307309304074093050761
:1080E0005093060741E061E081E00E94E187FCC314
:1080F00010920E08F101EB5AFF4F8081882309F49A
:10810000F3C385EA96E00CC081E080930E08F1018C
:10811000EB5AFF4F8081882309F4E6C380E996E09B
:108120000E94B39FE1C38090C9079090CA07A090B6
:10813000CB07B090CC074090CD075090CE07609011
:10814000CF077090D007C090D107D090D207E090B1
:10815000D307F090D407D1011C9113FF2BC01A96BE
:10816000EC911A971B96FC911B971C960C911C97EF
:108170001D96BC9080915108882361F023E333E37E
:108180004BEC51E4BF01802F9B2D0F947A0CFB0127
:10819000DC0102C0A02FBB2D2091F1073091F20726
:1081A0004091F3075091F407BF01CD010F946D0981
:1081B0004B015C0114FF2CC0D1011E96EC911E975F
:1081C0001F96FC911F9750960C91509751967C905A
:1081D00080915108882361F023E333E34BEC51E4B1
:1081E000BF01802F972D0F947A0CFB01DC0102C098
:1081F000A02FB72D2091F5073091F6074091F70792
:108200005091F807BF01CD010F946D092B013C017E
:1082100015FF2CC0D1015296EC9152975396FC91C8
:10822000539754961C91549755960C9180915108F0
:10823000882361F023E333E34BEC51E4BF01812F4A
:10824000902F0F947A0CFB01DC0102C0A12FB02FFC
:108250002091F9073091FA074091FB075091FC07F4
:10826000BF01CD010F946D096B017C01870176017F
:10827000A3019201C501B4010E94BC79F101808182
:1082800086FF32C3E689D1015796FC9157975896DD
:108290001C91589759960C9180915108882361F050
:1082A00023E333E34BEC51E4BF01812F902F0F9474
:1082B0007A0CFB01DC0102C0A12FB02F2091330307
:1082C000309134034091350350913603BF01CD0105
:1082D0000F947A0C0F94720A6093090870930A083D
:1082E00080930B0890930C08FFC28090F907909040
:1082F000FA07A090FB07B090FC0720910B07309184
:108300000C0740910D0750910E07C501B4010F9461
:10831000D9092DEC3CEC4CEC5DE30F94060C1816DF
:108320002CF48AE596E00E94BD9FDEC2F101228115
:108330008081918122FF0CC083FF02C00C94464CC7
:1083400080739927892B11F00C94464C0C944C4C5B
:1083500083FF6FC0C284D384E484F58420E030E0DE
:10836000A901C701B6010F94060C181664F420E0A9
:1083700030E040E251E4C701B6010F94D20918166B
:108380000CF459C00AC020E030E040E251ECC701D3
:10839000B6010F94060C87FD4EC0A5019401C701DC
:1083A000B6010F946E099B01AC01609117077091A3
:1083B00018078091190790911A070F946E0960931E
:1083C0001707709318078093190790931A070E9454
:1083D000E774409117075091180760911907709141
:1083E0001A0723E08DE595E00E949BA18091170775
:1083F00090911807A0911907B0911A0789879A8759
:10840000AB87BC8744E050E065E870E0CE01099698
:108410000F9456120E9444CF682F88E690E069AF0F
:108420000F94441269AD681721F088E690E00F942C
:108430005F1210E001C011E0F101808184FF71C082
:10844000C684D784E088F18820E030E0A901C70124
:10845000B6010F94060C181664F420E030E040E2F8
:1084600051E4C701B6010F94D20918160CF458C094
:108470000AC020E030E040E251ECC701B6010F94A1
:10848000060C87FD4DC0A5019401C701B6010F94EC
:108490006E099B01AC0160910F07709110078091EC
:1084A0001107909112070F946E0960930F07709354
:1084B000100780931107909312070E94E774409170
:1084C0000F0750911007609111077091120723E078
:1084D00082E495E00E949BA180910F079091100784
:1084E000A0911107B09112078D839E83AF83B88747
:1084F00044E050E069E870E0CE0105960F94561212
:108500000E9444CF682F88E690E069AF0F94441230
:1085100069AD681731F088E690E00F945F1201C0F2
:1085200011E0D1018C9185FF74C05296CD90DD9001
:10853000ED90FC90559720E030E0A901C701B6010D
:108540000F94060C18165CF420E030E040E251E491
:10855000C701B6010F94D20918165CF00EC020E0D6
:1085600030E040E251ECC701B6010F94060C87FFE2
:1085700004C08BEA95E00C94484CA5019401C70116
:10858000B6010F946E099B01AC01609107077091D1
:1085900008078091090790910A070F946E0960936C
:1085A0000707709308078093090790930A070E94B2
:1085B000E77440910707509108076091090770918F
:1085C0000A0723E087E295E00E949BA180910707BC
:1085D00090910807A0910907B0910A0789839A83AF
:1085E000AB83BC8344E050E06DE870E0CE010196BF
:1085F0000F9456120E9444CF682F88E690E069AF2E
:108600000F94441269AD681721F088E690E00F944A
:108610005F121111AECF89E48F9384E78F9383E2C9
:108620008F9380EF8F93F0EFAF2EF3E2BF2EF4E73E
:10863000CF2EF9E4DF2EE12CF12C00E411E4A601A9
:108640009501C601B5010E949E850F900F900F9075
:108650000F904AC180E00E94C7871092C90710920C
:10866000CA071092CB071092CC071092CD07109238
:10867000CE071092CF071092D0071092D107109218
:10868000D2071092D3071092D40760911303709110
:10869000140380911503909116030E943F7A8091F4
:1086A000470790914807A0914907B0914A07409128
:1086B0003F07509140076091410770914207C09079
:1086C0004307D0904407E0904507F09046075A01D1
:1086D000F62FE72F481759076A077B071CF45C0140
:1086E000FA2FEB2F85012F2F3E2F0C151D052E0580
:1086F0003F0514F497018601480159018C189D0823
:10870000AE08BF0868017901C41AD50AE60AF70A5B
:1087100028013901481A590A6A0A7B0AB501A401DD
:1087200080E093E20E94BFA0B701A60187EF92E22A
:108730000E94BFA0B301A2018EEE92E20E94BFA0F0
:10874000F1018081918192FFCDCC868D978DA0A182
:10875000B1A1181619061A061B060CF0C3CCC401E9
:108760000E94C11DC6010E94E11DC2010E94011E9E
:10877000B9CC7090C80775FA772470F880E00E9431
:10878000C7871092FD071092FE071092FF07109204
:10879000000810920108109202081092030810922B
:1087A000040810920508109206081092070810920B
:1087B00008081092C9071092CA071092CB071092AE
:1087C000CC071092CD071092CE071092CF071092CF
:1087D000D0071092D1071092D2071092D3071092AF
:1087E000D4071092110810921208109213081092D8
:1087F000140810921508109216081092170810927B
:1088000018081092190810921A0810921B0810925A
:108810001C086091130370911403809115039091CB
:1088200016030E943F7A00912B0710912C0720918C
:108830002D0730912E0780911F0790912007A0915E
:108840002107B0912207081B190B2A0B3B0B08517B
:108850001C4F2F4F3F4F80913F0790914007A091B1
:108860004107B091420748015901881A990AAA0A9A
:10887000BB0A8091470790914807A0914907B091A2
:108880004A0768017901C81AD90AEA0AFB0A8091E5
:10889000430790914407A0914507B0914607B9015D
:1088A000A801481B590B6A0B7B0B80E093E20E94E6
:1088B000BFA0B501A40187EF92E20E94BFA0B7015B
:1088C000A6018EEE92E20E94BFA0872D0E94C7876C
:1088D00009CC8091EA0282FF07C08CE594E20E94F5
:1088E000839FC1010E9471970F94090460938C1DAE
:1088F00070938D1D80938E1D90938F1DEC960FB6F7
:10890000F894DEBF0FBECDBFDF91CF911F910F91C5
:10891000FF90EF90DF90CF90BF90AF909F908F909F
:108920007F906F905F904F903F902F9008958FEAC7
:108930009CE00E942A9687EA9CE00E94839F0E9406
:10894000701D882321F084EA9CE00E94839F0E948E
:10895000751D882321F081EA9CE00E94839F37994E
:1089600022C08EE79CE01CC08DE19CE00E942A960C
:1089700085E19CE00E94839F0E94701D882321F066
:1089800082E19CE00E94839F0E94751D882321F054
:108990008FE09CE00E94839F3799F1C48CEE9BE0AE
:1089A0000E949C9FA1CF8EE99CE00E94839FD9CF1B
:1089B0008FE390E20E942A9680E00E94C7870E947F
:1089C000791D162F072FF82EE92E84E393E00E94DD
:1089D0002D1D9B01AC0180E393E029AF3AAF4BAF73
:1089E0005CAF0E942D1DEF92FF920F931F9350EFEB
:1089F000A52E53E2B52E54E7C52E59E4D52E860197
:108A0000750129AD3AAD4BAD5CAD0E949E8520E06D
:108A100041E060E081E00E94708869A77AA78BA797
:108A20009CA720E041E060E081E00E94708869A39B
:108A30007AA38BA39CA39B01AC0169A57AA58BA506
:108A40009CA50F946D096B017C010F900F900F9006
:108A50000F902DEC3CEC4CEC5DE30F94060C1816DB
:108A600054F02DEC3CEC4CEC5DEBC701B6010F94DF
:108A7000D20987FF1AC049895A896B897C8982EC9F
:108A80009BE00E94BFA089899A89AB89BC8988979D
:108A9000A105B10511F40C94103882E30E948023E3
:108AA000B301A20184EA9BE01BC18DE793E00F9420
:108AB00051129E8B8D8BD1018D919C91119792FFBC
:108AC0000BC05E968D919D910D90BC91A02D02974B
:108AD000A105B10509F458C40E94791D162F072F6E
:108AE000F82EE92E8CE393E00E942D1D9B01AC0132
:108AF00088E393E029AF3AAF4BAF5CAF0E942D1DE6
:108B0000EF92FF920F931F9300EFA02E03E2B02E7F
:108B100004E7C02E09E4D02E8601750129AD3AADD7
:108B20004BAD5CAD0E949E8520E041E060E081E0BD
:108B30000E9470886DA77EA78FA798AB20E041E0C8
:108B400060E081E00E94708869AB7AAB8BAB9CAB34
:108B50009B01AC016DA57EA58FA598A90F946D0909
:108B60006B017C010F900F900F900F902DEC3CEC5F
:108B70004CEC5DE30F94060C181654F02DEC3CEC15
:108B80004CEC5DEBC701B6010F94D20987FF21C001
:108B900049895A896B897C898FE49BE00E94BFA038
:108BA00029893A894B895C8928323105410551056B
:108BB00041F082E30E948023B301A20181E39BE0A4
:108BC0008FC08EE19BE00E949C9F86E09BE00C940E
:108BD00016388FE793E00F9451129E8F8D8FD1013D
:108BE0008D919C91119792FF0BC05E968D919D91F6
:108BF0000D90BC91A02D0297A105B10509F4D1C338
:108C00000E94791D162F072FF82EE92E84E493E099
:108C10000E942D1D9B01AC0180E493E029AF3AAF87
:108C20004BAF5CAF0E942D1DEF92FF920F931F93ED
:108C300010EFA12E13E2B12E14E7C12E19E4D12EAC
:108C40008601750129AD3AAD4BAD5CAD0E949E85A4
:108C500020E041E060E081E00E9470886B017C01CF
:108C600020E041E060E081E00E9470886DAB7EAB67
:108C70008FAB98AF9B01AC01C701B6010F946D0992
:108C80004B015C010F900F900F900F902DEC3CEC7E
:108C90004CEC5DE30F94060C181654F02DEC3CECF4
:108CA0004CEC5DEBC501B4010F94D20987FF42C0C3
:108CB00049895A896B897C898CED9AE00E94BFA012
:108CC00029893A894B895C8928323105410551054A
:108CD00049F182E30E948023B301A2018EEB9AE066
:108CE0000E94BFA0642D82E30E945D23642D8AE36D
:108CF0000E945D2382E30E948023F2E04F0E511C0C
:108D0000611C711C29893A894B895C892E5F3F4F10
:108D10004F4F5F4F298B3A8B4B8B5C8B31E03DA3E0
:108D20000C94DD378BEA9AE00E949C9F83E99AE0DD
:108D30000C94163829A13AA14BA15CA169A57AA58A
:108D40008BA59CA50F946E0920E030E040E05FE326
:108D50000F947A0C20E030E040EA52E40F947A0C51
:108D600020E030E048EC54E40F946D090F94720A4F
:108D70004B015C018D899E89AA2797FDA095BA2F8A
:108D80008D8B9E8BAF8BB88F29A93AA94BA95CA973
:108D90006DA57EA58FA598A90F946E0920E030E0FF
:108DA00040E05FE30F947A0C20E030E040EA52E4C8
:108DB0000F947A0C20E030E048EC54E40F946D09F5
:108DC0000F94720A2B013C012D8D3E8D442737FDF7
:108DD0004095542F2D8F3E8F4F8F58A32DA93EA91C
:108DE0004FA958ADC701B6010F946E0920E030E0DD
:108DF00040E05FE30F947A0C20E030E040EA52E478
:108E00000F947A0C20E030E048EC54E40F946D09A4
:108E10000F94720A6B017C0181E893E00F94511268
:108E20009C01442737FD4095542F29A33AA34BA317
:108E30005CA380E00E94F0800E94E7748BE590E2E2
:108E40000E94B39F40910B0750910C0760910D0752
:108E500070910E0722E086EC9FE10E949BA1898D14
:108E60009A8DAB8DBC8D8093030790930407A093DC
:108E70000507B093060784149504A604B70414F5F7
:108E80008C149D04AE04BF040CF042C0481859086D
:108E90006A087B082D8D3E8D4F8D58A1420E531EC2
:108EA000641E751EC818D908EA08FB0889A19AA192
:108EB000ABA1BCA1C80ED91EEA1EFB1E812C912CB1
:108EC000540152C0481459046A047B040CF54C1434
:108ED0005D046E047F04E4F484189508A608B708BE
:108EE0002D893E894F89588D820E931EA41EB51E72
:108EF000C418D508E608F70889A19AA1ABA1BCA1BE
:108F0000C80ED91EEA1EFB1E412C512C320125C071
:108F1000C814D904EA04FB0404F5C414D504E60417
:108F2000F704DCF48C189D08AE08BF082D893E8933
:108F30004F89588D820E931EA41EB51E4C185D08D5
:108F40006E087F088D8D9E8DAF8DB8A1480E591E7D
:108F50006A1E7B1EC12CD12C760191E9891691E005
:108F60009906A104B10474F4A1E94A16A1E05A06D5
:108F7000610471043CF4B1E9CB16B1E0DB06E10415
:108F8000F104FCF049895A896B897C8982E69AE070
:108F90000E94BFA088E49AE00E942A96B501A4012D
:108FA00084E49AE00E94BFA0B301A20180E49AE0A9
:108FB0000E94BFA0B701A6018CE39AE00E94BFA067
:108FC00093CCC4010E94C11DC2010E94E11DC601D3
:108FD0000E94011E80E00E945BCF0C9420382DEC93
:108FE0003CEC4CEC5DEBC301B2010F94D20987FF5E
:108FF00009C00C94963882ED99E00E949C9F8AEB00
:1090000099E0D0C09FEF291A390AA5019401C70140
:10901000B6010F946E0920E030E040E05FE30F946A
:109020007A0C2B013C0140910B0750910C07609189
:109030000D0770910E0722E08CEA99E00E949BA137
:109040002091F9073091FA074091FB075091FC07F6
:10905000C301B2010F946D099B01AC0160910B0734
:1090600070910C0780910D0790910E070F946E0977
:1090700060930B0770930C0780930D0790930E0776
:109080000E94E77440910B0750910C0760910D0707
:1090900070910E0722E08EE999E00E949BA10E9448
:1090A000791D162F072FF82EE92E84E493E00E94F5
:1090B0002D1D9B01AC0180E493E029AF3AAF4BAF8B
:1090C0005CAF0E942D1DEF92FF920F931F93A0EFB4
:1090D000AA2EA3E2BA2EA4E7CA2EA9E4DA2E8601AC
:1090E000750129AD3AAD4BAD5CAD0E949E8520E087
:1090F00041E060E081E00E9470886B017C0120E02B
:1091000041E060E081E00E9470886D8B7E8B8F8BE8
:10911000988F9B01AC01C701B6010F946D094B01FB
:109120005C010F900F900F900F902DEC3CEC4CECED
:109130005DE30F94060C181654F02DEC3CEC4CEC4F
:109140005DEBC501B4010F94D20987FF33C04D8593
:109150005E856F8578898FE699E00E94BFA02D8596
:109160003E854F8558892832310541055105A4F4C3
:1091700082E30E9480238D859E85AF85B889029603
:10918000A11DB11D8D879E87AF87B88BAC01BD0136
:1091900081E599E00C94BB388EE399E00E949C9F96
:1091A00086E299E00E942A9686ED9FE10E94BD9F8B
:1091B0000C94CD382D893E894F89588DC701B60151
:1091C0000F946E0920E030E040E05FE30F947A0CEA
:1091D0009B01AC01C301B2010F946D0920E030E0A6
:1091E00040EA52E40F947A0C6B017C0120E030E0FD
:1091F000A9010F94D20987FF27C0C701B601905873
:1092000020917707309178074091790750917A073C
:109210000F94D9099B01AC010F946E096B017C017D
:1092200022E0AB01BC018AE690E20E949BA1A7016B
:1092300096016091770770917807809179079091F6
:109240007A070F946D0918C080907707909078077F
:10925000A0907907B0907A07A5019401C701B601E3
:109260000F94D9099B01AC010F946E099B01AC01CD
:10927000C501B4010F946E09609377077093780766
:109280008093790790937A07C0907707D0907807FA
:10929000E0907907F0907A0720E030E040E153E475
:1092A000C701B6010F94D9094B015C012DEC3CECD0
:1092B0004CE85FE30F94060C181654F026E636E6E9
:1092C00046E65FE3C501B4010F94D20987FF13C0DE
:1092D00022E0B701A6018BE099E00E949BA180E00B
:1092E00090E0A0E1B3E48093770790937807A09390
:1092F0007907B0937A0722E049895A896B897C897A
:1093000083EF98E00E949BA14091770750917807E6
:109310006091790770917A0722E08BED98E00E94C6
:109320009BA194E02916310414F00C94CD382989BE
:109330003A894B895C8960917707709178078091B1
:10934000790790917A070F946D096B017C012DECE0
:109350003CEC4CEC5DE30F94060C181614F40C94E2
:1093600039382DEC3CEC4CEC5DEBC701B6010F94A9
:10937000D20987FF02C00C9439380C94CD388CE0A8
:109380009CE00E94839F0ACB41E061E081E00E9463
:10939000E1878FE390E20E942A9680E00E94C787CF
:1093A0009BCB41E061E081E00E94E1878FE390E2A6
:1093B0000E942A9680E00E94C78722CCC90188714A
:1093C0009927489709F474C120E041E060E081E00A
:1093D0000E9470882091F9073091FA074091FB07AD
:1093E0005091FC070F946D094B015C0120E041E0B6
:1093F00061E080E00E9470882091F9073091FA07BF
:109400004091FB075091FC070F946D092B013C0123
:109410009B01AC01C501B4010F946D096B017C0186
:109420002DEC3CEC4CEC5DE30F94060C181654F05C
:109430002DEC3CEC4CEC5DEBC701B6010F94D2096E
:1094400087FF21C022E0B701A6018AE998E00E94C7
:109450009BA182E30E94802346E150E060E070E03F
:109460008CE798E00E94BFA066E182E30E945D2342
:1094700066E18AE30E945D2382E30E94802388E7FD
:1094800098E00C940839A3019201C501B4010F942E
:109490006E0920E030E040E05FE30F947A0CAB010E
:1094A000BC0122E089E698E00E949BA11DCA809140
:1094B000030790910407A0910507B09106078D87D7
:1094C0009E87AF87B88BF1018081918192FF09C09F
:1094D000868D978DA0A1B1A10297A105B10509F4D0
:1094E000AEC041E061E081E00E94E1878FE390E25D
:1094F0000E942A9680E00E94C7870E94791D9F9350
:109500008F937F936F93F0EFAF2EF3E2BF2EF4E7CC
:10951000CF2EF9E4DF2E8601750120E030E0A901AD
:10952000CA01B9010E949E8520E041E060E081E02F
:109530000E9470884B015C0120E041E060E081E026
:109540000E9470886B017C019B01AC01C501B401D4
:109550000F946D092B013C010F900F900F900F900D
:109560002DEC3CEC4CEC5DE30F94060C181654F01B
:109570002DEC3CEC4CEC5DEBC301B2010F94D20935
:1095800087FF05C086ED9FE10E94BD9F9CCFA5018E
:109590009401C701B6010F946E0920E030E040E06D
:1095A0005FE30F947A0C6B017C0120E030E040E82F
:1095B0005FE30F94D20987FD86CFD1018D919C91F5
:1095C000119792FF0BC05E968D919D910D90BC916D
:1095D000A02D892B8A2B8B2B09F043C02D853E852E
:1095E0004F8558892093030730930407409305075C
:1095F0005093060781E00E94C787D1018D919C910D
:10960000119792FF0BC05E968D919D910D90BC912C
:10961000A02D0297A105B10509F446C081E00E9482
:10962000F08087EB98E00E94511E8EE390E20E944A
:109630002A962D853E854F8558890C946A4020E0F6
:1096400030E845EC53E420930B0730930C0740932C
:109650000D0750930E0780E00E945BCF0E94B8D1A7
:1096600040CF2091F9073091FA074091FB075091C4
:10967000FC07C701B6010F946D099B01AC01609115
:109680000B0770910C0780910D0790910E070F94B6
:109690006E0960930B0770930C0780930D079093EE
:1096A0000E070E94E7749ACF80E00E945BCFB6CF8E
:1096B00030FF27C0D1011E962D913D914D915C91B7
:1096C00051971A966D917D918D919C911D975D9604
:1096D000EC915D97EF935C96EC915C97EF935B96C2
:1096E000EC915B97EF935A96EC91EF93E0EFAE2EEF
:1096F000E3E2BE2EE4E7CE2EE9E4DE2E860175011C
:109700001BC00E94791DF10126853785408951894A
:1097100042845384648475849F938F937F936F9363
:1097200060EFA62E63E2B62E64E7C62E69E4D62E5D
:1097300086017501C301B2010E949E850F900F90B2
:109740000F900F9041CE80E090E00E94C11D80E01C
:1097500090E00E94E11D80E090E00E94011E80E008
:109760000E945BCF0E94B8D10C94A23D80E00E9481
:10977000F0800E94E7748BE590E20E94B39F4091D5
:109780000B0750910C0760910D0770910E0722E0B6
:1097900086EC9FE10E949BA10C94713F4C145D04E8
:1097A0006E047F041CF5481459046A047B04F4F425
:1097B000C418D508E608F70889899A89AB89BC8955
:1097C000C80ED91EEA1EFB1E84189508A608B70805
:1097D000800E911EA21EB31EC6010E94C11DC401AF
:1097E0000E94011E412C512C32012BC08C149D046F
:1097F000AE04BF0434F584149504A604B7040CF534
:10980000C818D908EA08FB0829893A894B895C8974
:10981000C20ED31EE41EF51E481859086A087B08BC
:109820008D899E89AF89B88D480E591E6A1E7B1E90
:10983000C6010E94C11DC2010E94E11D812C912C14
:10984000540191E9C91691E0D906E104F10414F438
:109850000C9430404D855E856F8578898BEC96E061
:109860000E94BFA0B701A60187EC96E00E94BFA0AE
:10987000B301A20183EC96E00E94BFA0B501A40150
:109880008FEB96E00E94BFA00C94903D80E396E0A1
:109890000E94BD9F0C940B43C6A4D7A4E0A8F1A8D6
:1098A00020E030E0A901C701B6010F94D209882356
:1098B00061F120E030E0A901C701B6010F94060C68
:1098C00018165CF420E030E040E251E4C701B60134
:1098D0000F94D2091816B4F00AC020E030E040E23C
:1098E00051ECC701B6010F94060C87FD0BC085E74C
:1098F00093E00E942D1D9B01AC01C701B6010F949E
:109900006E094DC087E096E0C3CF20E030E0A901AA
:109910006091F1077091F2078091F3079091F4073D
:109920000F94D209811161C020E030E0A90160915B
:10993000F5077091F6078091F7079091F8070F945B
:10994000D209811152C08091C80787FF2CC0C090F6
:109950008307D0908407E0908507F0908607609198
:1099600015087091160880911708909118080F94A7
:10997000A30A9B01AC010F947A0C9B01AC01C701B7
:10998000B6010F946D090F94E70C209149083091AE
:109990004A0840914B0850914C080F947A0C0E9451
:1099A0007C1D0C940B43C0908307D0908407E090FB
:1099B0008507F090860760911508709116088091D0
:1099C0001708909118089B01AC010F94410DC61A1D
:1099D000D70AE80AF90AC701B6010E94EED9BC010C
:1099E00080E090E00F94A30AD0CF84ED95E050CFB3
:1099F000CF93DF93EC014091EA028881998144FF83
:109A000009C082FD2AC081FF05C02E813F812F360B
:109A1000310519F582FF05C0CE01DF91CF910C947D
:109A2000BF3581FF05C0CE01DF91CF910C948B240F
:109A300091FF08C00E94431ECC5ADF4F8881DF91FE
:109A4000CF91E1C242FF13C08CE594E20E94839F54
:109A5000CE01DF91CF910C9471970F94090460931C
:109A60008C1D70938D1D80938E1D90938F1DDF91A3
:109A7000CF9108958091C60780FD1DC00E94649813
:109A80000E94F092EC0186E79AE00E9478CA209743
:109A9000B1F080918D09882341F0888181FF12C047
:109AA0008E819F814D9771F416C0CE01A1DFCE014A
:109AB0000E944F9804C086E79AE00E9478CA0E94EC
:109AC000DD79D8CFBE0182E299E00E948C9BCE0165
:109AD0000E943E98ECCF82E299E00E94019FF7CF6E
:109AE0000E946C8C0C949B23C5CFCF93DF93FC0119
:109AF000E05CFF4F208121FD1FC0DB014D915D9196
:109B00006D917C91DC01AF5BBF4F4D935D936D9385
:109B10007C931397EC01CB5BDF4FDC0117964D91E3
:109B20005D916D917C911A97488359836A837B83F9
:109B3000822F897F82608083DF91CF9108959F92E9
:109B4000AF92BF92CF92DF92EF92FF920F931F934B
:109B5000CF93DF93EC015B018C01005C1F4FF80198
:109B6000908092FC32C0CB84DC84ED84FE84A7011B
:109B700096016F81788589859A850F946D099F7705
:109B800020E030E040E85FE30F946E0920E030E031
:109B900040EA51E40F94060C1816BCF0F5018081E0
:109BA0009181A281B381FE01EF5BFF4F808391839E
:109BB000A283B383CB5BDF4FC882D982EA82FB8268
:109BC000892D897F8460F8018083DF91CF911F9177
:109BD0000F91FF90EF90DF90CF90BF90AF909F904C
:109BE00008958091C80784608093C80708952F92D4
:109BF0003F924F925F926F927F928F929F92AF921D
:109C0000BF92CF92DF92EF92FF920F931F93CF9369
:109C1000DF93CDB7DEB764970FB6F894DEBF0FBE03
:109C2000CDBF382E292E7A8769875A834983098BBD
:109C30001A8B2B8B3C8B4AA45BA46CA47DA423E3DE
:109C400033E948E853E4C501B4010F946E096D830C
:109C50007E838F83988720E030E0A901C301B201A1
:109C60000F94D209882359F12EA53FA548A959A9D7
:109C7000C301B2010F946E094B015C0120E030E09A
:109C800040EA50E4C301B2010F947A0CA50194019B
:109C90000F94D9096D877E878F87988BA3019201D6
:109CA0006EA57FA588A999A90F947A0CA5019401A6
:109CB0000F94D9096EA77FA788AB99AB08C080E045
:109CC00090E0A0EAB0E48D879E87AF87B88B2D81A6
:109CD0003E814F81588569897A898B899C89905802
:109CE0000F94D9090F94460A9B01AC01C701B60134
:109CF0000F947A0C6D837E838F83988769817A8134
:109D0000A985BA856A1B7B0B882777FD8095982FDC
:109D10000F94A50A20E030E040E05DE30F947A0C58
:109D200069877A878B879C87032D122D212C312CF4
:109D300089819A81AA2797FDA095BA2F89839A8352
:109D4000AB83BC83A89569817A818B819C810F94B8
:109D5000A50A6B017C01B101882777FD8095982FBA
:109D60000F94A50A29853A854B855C850F947A0C5A
:109D70009B01AC01C701B6010F946D096B017C0119
:109D800023E333E548E853E40F946E099B01AC01EB
:109D900069897A898B899C890F94D9090F94460A1D
:109DA0002D813E814F8158850F947A0C4B015C01C7
:109DB00020E030EC4FE755E40F947A0C2D853E857A
:109DC0004F8558890F947A0C2B013C01A501940111
:109DD0006EA57FA588A999A90F946E0920E030E0AF
:109DE00040EA50E40F947A0C9B01AC01C301B2012C
:109DF0000F94D9090F94720A6D3F9FE0790714F010
:109E00006CEF7FE0D8016D937C9320E030E040E080
:109E100051E4C701B6010F947A0C0F94720AF8014D
:109E200073836283FFEF2F1A3F0A0C5F1F4F81E29B
:109E30002816310409F086CF64960FB6F894DEBF79
:109E40000FBECDBFDF91CF911F910F91FF90EF908B
:109E5000DF90CF90BF90AF909F908F907F906F904A
:109E60005F904F903F902F900895CF92DF92EF92A6
:109E7000FF92CF93DF93EC018B898130A9F5CE8CD3
:109E8000DF8CE8A0F9A020E030E0A901C701B6010D
:109E90000F94D209882341F1688D70E080E090E052
:109EA0000F94A30A20E030E040E251E40F947A0CD2
:109EB000A70196010F94D9096FA378A789A79AA73C
:109EC000698D70E080E090E00F94A30A20E030E01C
:109ED00040E251E40F947A0CA70196010F94D9093E
:109EE0006BA77CA78DA79EA7DF91CF91FF90EF90E6
:109EF000DF90CF9008958EE092E0B7CF7F928F925F
:109F00009F92AF92BF92CF92DF92EF92FF920F9308
:109F10001F93CF93DF938BE592E09093910380930F
:109F2000900385E4782E7F92D2E9DF93C0EECF9341
:109F30001F921F921F921F921F92812C912C98ECBE
:109F4000A92E91E4B92EC12C20E5D22E23ECE22ECD
:109F500027E4F22E00E010E12BE835E44CE251E07A
:109F60006EEC7FEF87E194E042DE7F92DF93CF9348
:109F70001F921F921F921F921F9200E018E728E87D
:109F800035E44CE251E06CEE7FEF83E993E02FDEA5
:109F900080910A01806480930A013B9A8091680253
:109FA0002DB73EB7205F3F4F0FB6F8943EBF0FBEB0
:109FB0002DBF87FD0CC061E00F941D0580916902E3
:109FC000811105C061E0809168020F9456050F94DD
:109FD0000904609395027093960280939702909380
:109FE00098026D9A759887DFDF91CF911F910F913D
:109FF000FF90EF90DF90CF90BF90AF909F908F90A9
:10A000007F900C94E2DA4F925F926F927F92AF92C0
:10A01000BF92CF92DF92EF92FF920F931F93CF9355
:10A02000DF93CDB7DEB72C970FB6F894DEBF0FBE27
:10A03000CDBF8091090890910A08A0910B08B091BA
:10A040000C08E0919003F0919103838F948FA58F7A
:10A05000B68F2BE532E030939103209390038093E9
:10A06000E1079093E207A093E307B093E4074090E1
:10A0700064025090650260906602709067024092A0
:10A080003303509234036092350370923603A30178
:10A09000920160E070E080E89FE30F94D90960933B
:10A0A0004D0870934E0880934F0890935008C090CD
:10A0B0006A02D0906B02E0906C02F0906D02C09248
:10A0C0002303D0922403E0922503F09226036091AB
:10A0D0006E0270916F028091700290917102609394
:10A0E000F7027093F8028093F9029093FA0260935A
:10A0F0000703709308038093090390930A03A30155
:10A1000092010F947A0C0F94770A60933D08709334
:10A110003E0880933F089093400860932D08709309
:10A120002E0880932F08909330082091720230916E
:10A1300073024091740250917502C301B2010F94F1
:10A140007A0C9B01AC0160E074E284E798E40F9420
:10A15000D9090F94E00A0F94770A162F60935508D7
:10A16000A3019201C701B6010F947A0C9B01AC01C7
:10A1700060E074E284E798E40F94D9090F94E00A50
:10A180000F94770A603118F46093540803C08FE08D
:10A190008093540880915408811710F0109354084C
:10A1A0006091540870E080E090E00F94A30AA3014E
:10A1B00092010F947A0C9B01AC0160E074E284E799
:10A1C00098E40F94D9092B013C01A70196010F9443
:10A1D000D20987FF08C04092230350922403609263
:10A1E00025037092260386E892E03FDE2091F10776
:10A1F0003091F2074091F3075091F4072D833E838D
:10A200004F8358874090F5075090F6076090F70706
:10A210007090F8078091F9079091FA07A091FB07D9
:10A22000B091FC0789879A87AB87BC872091030789
:10A2300030910407409105075091060729833A831E
:10A240004B835C83E0909003F0909103F701818150
:10A250009281A381B4819C01AD0166277727CB0150
:10A26000621B730B840B950B0F94A50A2091410878
:10A270003091420840914308509144080F947A0C61
:10A280006093F7067093F8068093F9069093FA06A8
:10A29000F70185819681A781B0859C01AD01662774
:10A2A0007727CB01621B730B840B950B0F94A50AC8
:10A2B0002091450830914608409147085091480840
:10A2C0000F947A0C6093F3067093F4068093F5066E
:10A2D0009093F6068091FF06909100070E949D1FC3
:10A2E0008091C70780FF24C080910E038F938091D7
:10A2F0000D038F9380910C038F9380910B038F93A9
:10A3000030EFA32E33E2B32E34E7C32E39E4D32E3D
:10A31000E984FA840B851C85A30192016D817E81FD
:10A320008F8198850E94337E0F900F900F900F9031
:10A3300089819A81AB81BC81809303079093040744
:10A34000A0930507B093060780E00E94F0802C964A
:10A350000FB6F894DEBF0FBECDBFDF91CF911F9136
:10A360000F91FF90EF90DF90CF90BF90AF907F90D4
:10A370006F905F904F900C94F8DCE0910C02F0919C
:10A380000D0267817085818592850895E091900323
:10A39000F0919103858587FD06C061E09685911156
:10A3A00060E00D94560508958091680287FD07C00E
:10A3B00061E090916902911160E00D945605089555
:10A3C0002F923F924F925F926F927F928F929F92C5
:10A3D000AF92BF92CF92DF92EF92FF920F931F93B3
:10A3E000CF93DF9300D01F92CDB7DEB79C838B83D2
:10A3F000DC011196EC91E53338F4E23348F5EE23B5
:10A4000069F0ED3090F50DC0E43628F4E13648F4FB
:10A41000EC33F1F02AC0E436D9F027C049E150E02E
:10A4200026C0AB81BC8112968C91A82FB0E0AA0FF8
:10A43000BB1FA556BB4F4D915C918CEF9FE0841BD9
:10A44000950BAB81BC8114969C938E93139715C08A
:10A45000AB81BC8112968C91A82FB0E0AA0FBB1FD4
:10A46000A556BB4F4D915C9102C04FEF5FE0AB81B1
:10A47000BC8114965C934E931397AB81BC81139669
:10A480000D911C911497E53338F5E23308F0A0C024
:10A49000EE2309F450C0ED3008F081C1E1508E2F59
:10A4A00090E0FC01E45AF14F4491440FFC01EE0F9F
:10A4B000FF1FE859F14F85919491FC01859094908C
:10A4C000FC013296A590B4907CEF672E7FE0772E4A
:10A4D000601A710A52E03CC0E436C0F4E13608F07C
:10A4E000DBC0EC3309F05BC1B801882777FD8095AC
:10A4F000982F0F94A50A20E030E04AE754E40F9427
:10A500007A0C20E030E040E859E325C1E43609F058
:10A5100046C1B801882777FD8095982F0F94A50A2A
:10A5200020E030E04AEF53E40F947A0C20E030E072
:10A5300040E859E32CC180E090E0A8ECB1E4EB8165
:10A54000FC8187839087A187B28729C15101480187
:10A55000541708F011C1FC01E50FF11DE50FF11DC5
:10A5600005911491FC0161E0650FE60FF11D5E5F3E
:10A57000E60FF11D25903490601671063CF7B50189
:10A58000882777FD8095982F0F94A50A6B017C0191
:10A59000B30168197909882777FD8095982F0F9462
:10A5A000A50A2B013C01B1016A197B09882777FDB7
:10A5B0008095982F0F94A50A9B01AC01C301B201AD
:10A5C0000F947A0C2B013C01B80168197909ADC0D0
:10A5D000EE528E2F90E0FC01E45AF14F6491660F29
:10A5E000FC01EE0FFF1FE859F14F85919491FC019A
:10A5F00025903490FC0132968590949072E0761705
:10A6000008F044C0FC01E70FF11DE70FF11DA59014
:10A61000B490FC0121E0270FE20FF11D7E5FE20FF5
:10A62000F11D259134910A151B056CF5B40188279D
:10A6300077FD8095982F29833A830F94A50A6B01A3
:10A640007C01B80162197309882777FD8095982FDE
:10A650000F94A50A2B013C0129813A81B90168199F
:10A660007909882777FD8095982F0F94A50A9B017B
:10A67000AC01C301B2010F947A0C2B013C01B5016E
:10A680006219730952C049011501B9CFB901882770
:10A6900077FD8095982F75C0E23639F0A0901704A9
:10A6A000B0901804E7E1F4E006C0A0909303B090E6
:10A6B0009403E3E9F3E0828093804CEF642E4FE053
:10A6C000742E601A710A82E0048115818E5F2680E3
:10A6D0003780601671060CF049C0B401882777FDF9
:10A6E0008095982F0F94A50A6B017C01B3016A191C
:10A6F0007B09882777FD8095982F0F94A50A2B0159
:10A700003C01B10168197909882777FD8095982F58
:10A710000F94A50A9B01AC01C301B2010F947A0CFE
:10A720002B013C01B8016A197B09882777FD8095C8
:10A73000982F0F94A50A9B01AC01C301B2010F949D
:10A74000D9099B01AC01C701B6010F946E0920E045
:10A7500030E040E05EE30F947A0CAB81BC81179649
:10A760006D937D938D939C931A9719C03496823480
:10A7700019F041015801A8CFB101882777FD8095D4
:10A78000982F0F94A50A20E030E040E05EE30F949C
:10A790007A0CEB81FC8167837087818792870F90A9
:10A7A0000F900F900F90DF91CF911F910F91FF901D
:10A7B000EF90DF90CF90BF90AF909F908F907F9061
:10A7C0006F905F904F903F902F9008958F929F923F
:10A7D000AF92BF92CF92DF92EF92FF920F931F93AF
:10A7E000CF93DF93EC01CB01BA016B877C878D8718
:10A7F0009E87FE01E05CFF4F2081297F208320E0BF
:10A8000030E040E051E40F947A0C0F94720A4B014F
:10A810002981253318F5223308F08AC0222309F450
:10A8200048C02D3008F019C1215030E0F901E45A38
:10A83000F14FB490BB0CF901EE0FFF1FE859F14F37
:10A8400025913491F901E590F490F9013296459102
:10A850005491C12CD12CB2E0AB2E30C02436B0F4D0
:10A86000213608F0B4C02C3309F0F7C0882777FDF3
:10A870008095982F2CE0660F771F881F991F2A95C7
:10A88000D1F728EE33E040E050E09CC0243609F0D8
:10A89000E4C0882777FD8095982F0CE0660F771F1E
:10A8A000881F991F0A95D1F724EF31E040E050E06E
:10A8B00089C01E821D82D1C0A8017D01AB1498F50C
:10A8C000F901EA0DF11DEA0DF11DA591B4916D019B
:10A8D000F90111E01A0DE10FF11DA394A394E10F0A
:10A8E000F11D059114910815190534F79A01261BDD
:10A8F000370BC7018A1B9B0BDC016CEFC62E6FE088
:10A90000D62ECE18DF080F94C80D9A01201B310BEC
:10A91000442737FD4095542F0F94A60DC20ED31E29
:10A92000DE82CD829AC08CEF9FE08C199D0993C086
:10A930002E5230E0F901E45AF14FA491AA0FF90127
:10A94000EE0FFF1FE859F14F25913491F901059160
:10A950001491F901329645915491C12CD12CB2E059
:10A96000BA1768F5F901EB0FF11DEB0FF11DA5907A
:10A97000B4906501F901FF24F394FB0EEF0DF11D76
:10A98000BE5FEF0DF11DE590F4908E149F04A4F4CA
:10A990009A01261B370BD801AA19BB090F94C80DC1
:10A9A0009A012E193F09442737FD4095542F0F94E3
:10A9B000A60D200F311F08C0A7018501D1CFCD8280
:10A9C000DE824BC00F94A60D3E832D8346C02236F7
:10A9D00039F0E0901704F0901804A7E1B4E006C045
:10A9E000E0909303F0909403A3E9B3E012964D91A5
:10A9F0005C91139722E014960D911C9115972E5F90
:10AA00001696ED91FC911797E815F905D4F49A0183
:10AA1000261B370BD701A01BB10B0CEF1FE00E1943
:10AA20001F090F94C80D9A012E1B3F0B442737FDB9
:10AA30004095542F0F94A60D020F131F1E830D83F4
:10AA40000CC01496223419F0AF017801D4CF8CEFEA
:10AA50009FE0801B910B9E838D83DF91CF911F918F
:10AA60000F91FF90EF90DF90CF90BF90AF909F90AD
:10AA70008F9008959F92AF92BF92CF92DF92EF9204
:10AA8000FF920F931F93CF93DF936B017C01042FF1
:10AA9000922EE0910A02F0910B02C1E020E030E03A
:10AAA00040E751E463857485858596850F94060C8F
:10AAB00018160CF0C0E011E01C2720E030E041E95E
:10AAC00053E4C701B6010F94060C18166CF020E091
:10AAD00030E0A901C701B6010F94D20987FF0AC06F
:10AAE000C12CD12C760106C0C12CD12C91E9E92EC4
:10AAF00093E4F92EC02FD0E0FE01EE0FFF1FE65FBA
:10AB0000FD4FA080B180F5018181811103C0C12C6E
:10AB1000D12C7601B701A601C50158DE992081F03C
:10AB200020E030E040EF51E4C701B6010F94060C7D
:10AB3000181634F4F501E05CFF4F8081816080835A
:10AB400020E030E040E252E4C701B6010F94060C69
:10AB500087FD0EC023E82C9FC0012D9F900D11246E
:10AB6000855A9D4FFC01E458FF4F20813196208388
:10AB7000602F70E080E090E00F94A30AAB01BC016D
:10AB800020E084E292E20E94D8A120E0B701A60171
:10AB900088E294E20E949BA1E0910A02F0910B02EC
:10ABA00020E030E040E751E4638574858585968533
:10ABB0000F94060C18167CF0111119C0DF91CF917B
:10ABC0001F910F91FF90EF90DF90CF90BF90AF90CB
:10ABD0009F900C9479D6112351F00F94090460933F
:10ABE000ED067093EE068093EF069093F006DF91EA
:10ABF000CF911F910F91FF90EF90DF90CF90BF907A
:10AC0000AF909F900895CF92DF92EF92FF92CF93F3
:10AC10006B017C01C42F20E030E040EF52E40F9440
:10AC2000060C18166CF020E030E0A901C701B6014F
:10AC30000F94D20987FF0AC0C12CD12C760106C01F
:10AC4000C12CD12C20EFE22E22E4F22EA701960196
:10AC50006091190270911A0280911B0290911C025E
:10AC60000F94D209882341F1B701A6018EE092E04A
:10AC7000ADDDCC2379F020E030E040EF51E4C701B6
:10AC8000B6010F94060C18162CF480914E028160C8
:10AC900080934E024091190250911A0260911B025A
:10ACA00070911C0220E089E192E2CF91FF90EF9039
:10ACB000DF90CF900C949BA1CF91FF90EF90DF900D
:10ACC000CF900895E0910A02F0910B02168215824E
:10ACD0001386148615861686E081F0E0EE57F24E54
:10ACE0001082E0910C02F0910D02168215821386FB
:10ACF000148615861686E081F0E0EE57F24E10823B
:10AD00008FEF8093DE0208952F923F924F925F92D1
:10AD10006F927F928F929F92AF92BF92CF92DF926B
:10AD2000EF92FF920F931F93CF93DF93CDB7DEB7D0
:10AD3000E5970FB6F894DEBF0FBECDBF9DAB8CABD1
:10AD40004E8B5F8B688F798F2E8F0BAB0F9409041E
:10AD50006A8F7B8F8C8F9D8FACA9BDA996968C91A5
:10AD600090E0959587952C01662457FC6094762C8D
:10AD700086E092E20E94B39FA5DFBE8DB093DE0213
:10AD8000ACA9BDA9EC91F0E0EE57F24E96968C91ED
:10AD90008083BE8DB11104C08091D7028093D80208
:10ADA000530142012A8D3B8D4C8D5D8D2BA33CA31D
:10ADB0004DA35EA32F8F38A349A35AA319821F86E0
:10ADC00030EA388B41E4498B1A8A1B8A50EA5C8B43
:10ADD00081E48D8B1BA61CA61DA61EA61FA218A66D
:10ADE00019A61AA6C12CD12C76011FA618AA19AA39
:10ADF0001AAA91E099871E861D86A8958CA99DA9FF
:10AE0000DFDAACA9BDA917963C90179718960C915C
:10AE1000189719961C9119971A962C900F9409045B
:10AE20006D837E838F839887232D302F412F522D62
:10AE30006A897B898C899D890F94D20987FF04C018
:10AE40003A8A0B8B1C8B2D8A232D302F412F522DAC
:10AE500069817F85888999890F94D20987FD04C00B
:10AE600039820F87188B298AB985BB2309F449C019
:10AE70002E893F89488D598D632D702F812F922DFA
:10AE80000F94060C18160CF086C08D819E81AF8140
:10AE9000B8852BA13CA14DA15EA1821B930BA40BF5
:10AEA000B50B3E8D311105C044EC59E060E070E017
:10AEB00004C04CED55E060E070E0481759076A07A0
:10AEC0007B0708F068C0ECA9FDA92081E22FF0E023
:10AED000EE57F24E242D281920838FA798ABA9ABEB
:10AEE000BAABFE89FA8B2F892B8B388D3C8B498D21
:10AEF0004D8B8D819E81AF81B8858F8F98A3A9A33B
:10AF0000BAA32E893F89488D598D632D702F812FCB
:10AF1000922D0F94D20987FF11C28D819E81AF813E
:10AF2000B8852F8D38A149A15AA1821B930BA40B80
:10AF3000B50B3E8D3111EFC048E853E160E070E0A1
:10AF4000481759076A077B0708F0F8C14D855E85E9
:10AF5000452B09F0E5C0ACA9BDA9EC91F0E0EE5796
:10AF6000F24E882D840D8083ED85FE853196FE8717
:10AF7000ED87FE89F9832F892F87388D388B498D8E
:10AF8000498B8D819E81AF81B8858BA39CA3ADA396
:10AF9000BEA391E0998720E030E040E252E46E8960
:10AFA0007F89888D998D0F946E099B01AC01632D6B
:10AFB000702F812F922D0F94060C18161CF487E920
:10AFC00091E23BC08D819E81AF81B8852A8D3B8DFA
:10AFD0004C8D5D8D821B930BA40BB50B893E93406A
:10AFE000A105B10558F080E00E9426248D819E8144
:10AFF000AF81B8858A8F9B8FAC8FBD8F8D819E81ED
:10B00000AF81B885880F991FAA1FBB1F2BA13CA138
:10B010004DA15EA1821B930BA40BB50B2F8D38A104
:10B0200049A15AA1821B930BA40BB50B81389F44F5
:10B03000A241B105E8F08AE791E20E94BD9FE59642
:10B040000FB6F894DEBF0FBECDBFDF91CF911F9139
:10B050000F91FF90EF90DF90CF90BF90AF909F90B7
:10B060008F907F906F905F904F903F902F902ACE5F
:10B070004D855E85463051050CF443C08FE191E269
:10B080000E94B39F1FDE5BA9552309F459C1ACA9E7
:10B09000BDA95A96CD92DD92ED92FC925D972FA1BB
:10B0A00038A549A55AA55E962D933D934D935C9383
:10B0B00091972BA53CA54DA55EA592962D933D930A
:10B0C0004D935C93959781E053968C9380E0E59641
:10B0D0000FB6F894DEBF0FBECDBFDF91CF911F91A9
:10B0E0000F91FF90EF90DF90CF90BF90AF909F9027
:10B0F0008F907F906F905F904F903F902F900C9427
:10B100005BCF86E79AE00E9478CA61E086E79AE022
:10B110000E9479CA72CE48EB5BE060E070E010CF2D
:10B120002FA538A949A95AA9280F391F4A1F5B1F03
:10B1300029873A874B875C872FA538A949A95AA93F
:10B14000281B390B4A0B5B0BCA01B901A5019401FD
:10B150000F94410D29853A854B855C850F94A60D8A
:10B16000240D351D461D571D24313105410551055E
:10B17000A4F0ACA9BDA996968C9190E04497AA271B
:10B1800097FDA095BA2F29013A0182179307A407CA
:10B19000B50744F42C013D0105C044E1442E512C77
:10B1A000612C712CECA9FDA926A1822F869590E037
:10B1B000A0E0B0E084159505A605B7056CF4822FD4
:10B1C00090E001974C01AA2497FCA094BA2C841813
:10B1D0009508A608B70802C053014201B301A201B5
:10B1E0008EEF91E20E94A7A0B501A40189EF91E240
:10B1F0000E94A7A022E049815F856889798982EF52
:10B2000091E20E94D8A122E04A895B896C897D89FC
:10B210008BEE91E20E949BA12D853E852330310566
:10B220000CF499CEC501B4010F94A50A20E030E0DA
:10B2300040E850E40F947A0C6B017C0129813F8532
:10B24000488959896A897B898C899D890F946D0900
:10B2500020ED3FE049E450E40F947A0C9B01AC01EF
:10B26000C701B6010F94D9096B017C0169857A8504
:10B270008B859C850F94A50A20E030E04AE754E4D2
:10B280000F94D90969837A838B839C8322E0B70169
:10B29000A60185EE91E20E94D8A122E049815A815F
:10B2A0006B817C818FED91E20E949BA12AE939E9B3
:10B2B00049E15FE3C701B6010F947A0C6B017C0191
:10B2C0009B01AC010F946E0929813A814B815C810D
:10B2D0000F94D9096FA378A789A79AA729813A81E2
:10B2E0004B815C81C701B6010F947A0C20E030E0FD
:10B2F00040E05EE30F947A0C6BA77CA78DA79EA716
:10B3000082ED91E20E949C9F22E0B701A6018CECA5
:10B3100091E20E949BA122E04FA158A569A57AA5C0
:10B3200086EC91E20E949BA122E04BA55CA56DA555
:10B330007EA580EC91E20E949BA10DCE19862BCEBA
:10B34000E5960FB6F894DEBF0FBECDBFDF91CF916B
:10B350001F910F91FF90EF90DF90CF90BF90AF9033
:10B360009F908F907F906F905F904F903F902F9025
:10B370000895CF93DF930F940904AB01BC0188E1DA
:10B3800091E20E94A7A0E091E002F0E0EE0FFF1F23
:10B39000E65FFD4FC081D1814F81588569857A85EF
:10B3A00022E085EB93E20E94D8A14B855C856D85F8
:10B3B0007E8520E085EB93E20E94D8A1E881F0E051
:10B3C000EE57F24E608170E085EB93E2DF91CF9112
:10B3D0000C9481A08091C80782FF3CC060E070E0BF
:10B3E00083E091E20E9475A0E0910A02F0910B02C5
:10B3F00067817085818592850F94720A6051710909
:10B400006D31714018F484EE90E202C08EEE90E24D
:10B410000E949C9F8DE091E20E94839FE0910C022C
:10B42000F0910D0267817085818592850F94720A73
:10B43000605171096D31714018F08EEE90E202C0DA
:10B4400084EE90E20E949C9F87EB90E20E94BD9F59
:10B4500081E0089580E008952F923F924F925F928D
:10B460006F927F928F929F92AF92BF92CF92DF9214
:10B47000EF92FF920F931F93CF93DF93CDB7DEB779
:10B480002B970FB6F894DEBF0FBECDBFA8950F94D3
:10B49000090469837A838B839C832AE032E03B87AB
:10B4A0002A8748ED52E05F834E8352E35987212C6F
:10B4B0001D82AA85BB850D911D91BB87AA8721108E
:10B4C00027C020E030E040E252E4F8016781708557
:10B4D000818592850F94D20987FF13C020E030E068
:10B4E00040E252E4D8011B966D917D918D919C9123
:10B4F0001E970F94D20987FF04C0EE81FF8110824E
:10B5000007C0EE81FF8131978081AE81BF818C932E
:10B510008091DE02281609F4B8C2C8010E94E051E9
:10B520008091C80782FD26C0F801C780D084E184DD
:10B53000F28420E030E040E851E4C701B6010F9406
:10B54000D20987FD0AC020E030E046E953E4C70194
:10B55000B6010F94060C18166CF4809192038F5F5D
:10B56000809392038B3008F4C3C20E94F14D32DF06
:10B57000F1E0FD838091C80782FD87C233243394B4
:10B58000D8011B962D913D914D915C911E97179678
:10B590006D917D918D919C911A970F94060C87FD6A
:10B5A000312CB1E03B2641F47801E0E4EE0EF11CD1
:10B5B000D7018C9180FD9FC2C980DA80EB80FC802E
:10B5C000F801E75BFF4F4080518062807380580133
:10B5D000B1E4AB0EB11CF50180819181A281B381F0
:10B5E000A7019601281B390B4A0B5B0B4216530629
:10B5F0006406750608F068C0480130E4830E911CAB
:10B60000D401BC91B8878B2F867009F45DC08091FE
:10B61000C70786FF59C0B885B1FF81C27801E5E44C
:10B62000EE0EF11CD7012D913D914D915C91F801E9
:10B6300067817085818592850F946D0920E030E0E7
:10B6400040E85FE30F94D20987FF5EC280919203C6
:10B650008F5F809392038B30A8F10E94F14D41E0FF
:10B6600069E978E186E79AE00E94A6AB82E598E175
:10B670000E94BD9FD7012D913D914D915C91F801A4
:10B6800067817085818592850F946D09AB01BC013E
:10B6900022E08CEE9DE00E94D8A149815A816B8105
:10B6A0007C81F50180819181A281B381481B590B76
:10B6B0006A0B7B0B84EE9DE00E94A7A080EE9DE0CC
:10B6C0000E949C9FF1E0FD83F80187A5C780D0848C
:10B6D000E184F28424E0829FE00DF11D1124C0AAD0
:10B6E000D1AAE2AAF3AA8F5F8370D8019F968C93A8
:10B6F0009F9753968C915397813009F0CAC01B963F
:10B700008D909D90AD90BC901E9720E030E040EA77
:10B7100051E4C501B4010F94D20987FDCCC0A70143
:10B720009601C501B4010F946D094B015C0120E045
:10B7300030E040EA51E40F94060C18161CF4F801AE
:10B74000F6A0D3C020E030E040EA51ECC501B401DE
:10B750000F94D20987FDDAC0BE016F5F7F4FC80129
:10B760000E949F4DD8015A962D913D914D915C912B
:10B770005D97C501B4010F947A0C6B017C01F8014F
:10B780002489358946895789C501B4010F946E090A
:10B790004B015C01D8019B965C909B979C966C90AA
:10B7A0009C979D967C909D979E964C90252D362D2E
:10B7B000472D542D0F94D20987FD13C0F80157A0CF
:10B7C00060A471A442A4252D362D472D542DB4011B
:10B7D000C5010F94060C181624F0582C692C7A2CED
:10B7E0004B2C852D962DA72DB42DF801848B958B90
:10B7F000A68BB78B268D378D40A151A1652D762D57
:10B80000872D942D0F947A0C2DEC3CEC4CEC5DE3E1
:10B810000F947A0C9B01AC01C701B6010F946E091D
:10B820006B017C01D8019F968C91F801B4E08B9F4D
:10B83000E00DF11D1124D80117962D913D914D91E8
:10B840005C911A9760A971A982A993A90F946D09B7
:10B85000F80122A133A144A155A10F947A0C2FED38
:10B860003FE445E550E40F947A0C9B01AC01C7011D
:10B87000B6010F946E090F94720A77FD47C0D80184
:10B8800096962C9130E0261737070CF4B901F62E66
:10B8900098C0833009F09CC0F80183849484A58407
:10B8A000B68420E030E040EA51E4C501B4010F94D1
:10B8B000D20987FF07C0F801E05CFF4F8081897FD4
:10B8C000808324C0A7019601C501B4010F946D09BE
:10B8D0006B017C0120E030E040EA51E40F94060C5B
:10B8E000181654F4D8019696FC90BE016F5F7F4FF6
:10B8F000C8010E94754D65C020E030E040EA51EC7F
:10B90000C701B6010F94D20987FF02C0F12C59C0BC
:10B91000BE016F5F7F4FC8010E949F4DF801C78035
:10B92000D084E184F28420E030E040E450E4648993
:10B930007589868997890F947A0C4B015C01D8012F
:10B940009F968C91F801B4E08B9FE00DF11D1124BE
:10B9500020A931A942A953A9C701B6010F946D09C5
:10B960002FED3FE445E550E40F947A0C9B01AC01C8
:10B97000C501B4010F946E0920E030E040E85EE3B9
:10B980000F947A0CF801648B758B868B978B228DC4
:10B99000338D448D558D0F947A0C9B01AC01C701FA
:10B9A000B6010F946E09D8011B962D913D914D91D2
:10B9B0005C911E970F94060C18160CF4A7CFF80193
:10B9C000F08CD801EC91F0E0EE57F24EF0823DC0E1
:10B9D000823021F589819A81AB81BC81F80147854C
:10B9E0005089618972896C017D01C41AD50AE60A01
:10B9F000F70A29E8C21623E1D206E104F10428F18E
:10BA00002081E22FF0E0EE57F24E232D2195208386
:10BA1000F8018787908BA18BB28B08C0D801EC917D
:10BA2000F0E0EE57F24E832D81958083332039F07C
:10BA3000BE016F5F7F4FC8010E94754D06C0F801BF
:10BA4000E05CFF4F8081897F808320E030E041E926
:10BA500053E4F80167817085818592850F94060C07
:10BA6000181634F4D801EC91F0E0EE57F24E108243
:10BA700080919003909191038B960817190729F4F0
:10BA8000332011F02F9A01C02F982394B985BE5C02
:10BA9000B987EE81FF81ED57FF4FFF83EE83F2E020
:10BAA0002F1207CDCD80C11007C08091920388234B
:10BAB00019F08150809392038091C80782FF88C05B
:10BAC000E0910A02F0910B02E081F0E0EE57F24EB5
:10BAD0001082E0910C02F0910D02E081F0E0EE574F
:10BAE000F24E10828091EA0288608093EA0270C070
:10BAF00021E02D833FCD63E089850E94A4A2D70178
:10BB00008C918E7F8C9358CD8885897FD4018C93BE
:10BB1000BE016F5F7F4FC8010E94754DD5CDF80102
:10BB20002385348545855685678170858185928515
:10BB30000F946D099F7720E030E040EA51E40F94C4
:10BB4000060C1816A4F5809192038F5F80939203E0
:10BB50008B3008F4B7CD0E94F14D41E069E978E1FE
:10BB600086E79AE00E94A6AB82E598E10E94BD9F1D
:10BB7000F801EB5BFF4F408151816281738122E0CC
:10BB80008EEB9DE00E94D8A1D80117964D915D9152
:10BB90006D917C911A9722E083EB9DE00E94D8A1E1
:10BBA0008BEA9DE00E949C9FB1E0BD838DCDE8EEC5
:10BBB000CE0EE3E0DE1EE11CF11CC418D508E60839
:10BBC000F708D501CD92DD92ED92FC9213977CCDD2
:10BBD0002B960FB6F894DEBF0FBECDBFDF91CF918D
:10BBE0001F910F91FF90EF90DF90CF90BF90AF909B
:10BBF0009F908F907F906F905F904F903F902F908D
:10BC000008958FEF8EBD0DB407FEFDCF8EB508955C
:10BC1000DC01680F791F80E090E0A617B70779F084
:10BC20002D91E92FFF27E227EE0FFF1FEE51FD4E6A
:10BC300025913491982F882782279327EECF089556
:10BC40008EBD0DB407FEFDCF0895CF93FB0120E01C
:10BC500030E22F5F31932B30E1F7DC0190E037E0E9
:10BC60002A2FEB2F8D9181110AC0DA012C931196A6
:10BC7000EC9381E0FB019081903241F526C08F3238
:10BC8000A1F3282F8E3219F0E2EEF4E108C03A3029
:10BC9000E1F098E03AE0E4CF3196C817B1F0C491F2
:10BCA000C111FACF391718F080528F3508F02FE5FF
:10BCB00081E0890FFB01E90FF11D9FE9920F9A3195
:10BCC00008F420522083982FCBCF80E0CF910895A5
:10BCD0009B01255F3F4F80E0FB019191BF01482F01
:10BCE0004695F0E88F9F400D1124842F890F62172D
:10BCF000730791F7089561E0FC0180810F94560568
:10BD00008FEF9ECFCF93DF93EC018A810E94451D78
:10BD100060E08881DF91CF910D945605CF92DF923C
:10BD2000EF92FF920F931F93CF93DF93EC018B0160
:10BD30007A010F9409046B0164DF8B838F3F49F410
:10BD40000F9409046C197D096D327140A8F381E1EB
:10BD500031C08E3F11F08FE02DC0E114F104D9F015
:10BD6000C70101972FEF2EBDF8014FEF9F01201B58
:10BD7000310B2817390738F40DB407FEFDCF2EB567
:10BD800021934EBDF3CF0DB407FEFDCF2EB5F801C4
:10BD9000E80FF91F20831B8234DFD82E32DFC82E34
:10BDA000B701C80135DF2C2D30E03D2928173907B0
:10BDB00031F08BE18983CE019EDF80E003C0CE01AC
:10BDC0009ADF81E0DF91CF911F910F91FF90EF906B
:10BDD000DF90CF9008950F931F93CF93DF931F921F
:10BDE0001F92CDB7DEB78C0169837A838BDF40E089
:10BDF00052E069817A81C8010F900F90DF91CF9155
:10BE00001F910F918BCF0F931F93CF93DF93EB0174
:10BE10000F9409048B01F5DE8F3F49F00F9409045C
:10BE2000601B710B6C177D07B0F380E001C081E0EF
:10BE3000DF91CF911F910F910895BF92CF92DF9222
:10BE4000EF92FF920F931F93CF93DF93CDB7DEB79F
:10BE50002A970FB6F894DEBF0FBECDBF8C01B62E69
:10BE60002F83388749875A874DDF6CE271E0C8011C
:10BE7000CADFFE01319686E0DF011D928A95E9F75F
:10BE80008B2D806489838A858A8389858B838885C5
:10BE90008C838F818D83CE010696DF0120E059E0EF
:10BEA0004D9138E0220F642F622767FD2527440F4C
:10BEB0003150C1F7A817B90799F7220F21602E83D7
:10BEC0007F016E01B7E0CB0ED11CF70181917F019C
:10BED000B7DEEC14FD04C9F7FCE0BF1201C091DE2F
:10BEE000F12C8FDED80113968C9387FF05C0BFEF2E
:10BEF000FB1611F0F394F5CF2A960FB6F894DEBF37
:10BF00000FBECDBFDF91CF911F910F91FF90EF90AA
:10BF1000DF90CF90BF900895BF92CF92DF92EF92C3
:10BF2000FF920F931F93CF93DF93EC01B62E1C82E9
:10BF3000198248830F9409048B0161E088810F9472
:10BF40001D0561E088810F9456052398229A219A55
:10BF5000209A8BE08A830E94451DE4E1FE2E8FEF3C
:10BF60006FDEFA94E1F720E030E0A90160E0CE0155
:10BF700064DF813049F00F940904601B710B613D4F
:10BF8000774088F381E057C021E030E040E050E0A6
:10BF90006BE3CE0152DF813011F08AE14CC02AEA16
:10BFA00031E040E050E068E0CE0147DF853011F439
:10BFB00081E009C074E0F72E24DE8B83FA94E1F768
:10BFC0008A3A59F482E08C838C81823079F4C12CD6
:10BFD000D12CE12C60E4F62E0CC00F940904601BF8
:10BFE000710B613D7740D8F282E025C0C12CD12C85
:10BFF000760120E030E0A90167E3CE011EDFA70152
:10C00000960169E2CE0119DF882349F00F940904F3
:10C01000601B710B613D774060F38AE00CC08C813E
:10C020008230B1F420E030E0A9016AE3CE0105DFFF
:10C03000882329F088E08983CE015DDE14C0E1DD2C
:10C04000807C803C11F483E08C83DBDDDADDD9DD9C
:10C05000CE0151DE8EE08B1518F488E1898303C090
:10C06000BA8281E001C080E0DF91CF911F910F91F2
:10C07000FF90EF90DF90CF90BF9008950F931F93A4
:10C08000CF93DF93EC0189018C81833039F0F9E0A3
:10C09000440F551F661F771FFA95D1F79A01AB0120
:10C0A00061E1CE01CADE811109C040E052E0B80171
:10C0B000CE01DF91CF911F910F9130CE84E0898323
:10C0C000CE0119DE80E0DF91CF911F910F9108958D
:10C0D000CF93DF93EC018C81833039F089E0440FFA
:10C0E000551F661F771F8A95D1F79A01AB0162E150
:10C0F000CE01A3DE882331F085E08983CE01FBDD0C
:10C1000080E003C0CE01F7DD81E0DF91CF9108959B
:10C11000CF93DF93EC01F6DD20E030E0A9016CE085
:10C12000CE018BDE882331F083E08983CE01E3DD0D
:10C1300080E003C0CE01DFDD81E0DF91CF91089583
:10C14000CF92DF92EF92FF920F931F93CF93DF93E3
:10C150001F92CDB7DEB78C01E62E6A0160E072E077
:10C16000CA0156DDF82E8E2D99836ADDF601808195
:10C170008EBD418122E030E099810DB407FEFDCFF4
:10C180004EBD2115F2E03F0739F0F601E20FF31F33
:10C1900040812F5F3F4FF1CF0DB407FEFDCF892FB8
:10C1A0004FDD8F2D4DDD2DDDF80183838F718530BF
:10C1B00031F083E18183C8019EDD80E001C081E030
:10C1C0000F90DF91CF911F910F91FF90EF90DF9033
:10C1D000CF9008950F931F93CF93DF93EC018901C4
:10C1E0008C81833039F039E0440F551F661F771F6B
:10C1F0003A95D1F79A01AB0168E1CE011EDE8823A2
:10C2000011F086E01EC0A8016EEFCE0199DF8823F1
:10C21000C9F068E572E0CE01F6DD182F811102C089
:10C2200087E10FC020E030E0A9016DE0CE0105DE1E
:10C23000811106C0E6DC811103C0CE015CDD05C0C2
:10C2400086E18983CE0157DD10E0812FDF91CF9108
:10C250001F910F9108950F931F93CF93DF93EC01DC
:10C260008B0150DD68E572E0CE01CDDD882351F011
:10C27000A8016CEFCE0164DF182F882319F0CE01DE
:10C280003ADD05C085E18983CE0135DD10E0812FDF
:10C29000DF91CF911F910F9108958F929F92AF924E
:10C2A000BF92CF92DF92EF92FF920F931F93CF93A3
:10C2B000DF93EC016A017B014801590120E030E085
:10C2C000A90167E3BADDA501940167E1CE01B5DDFF
:10C2D000882311F089E012C08C81833039F049E065
:10C2E000CC0CDD1CEE1CFF1C4A95D1F7A701960172
:10C2F00069E1CE01A2DD882331F087E08983CE0198
:10C30000FADC80E003C0CE01F6DC81E0DF91CF9162
:10C310001F910F91FF90EF90DF90CF90BF90AF9063
:10C320009F908F9008951F93CF93DF93EC01EADCE9
:10C3300068E572E0CE0167DD882361F08DEF80DC77
:10C3400068E572E0CE015FDD182F882319F0CE0179
:10C35000D2DC05C082E18983CE01CDDC10E0812FE3
:10C36000DF91CF911F9108950F931F93CF938091E9
:10C37000AF0480FF41C04091B0045091B10460917E
:10C38000B2047091B30424EB34E08091A90490913D
:10C39000AA0420DFC82F811102C0C0E02EC0809106
:10C3A000AF0481FD06C08091AF048E7F8093AF04FF
:10C3B00024C00091AB041091AC042091AD043091E5
:10C3C000AE04011511052105310569F34091B00452
:10C3D0005091B1046091B2047091B304400F511FA9
:10C3E000621F731F24EB34E08091A9049091AA048A
:10C3F000F1DE8111D8CFD1CFC1E08C2FCF911F9129
:10C400000F910895CF92DF92EF92FF92CF936B013D
:10C410007C01C42F8091B0049091B104A091B2042A
:10C42000B091B3048C159D05AE05BF05F9F09CDFF6
:10C43000811103C080E090E021C0C2FF0BC01092C8
:10C44000AF04C092B004D092B104E092B204F09272
:10C45000B3040CC024EB34E0B701A6018091A90419
:10C460009091AA040BDE8111EACFE4CFC3708091D2
:10C47000AF048C2B8093AF0484EB94E0CF91FF90BA
:10C48000EF90DF90CF900895CF93DF93EC01462F8C
:10C490006F85788989899A89B5DF009739F02C8171
:10C4A00030E2239F800D911D112402C080E090E0B6
:10C4B000DF91CF9108950F931F93CF93DF93EC01FA
:10C4C0008B818823D1F1898187FF32C061E0CE0161
:10C4D000DBDF8C01009789F1FC018081853E69F1E9
:10C4E0008B81823040F44B895C896D897E89448FD1
:10C4F000558F668F778F4F89588D698D7A8DF801AA
:10C50000538F428F758B648BE091B406F091B50622
:10C51000309759F0B8016A5E7F4FC8014896199567
:10C52000F801808D918D938B828B89818F778983A0
:10C53000DF91CF911F910F9117CF81E0888380E029
:10C54000DF91CF911F910F910895CF93DF93EC016D
:10C55000B2DF1B82DF91CF9108958FEF9FEFDC0157
:10C560008093B0049093B104A093B204B093B30449
:10C570001092AF0408958F929F92AF92BF92CF9284
:10C58000DF92EF92FF920F931F93CF93DF93EC0113
:10C590006A017B018901423051056105710508F48A
:10C5A00054C089859A85AB85BC850196A11DB11DB6
:10C5B00084179507A607B70708F447C08F8980310D
:10C5C00029F49927872F762F652F0BC08032E9F544
:10C5D000CB01BA0127E096958795779567952A95BF
:10C5E000D1F78B889C88AD88BE88680D791D8A1D1F
:10C5F0009B1D42E007DF009741F12F89203169F44C
:10C60000DD24EE24FF24F601EE0FFF1FE80FF91FD3
:10C6100080819181A0E0B0E011C0E894C7F8DD24EA
:10C62000EE24FF24F601EE0FFF1FEE0FFF1FE80FB1
:10C63000F91F80819181A281B381BF70F80180834D
:10C640009183A283B38381E001C080E0DF91CF9129
:10C650001F910F91FF90EF90DF90CF90BF90AF9020
:10C660009F908F9008952F923F924F925F927F926A
:10C670008F929F92AF92BF92CF92DF92EF92FF92F2
:10C680000F931F93CF93DF93EC017B016A018B81A2
:10C69000811103C08FEF9FEF17C1898180FFFACF0F
:10C6A0004B895C896D897E898B859C85AD85BE852E
:10C6B0004601A12CB12C8A019B01081B190B2A0BE6
:10C6C0003B0B80169106A206B30618F06A01C81A41
:10C6D000D90A86014E0127E0820E911C0115110531
:10C6E00009F46EC02B843C844D845E84510181E04A
:10C6F000B8228D819E81B201A101E9E0769567950E
:10C7000057954795EA95D1F7FC0174807A94742285
:10C710002B81223049F4228C338C448C558C240E8E
:10C72000351E461E571E37C0A114B104C1F4711046
:10C7300016C023282428252849F48F89988DA98D8F
:10C74000BA8D8F839887A987BA8709C04F8158858A
:10C7500069857A8594010FDF882309F49BCFED81E9
:10C76000FE81A4812F81388549855A85225031095F
:10C7700041095109B0E00F94E30D1B012C0186859E
:10C780009785A089B189280E391E4A1E5B1E270C89
:10C79000311C411C511CA114B104A1F40115F2E09B
:10C7A0001F0780F08091B0049091B104A091B20471
:10C7B000B091B304281639064A065B06D9F402C0C4
:10C7C000C60182C040E0C201B1011CDE009709F43D
:10C7D00061CF20E032E02A193B09280120173107F8
:10C7E00008F42901BC016A0D7B1DA201C7010F9449
:10C7F000EB112AC00115E4E01E07B8F1B12EB69482
:10C800002B81223009F040C0281639064A065B0603
:10C8100008F043C0B201A1018091A9049091AA043B
:10C8200057DC882309F436CF1701412C8091A904E5
:10C830009091AA044B103BC06BDC882309F42ACFEB
:10C84000512C542C4424550CE40CF51C8B859C85F0
:10C85000AD85BE85840D951DA11DB11D8B879C875F
:10C86000AD87BE870419150939CF9701B201A1011F
:10C870008091A9049091AA0401DC882309F40ACFCD
:10C88000412C42E0542EE0CFED81FE812481271916
:10C890002B1508F0B9CFB22EB7CF8B0D911DA11D6E
:10C8A000B11D281639064A065B0650F0B3CFB10118
:10C8B00092DA2EEF321A882309F4ECCE4394B6CFE5
:10C8C00053DD8111A7CFE6CEDF91CF911F910F915C
:10C8D000FF90EF90DF90CF90BF90AF909F908F90A0
:10C8E0007F905F904F903F902F900895CF93DF936C
:10C8F0001F92CDB7DEB741E050E0BE016F5F7F4FC2
:10C90000B2DE019719F4898190E002C08FEF9FEFAA
:10C910000F90DF91CF9108951F93CF93DF93EC0198
:10C920008B81823018F480E090E023C04B855C85D9
:10C930006D857E85A5E07695679557954795AA956F
:10C94000D1F7142F1F70CE01D1DF97FDECCF4B85AF
:10C950005C856D857E85415E5F4F6F4F7F4F4B8756
:10C960005C876D877E8720E2129FC00111248C5462
:10C970009B4FDF91CF911F910895AF92BF92CF92BD
:10C98000DF92EF92FF920F931F93CF93DF931F924B
:10C99000CDB7DEB77C018A014115510511F0DA01EE
:10C9A0001C9241E0BDE0CB2EA895C7014983B4DFBE
:10C9B0005C014981009709F47AC0FC01208122239F
:10C9C00009F475C0253009F467C0253E09F464C038
:10C9D000FC018385982F9F739F3009F054C0011587
:10C9E000110511F3828D938D892BF1F62F71E1F2F0
:10C9F0002330D4F6332727FD309521503109C29ECC
:10CA0000F001C39EF00D1124E00FF11FD501119626
:10CA10008C911197808313968C911397818315962F
:10CA20008C911597828317968C911797838319960B
:10CA30008C91199784831E968C911E9785835096AE
:10CA40008C915097868352968C91529787835496F7
:10CA50008C915497808756968C91569781875896DB
:10CA60008C91589782875C968C915C9783875E96B1
:10CA70008C915E978487442309F496CF1D96DC90B1
:10CA8000158640E091CF982F967031F42E3261F4E4
:10CA9000F50191819E3241F00115110511F441E03B
:10CAA00083CFD8011C92FBCF83FD7ECF03C080E0F3
:10CAB00090E011C00115110569F0411105C0B501E3
:10CAC000C70106D9D81631F0A501B80182E299E074
:10CAD0000E94619DC5010F90DF91CF911F910F9131
:10CAE000FF90EF90DF90CF90BF90AF9008954F925E
:10CAF0005F926F927F92AF92BF92CF92DF92EF924E
:10CB0000FF920F931F93CF93DF93EC016A017B0198
:10CB10002B81222349F08B899C89AD89BE8984179A
:10CB20009507A607B70710F480E073C0223049F4D8
:10CB3000CB86DC86ED86FE861F82188619861A86CD
:10CB400067C0C114D104E104F10449F41F821886BE
:10CB500019861A861B861C861D861E8659C08B85E3
:10CB60009C85AD85BE85ED81FE81E585F0E0399639
:10CB7000AC01BD0141505109610971090E2E04C07B
:10CB800076956795579547950A94D2F79701860150
:10CB9000015011092109310904C0369527951795CF
:10CBA0000795EA95D2F7041715072607370720F0EF
:10CBB000892B8A2B8B2B49F48F89988DA98DBA8D5F
:10CBC0008F839887A987BA8704C0041B150B260B8F
:10CBD000370B280139015E0187E0A80EB11C411412
:10CBE00051046104710481F04F81588569857A850B
:10CBF00095018D819E81BFDC91E0491A5108610841
:10CC000071088111ECCF05C0CB86DC86ED86FE86EF
:10CC100081E0DF91CF911F910F91FF90EF90DF9016
:10CC2000CF90BF90AF907F906F905F904F9008959E
:10CC300040E050E0BA015BCFAF92BF92CF92DF925B
:10CC4000EF92FF920F931F93CF93DF936C01A42E6B
:10CC50007901E801FC018381823008F43DC0C601FE
:10CC6000E7DFB12CA895C60157DE0097B9F1FC01AA
:10CC70002081222399F1253011F0253E91F7FC0106
:10CC800083858F738F3031F1209721F11A1414F5B9
:10CC9000BA1404F1088119812A813B81012B022BEE
:10CCA000032BC1F4F60183859485A585B68580970D
:10CCB000A109B109FB2D40E2F40290011124821B6D
:10CCC000930BA109B10988839983AA83BB83F701D8
:10CCD000B08202C0B394C6CF81E001C080E0DF9192
:10CCE000CF911F910F91FF90EF90DF90CF90BF9069
:10CCF000AF900895AF92BF92CF92DF92EF92FF92E2
:10CD00000F931F93CF93DF9300D01F92CDB7DEB761
:10CD10008C01FC018789908DA18DB28D89839A83C6
:10CD2000AB83BC83A12CB12C49815A816B817C815E
:10CD30009E012F5F3F4FD80115968D919C911697BC
:10CD40001ADC8823C1F1D8011596ED91FC91169754
:10CD50008481A80EB11CA114B0E1BB0658F5C980AE
:10CD6000DA80EB80FC808789803149F481E0E8EF4C
:10CD7000CE16EFEFDE06E104F10450F4D5CF81E0EA
:10CD8000F8EFCF16FFEFDF06EF06FFE0FF0660F2D9
:10CD9000A50160E070E099E0440F551F661F771F02
:10CDA0009A95D1F7D80153964D935D936D937C93EB
:10CDB000569701C080E00F900F900F900F90DF9179
:10CDC000CF911F910F91FF90EF90DF90CF90BF9088
:10CDD000AF900895CF93DF93EC01FB018B81882303
:10CDE00011F080E03BC07E836D838789803101F143
:10CDF0008032B9F783E08B83428D538D648D758DBE
:10CE00004F8B588F698F7A8FCE0174DF882349F357
:10CE100081E089831F82188619861A861B861C86E4
:10CE20001D861E861F86188A198A1A8A1C8216C0B9
:10CE300082E08B831F8A188E198E1A8E408D518D39
:10CE400060E070E025E0440F551F661F771F2A95AC
:10CE5000D1F74B8B5C8B6D8B7E8BDACFDF91CF91D3
:10CE600008950F931F93CF93DF938C01EC01A3964A
:10CE7000662321F0D093B706C093B606F80186A1C9
:10CE8000882311F0CE0161DBB8016B5F7F4FCE01CB
:10CE9000DF91CF911F910F919DCF8F929F92AF9273
:10CEA000BF92CF92DF92EF92FF920F931F93CF9397
:10CEB000DF93EC016A017B014801590142305105C1
:10CEC0006105710508F44DC049855A856B857C85DF
:10CED0004F5F5F4F6F4F7F4F4C155D056E057F05B0
:10CEE00008F43FC08F89803129F499278F2D7E2D3A
:10CEF0006D2D0BC08032A9F5C701B60157E096959C
:10CF00008795779567955A95D1F70B891C892D8957
:10CF10003E89600F711F821F931F43E073DA0097F1
:10CF200001F12F89203159F4DD24EE24FF24F6018C
:10CF3000EE0FFF1FE80FF91F9182808210C0E89466
:10CF4000C7F8DD24EE24FF24F601EE0FFF1FEE0FDD
:10CF5000FF1FE80FF91F80829182A282B38281E0D5
:10CF600001C080E0DF91CF911F910F91FF90EF9072
:10CF7000DF90CF90BF90AF909F908F9008952F92A9
:10CF80003F924F925F926F927F928F929F92AF9259
:10CF9000BF92CF92DF92EF92FF920F931F93CF93A6
:10CFA000DF93CDB7DEB72F970FB6F894DEBF0FBE75
:10CFB000CDBF1C014C875D876E877F873B872A87A3
:10CFC000DC0119960D911D912D913C911C970F5FDD
:10CFD0001F4F2F4F3F4F0D831E832F833887EA85C6
:10CFE000FB8580809180A280B38081149104A1048C
:10CFF000B10431F0FFEF8F1A9F0AAF0ABF0A10C0C9
:10D00000DC018D909D90AD90BC90B1E0B9870C850E
:10D010001D852E853F85013011052105310509F05B
:10D02000198675016401412C512C3201F101818571
:10D030009285A385B485481659066A067B0608F0D2
:10D040004EC00D811E812F8138850C151D052E05C2
:10D050003F0550F472E0C72ED12CE12CF12CE2E018
:10D060008E2E912CA12CB12C9E012F5F3F4FB7012A
:10D07000A601C10180DA882391F149815A816B812F
:10D080007C81D701C6010196A11DB11D452B462B00
:10D09000472B19F04C015D010FC0AC01BD014819CF
:10D0A00059096A097B090C851D852E853F85401726
:10D0B00051076207730741F01FEF411A510A610AD5
:10D0C000710A6C017D01B2CF0FEF1FEF2FEF3FE030
:10D0D000B701A601C101E1DE8D83811113C01D825C
:10D0E0003DC02601370121E0421A5108610871084C
:10D0F00097018601B301A201C101CFDE882379F334
:10D10000730162018C149D04AE04BF0450F3AA8520
:10D11000BB854D915D916D917C91411551056105E6
:10D120007105A9F4EA85FB8580829182A282B3828F
:10D13000F985FF2399F00FEF801A900AA00AB00A30
:10D14000D1018D929D92AD92BC92139707C095012B
:10D150008401C101A2DE8111E5CFC1CF8D812F965F
:10D160000FB6F894DEBF0FBECDBFDF91CF911F91F8
:10D170000F91FF90EF90DF90CF90BF90AF909F9076
:10D180008F907F906F905F904F903F902F90089579
:10D19000CF93DF93EC019C01295F3F4F41E050E0CA
:10D1A00060E070E08D819E81EADE882399F04F89EE
:10D1B000588D698D7A8D452B462B472B59F44F811D
:10D1C000588569857A854F8B588F698F7A8F9981B9
:10D1D00090689983DF91CF9108952F923F924F925B
:10D1E0005F926F927F928F929F92AF92BF92CF92F7
:10D1F000DF92EF92FF920F931F93CF93DF93CDB700
:10D20000DEB728970FB6F894DEBF0FBECDBF7C0106
:10D210005B014A01DC0111968C9181FFB0C182FD56
:10D2200002C064018DC0F7014389548965897689FC
:10D2300083859485A585B68584179507A607B707C6
:10D2400081F3C70154DC8111ECCF99C1D701159648
:10D250008D919C911697FC0134803A94B901A801F4
:10D2600029E076956795579547952A95D1F7342209
:10D270001170332009F470C0D70113968C91139765
:10D280001596ED91FC911697823009F0A9C01B9676
:10D290004D905D906D907C901E9789E07694679498
:10D2A000579447948A95D1F7828D938DA48DB58D2F
:10D2B000480E591E6A1E7B1E0115110509F4AFC0E8
:10D2C00080E092E0801B910B16018C159D0508F4FF
:10D2D0001C010115110509F0A7C0F701438554850C
:10D2E0006585768583899489A589B6894817590704
:10D2F0006A077B0708F498C045E0C301B20182D8F1
:10D30000009709F43CC1A101B501800F911F0F9452
:10D31000EB11020D131D0115124009F487C0F7012E
:10D3200083859485A585B685820D931DA11DB11DAC
:10D3300083879487A587B687A20CB31CC218D3082D
:10D34000D7011B960D911D912D913C911E97C114F3
:10D35000D10409F07BCFE7C00115110509F08CCF8E
:10D3600017964D915D916D917C911A9741155105DC
:10D370006105710509F19E012F5F3F4FFCD888239D
:10D3800009F4FDC089819A81AB81BC81F7012581B7
:10D390003681F9012789203139F4883FFFEF9F0753
:10D3A000A105B10590F416C0883F2FEF9207A207A0
:10D3B0002FE0B20778F009C0F7018789908DA18D21
:10D3C000B28D0097A105B10529F4C701E1DE8111F5
:10D3D00053CFD5C0F70187839087A187B2874CCF01
:10D3E0008481D70117962D913D914D915C911A97AB
:10D3F0002250310941095109A82FB0E00F94E30DE3
:10D400002B013C0186859785A089B189480E591E5C
:10D410006A1E7B1E430C511C611C711C4DCFC11434
:10D42000B2E0DB0640F44CCF41E067CF0E94B4612C
:10D43000811175CFA4C0C11424E0D206F0F480910C
:10D44000B0049091B104A091B204B091B3048415DA
:10D450009505A605B70509F480D89501B301A20189
:10D460008091A9049091AA040E94EA60882309F49B
:10D4700086C0212CA2E03A2E52CF848183193D2C04
:10D480003694831508F4382E032D10E020E030E0A8
:10D49000B301A2018091A9049091AA040E944D6158
:10D4A000882309F46CC085014D825E826F82788684
:10D4B0008D818419831548F58091B0049091B10451
:10D4C000A091B204B091B3042D813E814F81588563
:10D4D000281739074A075B0709F43FD8B80180913C
:10D4E000A9049091AA040E942B611E5F2D813E81A8
:10D4F0004F8158852F5F3F4F4F4F5F4F2D833E83A6
:10D500004F8358878111D4CF3AC08091A90490915C
:10D51000AA040E949361882391F1232C312C322C90
:10D520002224330CFCCE53968D919D910D90BC918D
:10D53000A02DF701418180179107A207B30738F4A6
:10D54000038B148B258B368B406841830CC08091F4
:10D55000B4069091B506892B31F08114910419F02D
:10D560004068F7014183D70111968C9183FD02C079
:10D57000C4010AC0C7010E945B628111F9CF81E03A
:10D58000F70180838FEF9FEF28960FB6F894DEBFE8
:10D590000FBECDBFDF91CF911F910F91FF90EF9004
:10D5A000DF90CF90BF90AF909F908F907F906F90C3
:10D5B0005F904F903F902F900895AF92BF92CF927F
:10D5C000DF92EF92FF920F931F93CF93DF9300D0E0
:10D5D0001F92CDB7DEB75C016A017B0182E090E06B
:10D5E000A0E0B0E0F50180839183A283B3839E0124
:10D5F0002F5F3F4FB701A601C5010E94BB62811199
:10D6000002C080E023C000E010E09801B701A6014D
:10D61000C50143DC8823A9F3C980DA80EB80FC8054
:10D62000F5018789803149F481E0F8EFCF16FFEFEB
:10D63000DF06E104F10450F4DACF81E098EFC91677
:10D640009FEFD906E9069FE0F90688F20F900F9048
:10D650000F900F90DF91CF911F910F91FF90EF905E
:10D66000DF90CF90BF90AF9008954F925F926F92EE
:10D670007F92AF92BF92CF92DF92EF92FF920F9381
:10D680001F93CF93DF9300D01F92CDB7DEB75C011D
:10D690006A017B01FC0183818130E9F4818181FF92
:10D6A0001AC0F50183899489A589B68984179507DD
:10D6B000A607B70780F0892B8A2B8B2B09F474C03F
:10D6C000F5014384548465847684B701A601C501BD
:10D6D0000EDA811102C080E068C0F5018581968173
:10D6E000C114D104E104F10469F44789508D618DBE
:10D6F000728D63DF882379F3F501178A108E118EFE
:10D70000128E38C0F50147815085618572859E0172
:10D710002F5F3F4F0E94BB628823E9F249815A8103
:10D720006B817C81F50185819681FC0127892031FF
:10D7300039F4483FFFEF5F0761057105D8F407C072
:10D74000483F2FEF520762072FE0720798F435DF4A
:10D75000882309F4C0CFF501478150856185728522
:10D760000FEF1FEF2FEF3FE08581968196DB882337
:10D7700009F4B1CFF501C38AD48AE58AF68A81819A
:10D7800080688183C5010E945B62882309F4A3CF6E
:10D79000B701A6014C145D046E047F0410F4B301BC
:10D7A000A201C501A4D901C081E00F900F900F9094
:10D7B0000F90DF91CF911F910F91FF90EF90DF902D
:10D7C000CF90BF90AF907F906F905F904F900895F3
:10D7D000BF92CF92DF92EF92FF920F931F93CF935E
:10D7E000DF93EC01B42E80E2689FF0011124EC5429
:10D7F000FB4F8091B0049091B104A091B204B0911C
:10D80000B3048F87988BA98BBA8B6C830489158995
:10D8100020E030E0980111270027C28CD38CE12C46
:10D82000F12C0C291D292E293F290F8B188F298FA8
:10D830003A8F8385887151F4048D158D268D378D2F
:10D840000B8B1C8B2D8B3E8B81E00BC08031F1F458
:10D85000CE0150DA811104C01B8A1C8A1D8A1E8ADF
:10D8600084E08B838B2D8F7089831F8218861986A5
:10D870001A861B861C861D861E86B4FE0AC040E0E2
:10D8800050E0BA01CE01F1DE811103C01B8280E0BD
:10D8900012C0B5FE0FC04B895C896D897E89CE01AF
:10D8A000DF91CF911F910F91FF90EF90DF90CF907C
:10D8B000BF901DC981E0DF91CF911F910F91FF9023
:10D8C000EF90DF90CF90BF900895DF92EF92FF929C
:10D8D0000F931F93CF93DF938C01EB017A01D22E2C
:10D8E0008D819E81F801968385838381811128C073
:10D8F000209731F127FD24C0A70165E0440F551F93
:10D900006A95E1F760E070E0CE01F1D88823C1F0BC
:10D91000CE0102D80097A1F0FC018081882381F01C
:10D92000853E71F08E3261F06E2D6F704D2DC80105
:10D93000DF91CF911F910F91FF90EF90DF9048CF33
:10D9400080E0DF91CF911F910F91FF90EF90DF90DA
:10D9500008952F923F924F925F926F927F928F9293
:10D960009F92AF92BF92CF92DF92EF92FF920F936E
:10D970001F93CF93DF93CDB7DEB7C454D1090FB651
:10D98000F894DEBF0FBECDBF4C017B016A01422E71
:10D99000302E1EAA1FAA18AE19AEDB0115968D9166
:10D9A0009C911697F40196838583CB0141D946FE5D
:10D9B0001AC0F60101900020E9F73197EC1977249D
:10D9C0007394E9300CF0712C8E2F6DE00F94500D94
:10D9D00021E0911101C020E08E2F6DE00F94500DD9
:10D9E000582E520E03C055245A94712C8E010A5C95
:10D9F0001F4F252D44EE59E0B501C7010E94BD64BB
:10DA00005C01009779F1A895D7011B968D919D91A6
:10DA10000D90BC91A02D23968CAF9DAFAEAFBFAF44
:10DA20002397B60184EE99E00E94789D8111DECFA4
:10DA300047FE02C080E08FC123968CAD9DADAEAD98
:10DA4000BFAD23974F97A109B109F5E0B695A7950A
:10DA500097958795FA95D1F7682F6F70442DC4017B
:10DA6000B7DE79C1842D8274823421F79E01265C51
:10DA70003F4F452DFE0131965F01BF01C701DCD844
:10DA80008EA99FA9A8ADB9AD892B8A2B8B2BA9F4A0
:10DA9000D70113962C9113971B968D919D910D9004
:10DAA000BC91A02D223009F046C18115E0E49E070B
:10DAB000A105B10508F0BECF3EC122242394D701B1
:10DAC00011968C911197826011968C934EA95FA943
:10DAD00068AD79ADC7010BD8711037C06EE270E048
:10DAE000C6010F94FF113C0186010A5F1F4F00978A
:10DAF00061F044E050E0BC01CE01C1960F941A12CF
:10DB00001DAA0615170518F401C019AA38016C18CA
:10DB10007D087724A301B601CE0181960F94EB1105
:10DB2000E1E2F0E0EC0FFD1FE60DF71D108263E669
:10DB300073E0CE0181960F94F411BE016F5C7F4FAC
:10DB4000CE0181960F94F41105C0B601CE018196E5
:10DB50000F941312AE014F5C5F4FB501CE01819659
:10DB60000E94255EB501C4010E94685E782EF60110
:10DB700001900020E9F78F01015011090C191D09CE
:10DB8000652C252D332727FD309525963FAF2EAFE9
:10DB9000259711279E01215F3F4F3CAF2BAF225F9E
:10DBA0003F4F3EAF2DAF662009F460C0862D90E058
:10DBB000BC01615071093DE0639F602D1124D501C6
:10DBC000E0E21D92EA95E9F72FE02C8725962EAD2D
:10DBD0003FAD25978217930711F480E401C080E0E0
:10DBE0008629898340E050E0FE01329670E0C6014C
:10DBF000860F971F21969FAF8EAF2197CF01029678
:10DC00009A01260F371F0217130734F49C01AFEF58
:10DC1000BFEFB183A0830DC09C012196AEADBFAD17
:10DC20002197A40FB51F8C91992787FD909591831B
:10DC30008083443029F04A3029F42DAD3EAD02C036
:10DC40002BAD3CAD4F5F5F4F4D30510511F0F901E9
:10DC5000D5CF7E8640E250E0B501C701BEDA97FD20
:10DC6000E9CEC7010E945B626A949DCF80E2F50114
:10DC700011928A95E9F7AE014F5C5F4FB501CE0175
:10DC800081960E94255E332011F080E101C080E280
:10DC90008C8781E298E29A8B898B20E038E0388B80
:10DCA0002F879C8B8B8B9A8F898F388F2F8B40E29D
:10DCB00050E0B501C70191DA97FDBCCEC7010E94C3
:10DCC0005B6280E2D5011D928A95E9F7222011F06E
:10DCD00085EE8983D12C052D112707FD10958AAD7E
:10DCE000992787FD9095801B910B2D2D332727FDBC
:10DCF00030952817390764F440E250E0B501C701B8
:10DD00006CDA97FD97CEC7010E945B62D394E7CF90
:10DD1000242D2F774EA95FA968AD79ADE5E0769502
:10DD2000679557954795EA95D1F7400F511FB70171
:10DD3000C401CBDD10C021E0250D2AAF0097A1055D
:10DD4000B10539F08097A109B1098EAB9FABA8AF9F
:10DD5000B9AF212CB4CECC5BDF4F0FB6F894DEBF49
:10DD60000FBECDBFDF91CF911F910F91FF90EF902C
:10DD7000DF90CF90BF90AF909F908F907F906F90EB
:10DD80005F904F903F902F900895BF92CF92DF9277
:10DD9000EF92FF920F931F93CF93DF93CDB7DEB730
:10DDA000A0970FB6F894DEBF0FBECDBF7C016B010C
:10DDB000FB018381823088F101E023ECC701C9DDDA
:10DDC000B82E882351F18E010F5F1F4F80E2F801BA
:10DDD00011928A95E9F721E238E23A8B298B80E0AB
:10DDE00098E0988B8F873C8B2B8B3A8F298F988F5D
:10DDF0008F8B8EE2898380E18C87FE013296CE0183
:10DE00000C9620E22193E817F907E1F740E250E091
:10DE1000B801C701E2D997FF02C0B12C37C0C701D2
:10DE20000E945B628EE28A83F60183818250823097
:10DE300028F41C8E1B8E1E8A1D8A09C0F601478994
:10DE4000508D618D728D5C8F4B8F7E8B6D8B40E220
:10DE500050E0B801C701C1D997FDDFCFC7010E94CB
:10DE60005B6280E2F80111928A95E9F740E250E0A6
:10DE7000B801C701B2D997FDD0CFC7010E945B623C
:10DE800084E0F70183838181806881838B2DA09654
:10DE90000FB6F894DEBF0FBECDBFDF91CF911F91BB
:10DEA0000F91FF90EF90DF90CF90BF9008952F9249
:10DEB0003F924F925F926F927F928F929F92AF921A
:10DEC000BF92CF92DF92EF92FF920F931F93CF9367
:10DED000DF93CDB7DEB7C154D1090FB6F894DEBFDA
:10DEE0000FBECDBF4B016A0139011801EFAE1E8E86
:10DEF00019A219821C82F90110826115710511F4B1
:10DF000080E08AC0FC0183818111FACFFA0180810F
:10DF10008F3261F4CA016C010196F60120812F3223
:10DF2000D1F3F40183818250823010F454010CC08B
:10DF3000F40165817681CE0101960E94EA6688230C
:10DF4000F9F2CE0101965C017E019EE1E90EF11C21
:10DF5000FCAEEBAEFE013196FEAFEDAF2196EFAE1B
:10DF600021972296FFAE229734C092012C193D09C9
:10DF7000022F112707FD1095A801B601C3010F94C8
:10DF8000EB11F301E00FF11F1082F2018181882370
:10DF9000D9F100E021E0A301B501C701DADC882353
:10DFA00009F1A814B90419F0C5010E94A5628BAD4E
:10DFB0009CADE816F90609F121969FAD21972296AE
:10DFC0008FAD22976201EFEFCE1ADE0A5701E92EDC
:10DFD000F82E6FE270E0C6010F94FF112C0100973C
:10DFE00021F60EC0FFADFF2309F48ACFA301B501CE
:10DFF000C701CBDE8111D5CF83CF9DAD8EADE2CFF2
:10E00000B601C3010F9413128DE1F501D101019006
:10E010000D928A95E1F781E0CF5BDF4F0FB6F89460
:10E02000DEBF0FBECDBFDF91CF911F910F91FF904B
:10E03000EF90DF90CF90BF90AF909F908F907F90A8
:10E040006F905F904F903F902F900895CF92DF9206
:10E05000EF920F931F93CF93DF93CDB7DEB7E9977E
:10E060000FB6F894DEBF0FBECDBF6C0119821C82C3
:10E07000E22E8E010F5F1F4F9E01225E3F4F17DF82
:10E08000882339F0AE01425E5F4FB801C6017DDEE4
:10E0900001C080E0E9960FB6F894DEBF0FBECDBF99
:10E0A000DF91CF911F910F91EF90DF90CF90089566
:10E0B000CF93DF93CDB7DEB76D970FB6F894DEBF81
:10E0C0000FBECDBF242F19821C828396AB01BC01E9
:10E0D000CE010196BBDF6D960FB6F894DEBF0FBE82
:10E0E000CDBFDF91CF910895CF92DF92EF92FF9253
:10E0F0000F931F93CF93DF93CDB7DEB7E9970FB69A
:10E10000F894DEBF0FBECDBF6C01F22E19821C82C7
:10E11000E12C8E010F5F1F4F9E01225E3F4FC7DE35
:10E12000882371F08E8D882369F000E02F2DAE01D9
:10E13000425E5F4FBE016F5F7F4FC6010ADC03C0C6
:10E1400080E001C081E0E9960FB6F894DEBF0FBE13
:10E15000CDBFDF91CF911F910F91FF90EF90DF9096
:10E16000CF900895FF920F931F93CF93DF93CDB776
:10E17000DEB76D970FB6F894DEBF0FBECDBFFB01C3
:10E18000F42E19821C8220812F3239F42181211131
:10E1900004C0642F0E9431671EC08C010D5D1F4FAB
:10E1A00021E0AF01B801CE0101969EDF882399F0EE
:10E1B0009C81923078F09DE1FE013196D80101906A
:10E1C0000D929A95E1F7FF2031F01093B706009376
:10E1D000B60601C080E06D960FB6F894DEBF0FBEA4
:10E1E000CDBFDF91CF911F910F91FF900895FB015B
:10E1F000242F6091B6067091B706AF0175CFCF930B
:10E20000DF93EC0140E050E0BA012FDA882371F08F
:10E2100061E0CE010E944462009741F025EEFC01CE
:10E2200020831B82DF91CF910C94B46180E0DF9159
:10E23000CF910895CF93DF93CDB7DEB76D970FB62B
:10E24000F894DEBF0FBECDBFAB0119821C8222E065
:10E25000BC01CE01019648DF882319F0CE0101965A
:10E26000CEDF6D960FB6F894DEBF0FBECDBFDF9147
:10E27000CF9108958396DECF0F931F93CF93DF93B3
:10E28000EC018B81843061F5CE010E9418660B850C
:10E290001C852D853E854B895C896D897E89041797
:10E2A00015072607370748F4CE010E948C640097B3
:10E2B000B9F0FC01208121110BC081E08B838981A1
:10E2C00082608983CE01DF91CF911F910F9197CF0B
:10E2D000253EE9F22E32D9F2FC01838583FDD7CFAA
:10E2E00080E0DF91CF911F910F910895CF93DF933D
:10E2F000CDB7DEB76D970FB6F894DEBF0FBECDBFBA
:10E3000019821C8241E0CE01019671DF882319F049
:10E31000CE010196B1DF6D960FB6F894DEBF0FBE49
:10E32000CDBFDF91CF9108954F925F926F927F9210
:10E33000AF92BF92CF92DF92EF92FF920F931F9313
:10E34000CF93DF93EC01142F7093AA046093A90478
:10E350001F8A82E090E0A0E0B0E088839983AA83DE
:10E36000BB831092AF048FEF9FEFDC018093B0046A
:10E370009093B104A093B204B093B3041092AB0491
:10E380001092AC041092AD041092AE04442361F1DB
:10E39000453008F0D6C040E060E070E0CB010E945C
:10E3A0000262009709F4CDC0FC0120E1129FE00D4C
:10E3B000F11D1124E255FE4F80818F7709F0C1C015
:10E3C0004485558566857785443651056105710517
:10E3D00008F4B7C0C084D184E284F384C114D104AA
:10E3E000E104F10421F4ADC0C12CD12C760140E050
:10E3F000C701B6010E940262FC01009709F4A1C0A6
:10E40000838594858115924009F09BC02089222341
:10E4100009F497C086859785892B09F492C0858574
:10E42000882309F48EC02A8B25852C831D8630E035
:10E4300041E050E06D85062FCA01062E02C0880F0C
:10E44000991F0A94E2F72817390731F081E0860F07
:10E450008D87683078F375C0268937892115310595
:10E4600019F040E050E004C024A135A146A157A115
:10E470002D833E834F8358872093AB043093AC04A5
:10E480004093AD045093AE048685978526013701ED
:10E49000480E591E611C711C4B8A5C8A6D8A7E8AEB
:10E4A000A188B288B98EA88EA089B0E00F94E30D40
:10E4B000640D751D861D971D6A8F7B8F8C8F9D8FB8
:10E4C00015E0AA0CBB1C1A95E1F741E0A41A4EEF27
:10E4D000B40AAB2CBB24A694DC01CB018A0D9B1D96
:10E4E000A11DB11D8E879F87A88BB98B4388548847
:10E4F0004114510419F0612C712C04C040A051A0AA
:10E5000062A073A0A7019601281B390B4A0B5B0B75
:10E51000DA01C901840D951DA61DB71D04C0B6956D
:10E52000A795979587950A95D2F789879A87AB879C
:10E53000BC87853F3FE09307A105B10520F48CE03F
:10E540008F8B80E012C0853F9F4FA105B10510F46D
:10E5500080E109C084A595A5A6A5B7A58A8F9B8F44
:10E56000AC8FBD8F80E28F8B81E0DF91CF911F91C7
:10E570000F91FF90EF90DF90CF90BF90AF907F9082
:10E580006F905F904F9008950F931F93CF93DF93F9
:10E59000EC01842F462F682FCE010E948C5F8823C8
:10E5A000B9F08E010B5F1F4F41E0BE01C801BCDE18
:10E5B000882341F061E0CE01DF91CF911F910F914F
:10E5C0000C94316740E0BE01C801AEDE8111F2CF8C
:10E5D00080E0DF91CF911F910F9108950C94ED6829
:10E5E000682F8AE39BE00C947CD92F923F924F9244
:10E5F0005F926F927F928F929F92AF92BF92CF92D3
:10E60000DF92EF92FF920F931F93CF93DF93CDB7DB
:10E61000DEB76D970FB6F894DEBF0FBECDBF7B019E
:10E62000342E59014801CB010E941866C12CD12C0F
:10E6300022242394230C00E010E020E044EE59E073
:10E64000B601C7010E94BD646C01009739F0A8951E
:10E65000D6011B961C9113FF03C0EDCF80E0C2C012
:10E6600068E673E084EE99E00F940A12892B19F39F
:10E670001871103109F067C0B1E0B315E0F2A114D0
:10E68000B10491F4332041F08BEA99E00E94C79FD6
:10E6900086E294E20E94839F84EE99E00E94C79FE5
:10E6A00086E294E20E949C9F19821C82332031F002
:10E6B00066E673E08BEA99E00F94F41164EE79E07A
:10E6C0008BEA99E00F94F411F70143845484658434
:10E6D0007684FFE14F1A51086108710845E076948D
:10E6E0006794579447944A95D1F721E0A201B70166
:10E6F000CE010196EAD8882351F084019501422D7C
:10E70000BE016F5F7F4FCB0170DF81116AC08FEF59
:10E71000481A580A35E0440C551C3A95E1F7A20115
:10E7200060E070E0C7010E9477656FE270E08BEAFD
:10E7300099E00F942912009719F0DC011C927BCF0D
:10E740001092AB0978CFA114B10489F1EBEAF9E09A
:10E75000DF010D900020E9F78D01015011090B5ADE
:10E760001940702E402F552747FD5095B501CF0118
:10E770000E94B59D81115FCF10161CF4772473940D
:10E78000700EB501670D711D77FC7A9584EE99E0E6
:10E790000E94789D81114FCF8114910411F18DE178
:10E7A000F701D40101900D928A95E1F71AC0332048
:10E7B00041F08BEA99E00E94C79F86E294E20E94B2
:10E7C000839F84EE99E00E94C79FF601448D558D8A
:10E7D000668D778D85EB93E20E94A7A00E941C2492
:10E7E0002ACF81E06D960FB6F894DEBF0FBECDBF85
:10E7F000DF91CF911F910F91FF90EF90DF90CF901D
:10E80000BF90AF909F908F907F906F905F904F9050
:10E810003F902F900895EF92FF920F931F93CF9305
:10E82000DF93CDB7DEB76D970FB6F894DEBF0FBE9E
:10E83000CDBF7C0119821C820E941866EBEAF9E0C8
:10E840001082D7015C96FC93EE935B978DE1F70104
:10E85000DE01119601900D928A95E1F700E010E03B
:10E8600020E030E040E0BE016F5F7F4FC701BDDEBA
:10E870006D960FB6F894DEBF0FBECDBFDF91CF917E
:10E880001F910F91FF90EF900895882321F08091C0
:10E890000B018D7F03C080910B01826080930B017F
:10E8A0000895882321F080910B018E7F03C0809111
:10E8B0000B01816080930B010895882321F08091E2
:10E8C0000B018B7F03C080910B01846080930B014F
:10E8D0000895FB01DC0180915108882349F023E36E
:10E8E00033E34BEC51E4CD010F947A0CFB01DC01D6
:10E8F000BF01CD010895CF93DF931F92CDB7DEB74F
:10E900009091C80790FF02C0811143C02091C707B2
:10E9100023FD3FC091609093C807179A169A159AE5
:10E9200089830E94D4518981811125C020E040E073
:10E9300060E070E0CB010E943A5520E041E060E0E9
:10E9400070E0CB010E943A5540E060E070E0CB01FE
:10E950000E94035640E069E877E186E79AE00E946A
:10E96000A6AB86E79AE00E94FAAE8091C70788605E
:10E970008093C7070EC040E068E777E186E79AE03A
:10E980000E94A6AB86E79AE00F90DF91CF910C949E
:10E99000FAAE0F90DF91CF910895CF93C091C80741
:10E9A000CD7FC093C80720E030E0A90160918002CC
:10E9B0007091810280918202909183020F94D2091A
:10E9C000882319F0C260C093C807CF9108952F9291
:10E9D0003F924F925F926F927F928F929F92AF92EF
:10E9E000BF92CF92DF92EF92FF920F931F93CF933C
:10E9F000DF93CDB7DEB76D970FB6F894DEBF0FBECD
:10EA0000CDBF8BE793E00F94511290934E07809304
:10EA10004D0789E793E00F94511290934C07809330
:10EA20004B07C0902F03D0903003E0903103F0905B
:10EA30003203C0922B03D0922C03E0922D03F0926C
:10EA40002E03C0922703D0922803E0922903F0926C
:10EA50002A038091030390910403A0910503B091D0
:10EA600006038093FF0290930003A0930103B093E9
:10EA700002038093FB029093FC02A093FD02B093EB
:10EA8000FE028091130390911403A0911503B0919D
:10EA9000160380930F0390931003A0931103B09378
:10EAA000120380930B0390930C03A0930D03B09378
:10EAB0000E0380911F0390912003A0912103B09138
:10EAC000220380931B0390931C03A0931D03B09318
:10EAD0001E038093170390931803A0931903B09318
:10EAE0001A038091F3029091F402A091F502B09183
:10EAF000F6028093EF029093F002A093F102B0939C
:10EB0000F2028093EB029093EC02A093ED02B0939B
:10EB1000EE0220910B0730910C0740910D075091A8
:10EB20000E07C701B6010F947A0C0F94720A609316
:10EB30002B0770932C0780932D0790932E0720911D
:10EB40001707309118074091190750911A07C7010C
:10EB5000B6010F947A0C0F94720A60932707709392
:10EB600028078093290790932A0720910F07309157
:10EB700010074091110750911207C701B6010F9479
:10EB80007A0C0F94720A6093230770932407809382
:10EB90002507909326072091070730910807409199
:10EBA000090750910A07C701B6010F947A0C0F9418
:10EBB000720A60931F077093200780932107909338
:10EBC0002207C0907707D0907807E0907907F090FF
:10EBD0007A0781E993E00E942D1D9B01AC01C701DA
:10EBE000B6010F946E092B013C01C0907707D090BD
:10EBF0007807E0907907F0907A0785E993E00E9422
:10EC00002D1D9B01AC01C701B6010F946E094B018C
:10EC10005C01C0907707D0907807E0907907F0907A
:10EC20007A0789E993E00E942D1D9B01AC01C70181
:10EC3000B6010F946E096B017C0185E893E00E9498
:10EC40002D1D2BED3FE049E450E40F947A0C20E0B9
:10EC500030E044E353E40F94D9090F94D6099B01A3
:10EC6000AC01C301B2010F947A0C20912F033091B3
:10EC7000300340913103509132030F947A0C20E01D
:10EC800030E040E05FE30F946E090F94E00A0F94C8
:10EC9000720A60936F077093700780937107909367
:10ECA000720785E893E00E942D1D2BED3FE049E4BB
:10ECB00050E40F947A0C20E030E044E353E40F94E6
:10ECC000D9090F94DD0C9B01AC01C301B2010F9473
:10ECD0007A0C20912F0330913003409131035091F1
:10ECE00032030F947A0C20E030E040E05FE30F94B1
:10ECF0006E090F94E00A0F94720A60936B07709389
:10ED00006C0780936D0790936E0789E893E00E94EB
:10ED10002D1D2BED3FE049E450E40F947A0C20E0E8
:10ED200030E044E353E40F94D9090F94D6099B01D2
:10ED3000AC01C501B4010F947A0C20912F033091DE
:10ED4000300340913103509132030F947A0C20E04C
:10ED500030E040E05FE30F946E090F94E00A0F94F7
:10ED6000720A6093670770936807809369079093AE
:10ED70006A0789E893E00E942D1D2BED3FE049E4EE
:10ED800050E40F947A0C20E030E044E353E40F9415
:10ED9000D9090F94DD0C9B01AC01C501B4010F949E
:10EDA0007A0C20912F033091300340913103509120
:10EDB00032030F947A0C20E030E040E05FE30F94E0
:10EDC0006E090F94E00A0F94720A609363077093C0
:10EDD000640780936507909366078DE893E00E942F
:10EDE0002D1D2BED3FE049E450E40F947A0C20E018
:10EDF00030E044E353E40F94D9090F94D6099B0102
:10EE0000AC01C701B6010F947A0C20912F03309109
:10EE1000300340913103509132030F947A0C20E07B
:10EE200030E040E05FE30F946E090F94E00A0F9426
:10EE3000720A60935F0770936007809361079093F5
:10EE400062078DE893E00E942D1D2BED3FE049E421
:10EE500050E40F947A0C20E030E044E353E40F9444
:10EE6000D9090F94DD0C9B01AC01C701B6010F94C9
:10EE70007A0C20912F03309130034091310350914F
:10EE800032030F947A0C20E030E040E05FE30F940F
:10EE90006E090F94E00A0F94720A60935B077093F7
:10EEA0005C0780935D0790935E0785EA93E00E947C
:10EEB0002D1D6B017C0181E793E00E942D1D9B01BC
:10EEC000AC01C701B6010F946E0920912F03309158
:10EED000300340913103509132030F947A0C0F9418
:10EEE000770A6093870770938807809389079093C8
:10EEF0008A0789EA93E00E942D1D6B017C0181E75E
:10EF000093E00E942D1D9B01AC01C701B6010F9437
:10EF10006E0920912F0330913003409131035091BD
:10EF200032030F947A0C0F94770A609383077093DF
:10EF3000840780938507909386078DEA93E00E946B
:10EF40002D1D6B017C0181E793E00E942D1D9B012B
:10EF5000AC0140902F0350903003609031037090CB
:10EF60003203C701B6010F946E09A30192010F94F9
:10EF70007A0C0F94770A4B015C01C0908707D09000
:10EF80008807E0908907F0908A071091C8078FEFF3
:10EF9000C816D806E104F104C0F4609177077091B7
:10EFA00078078091790790917A079B01AC010F94C3
:10EFB0006E09A30192010F947A0C20E03EEF4FE717
:10EFC00057E40F94060C1816D4F510681093C80770
:10EFD000C701B6010F94A30A9B01AC010F947A0CF0
:10EFE00060938707709388078093890790938A07B7
:10EFF00060918307709184078091850790918607BF
:10F000000F94A30A9B01AC010F947A0C60938307C1
:10F01000709384078093850790938607C501B40198
:10F020000F94A30A9B01AC010F947A0C60937F07A5
:10F0300070938007809381079093820733C01F7776
:10F040001093C807A7019601C701B6010F94410D9F
:10F0500060938707709388078093890790938A0746
:10F06000609183077091840780918507909186074E
:10F070009B01AC010F94410D60938307709384074B
:10F080008093850790938607A5019401C501B4017B
:10F090000F94410D60937F077093800780938107E1
:10F0A000909382078DE993E00E942D1D9B01AC0196
:10F0B0000F947A0C60937B0770937C0780937D0795
:10F0C00090937E07198A1A8A1B8A1C8A1D861E86BF
:10F0D0001F86188A80912B0790912C07A0912D07ED
:10F0E000B0912E078D8B9E8BAF8BB88FBE016F5F5B
:10F0F0007F4FCE010D960E9418ED89819A81AB81D8
:10F10000BC8180938B0790938C07A0938D07B0935D
:10F110008E0780912B0790912C07A0912D07B0911D
:10F120002E0780932F0790933007A0933107B09359
:10F1300032078093330790933407A0933507B09339
:10F14000360710921F071092200710922107109285
:10F15000220710922307109224071092250710927D
:10F16000260710922707109228071092290710925D
:10F170002A0740902F035090300360903103709025
:10F18000320320E030E040E751E4C301B2010F94C4
:10F190007A0C0F94720A60937307709374078093CC
:10F1A00075079093760787E2882E83E0982E91E486
:10F1B000A92E98E0B92E0BEF12E021E3222E28E0D1
:10F1C000322EEBEEF2E0FD8FEC8F81E298E09B8F28
:10F1D0008A8F198EF401C190D190E190F1904F0186
:10F1E000A701960160E070E080E89FE30F94D909E1
:10F1F000F50161937193819391935F01F80161919E
:10F200007191819191918F01A70196010F947A0CD0
:10F210000F94770AF10161937193819391931F0188
:10F22000EC8DFD8D6191719181919191FD8FEC8FAC
:10F23000A70196010F947A0C0F94770AEA8DFB8D43
:10F240006193719381939193FB8FEA8FF98DFF5FA7
:10F25000F98FF43009F0BECFA090EB02B090EC0231
:10F26000C090ED02D090EE02E090FB02F090FC0224
:10F270000091FD021091FE029501A601B701C8019F
:10F280000F94D20987FF02C07501860120912703E0
:10F29000309128034091290350912A03B701C801F6
:10F2A0000F947A0C9B01AC0160E070E080E090E488
:10F2B0000F94D9090F94E70C9B01AC01B701C80169
:10F2C0000F947A0C60933B0770933C0780933D0743
:10F2D00090933E07A090F302B090F402C090F50224
:10F2E000D090F602E0900303F09004030091050330
:10F2F000109106039501A601B701C8010F94D20928
:10F3000087FF02C0750186019701A801C301B20100
:10F310000F947A0C9B01AC0160E070E080E090E417
:10F320000F94D9090F94E70C9B01AC01B701C801F8
:10F330000F947A0C609337077093380780933907DE
:10F3400090933A072ADB6D960FB6F894DEBF0FBE96
:10F35000CDBFDF91CF911F910F91FF90EF90DF9084
:10F36000CF90BF90AF909F908F907F906F905F9065
:10F370004F903F902F900895EF92FF920F931F931D
:10F380006093C9077093CA078093CB079093CC070B
:10F390002093CD073093CE074093CF075093D007EB
:10F3A000E092D107F092D2070093D3071093D407CD
:10F3B0001F910F91FF90EF900895CF92DF92EF92FF
:10F3C000FF9281E00E94211E86E79AE00E9478CA9F
:10F3D0000F94090420912C0C211148C02091C507DD
:10F3E00022FD44C0C0908C1DD0908D1DE0908E1DDC
:10F3F000F0908F1D9B01AC012C193D094E095F094E
:10F4000069017A018091420390914303A0914403E2
:10F41000B09145030097A105B10541F08C159D05FC
:10F42000AE05BF0518F480E066DA05C08091C70715
:10F43000877F8093C70780913E0390913F03A091FF
:10F440004003B09141030097A105B10539F08C1537
:10F450009D05AE05BF0510F481E04DDA82E299E02A
:10F46000FF90EF90DF90CF900C94F69A60938C1DF4
:10F4700070938D1D80938E1D90938F1DEFCFAF9253
:10F48000BF92CF92DF92EF92FF920F931F93CF9391
:10F49000DF93EB01D82EC92E1092FD071092FE07C4
:10F4A0001092FF07109200081092010810920208B3
:10F4B0001092030810920408109205081092060892
:10F4C000109207081092080861E178E08DEF97E04C
:10F4D0000E9418ED60912B0770912C0780912D07E9
:10F4E00090912E070F94A50A20E030E040EC5FE3F6
:10F4F0000F947A0C0F94720A7B018C0121E02F93F8
:10F500002F93CF92DF92DF93CF93A12CB12C650183
:10F5100020E030E0A90160E070E0CB010E942CF80F
:10F520001092F7061092F8061092F9061092FA0659
:10F530001092F3061092F4061092F5061092F60659
:10F540000F900F900F900F900F900F90DF91CF9131
:10F550001F910F91FF90EF90DF90CF90BF90AF90F1
:10F5600008954F925F926F927F928F929F92AF9287
:10F57000BF92CF92DF92EF92FF920F931F93CF93A0
:10F58000DF9300D01F92CDB7DEB760911303709167
:10F590001403809115039091160371DF60912F037E
:10F5A0007091300380913103909132039B01AC0143
:10F5B0000F946E0920E030E040EA50EC0F947A0C92
:10F5C0000F94720A2B013C011F92992493949F92ED
:10F5D00020E030E040E05FE360911303709114039A
:10F5E00080911503909116030F947A0C9F938F933B
:10F5F0007F936F93A12CB12C65018301720120E0F0
:10F6000030E0A90160E070E0CB010E942CF820E01E
:10F6100030E040E05FE36091130370911403809148
:10F620001503909116030F947A0C29DF20E030E047
:10F6300040EA50EC60912F037091300380913103C8
:10F64000909132030F947A0C0F94720A1F929F923A
:10F65000209116032F93209115032F9320911403CB
:10F660002F93209113032F937B018C0120E030E036
:10F67000A90160E070E0CB010E942CF88DE793E0D7
:10F680000F9451128090270790902807A090290787
:10F69000B0902A07B094A09490948094811C911CFF
:10F6A000A11CB11CAA2797FDA095BA2F881A990A08
:10F6B000AA0ABB0A8FE793E00F945112C090230768
:10F6C000D0902407E0902507F0902607F094E0946E
:10F6D000D094C094C11CD11CE11CF11CAA2797FD39
:10F6E000A095BA2FC81AD90AEA0AFB0A81E893E062
:10F6F0000F94511240911F075091200760912107EC
:10F700007091220770956095509541955F4F6F4FAE
:10F710007F4FAA2797FDA095BA2F481B590B6A0B5C
:10F720007B0B0FB6F894DEBF0FBECDBF2A013B01A5
:10F730008C149D04AE04BF0444F484169506A606FA
:10F74000B70654F42401350107C0C416D506E606F1
:10F75000F70614F42601370184189508A608B7089F
:10F76000C418D508E608F708DB01CA018419950911
:10F77000A609B70989839A83AB83BC831092FD07DE
:10F780001092FE071092FF071092000810920108D5
:10F7900010920208109203081092040880912B071F
:10F7A00090912C07A0912D07B0912E07809305080A
:10F7B00090930608A0930708B093080861E178E0E9
:10F7C0008DEF97E00E9418ED80911108909112083A
:10F7D000A0911308B091140888199909AA09BB09C6
:10F7E0008093110890931208A0931308B093140803
:10F7F0008091150890911608A0911708B0911808EB
:10F800008C199D09AE09BF098093150890931608BD
:10F81000A0931708B09318088091190890911A08BE
:10F82000A0911B08B0911C0829813A814B815C8111
:10F83000821B930BA40BB50B8093190890931A08A5
:10F84000A0931B08B0931C081F9281E08F938091B6
:10F8500016038F93809115038F93809114038F93D8
:10F86000809113038F93A12CB12C65018301720148
:10F8700020E030E0A90160E070E0CB010E942CF8AC
:10F880001092FD071092FE071092FF0710920008D9
:10F8900010920108109202081092030810920408B6
:10F8A00080912B0790912C07A0912D07B0912E07E6
:10F8B0008093050890930608A0930708B093080862
:10F8C0001092C9071092CA071092CB071092CC076A
:10F8D0001092CD071092CE071092CF071092D0074A
:10F8E0001092D1071092D2071092D3071092D4072A
:10F8F00061E178E08DEF97E00E9418ED80911108AA
:10F9000090911208A0911308B091140880934F07AA
:10F9100090935007A0935107B09352078091150818
:10F9200090911608A0911708B0911808809353077A
:10F9300090935407A0935507B093560780911908E8
:10F9400090911A08A0911B08B0911C08809357074A
:10F9500090935807A0935907B0935A0760918B076B
:10F9600070918C0780918D0790918E070F94A50A56
:10F970006B017C0120E030E040EA50E460912F030D
:10F980007091300380913103909132030F947A0C7F
:10F990009B01AC01C701B6010F946E090F94720A66
:10F9A00060938B0770938C0780938D0790938E07DD
:10F9B0000F900F900F900F900F900F90E091900389
:10F9C000F091910380810F900F900F900F90DF9135
:10F9D000CF911F910F91FF90EF90DF90CF90BF904C
:10F9E000AF909F908F907F906F905F904F900C940E
:10F9F00003500F931F93CF93DF9380910F08C1E0C3
:10FA000018161CF0C0E08F5F01C0815080930F0872
:10FA10001798169815988091C8078E7F8093C8070D
:10FA20000091090110910901D09109018C2F0E94C8
:10FA300045748C2F0E9451748C2F0E945D7481E05C
:10FA400090E00F945D04409A419A429A82E090E0DF
:10FA50000F945D04409841984298C1E001FB8827CB
:10FA600080F98C270E944574812F81708C270E9419
:10FA70005174D2FB882780F98C27DF91CF911F9199
:10FA80000F910C945D744F925F926F927F928F9260
:10FA90009F92AF92BF92CF92DF92EF92FF920F931D
:10FAA0001F93CF93DF93CDB7DEB728970FB6F894A7
:10FAB000DEBF0FBECDBF2B013C0129833A834B83B0
:10FAC0005C83ED82FE820F8318878501740120918B
:10FAD0009D0730919E0740919F075091A0070F947A
:10FAE0007A0C4B015C012091A9073091AA07409143
:10FAF000AB075091AC0769817A818B819C810F940F
:10FB00007A0C9B01AC01C501B4010F946E094B0145
:10FB10005C012091B5073091B6074091B70750912D
:10FB2000B8076D817E818F8198850F947A0C9B0137
:10FB3000AC01C501B4010F946E09F60160837183B5
:10FB4000828393832091A1073091A2074091A3075C
:10FB50005091A407C301B2010F947A0C4B015C01D0
:10FB60002091AD073091AE074091AF075091B0079B
:10FB700069817A818B819C810F947A0C9B01AC0105
:10FB8000C501B4010F946E094B015C012091B907C6
:10FB90003091BA074091BB075091BC076D817E81BF
:10FBA0008F8198850F947A0C9B01AC01C501B4013B
:10FBB0000F946E09F801608371838283938320918F
:10FBC000A5073091A6074091A7075091A807C30148
:10FBD000B2010F947A0C4B015C012091B107309176
:10FBE000B2074091B3075091B40769817A818B8144
:10FBF0009C810F947A0C9B01AC01C501B4010F9458
:10FC00006E094B015C012091BD073091BE07409108
:10FC1000BF075091C0076D817E818F8198850F94B9
:10FC20007A0C9B01AC01C501B4010F946E09F70178
:10FC3000608371838283938328960FB6F894DEBF26
:10FC40000FBECDBFDF91CF911F910F91FF90EF902D
:10FC5000DF90CF90BF90AF909F908F907F906F90EC
:10FC60005F904F9008954F925F926F927F928F9224
:10FC70009F92AF92BF92CF92DF92EF92FF920F933B
:10FC80001F93CF93DF93CDB7DEB764970FB6F89489
:10FC9000DEBF0FBECDBF69837A838B839C832D83A8
:10FCA0003E834F835887E986FA860B871C87250198
:10FCB0003601E62EF72E082F192F20EF33E244E706
:10FCC00059E4B701C8010F94D20981110DC0809188
:10FCD000F1079091F207A091F307B091F40789839F
:10FCE0009A83AB83BC830AC0C701D8018093F10714
:10FCF0009093F207A093F307B093F407CD80DE80D2
:10FD0000EF80F88420EF33E244E759E4C701B601FD
:10FD10000F94D20981110DC08091F5079091F607DB
:10FD2000A091F707B091F8078D839E83AF83B887C2
:10FD300008C0C092F507D092F607E092F707F0925C
:10FD4000F807C984DA84EB84FC8420EF33E244E7CB
:10FD500059E4C701B6010F94D20981110DC08091F9
:10FD6000F9079091FA07A091FB07B091FC078987EA
:10FD70009A87AB87BC8708C0C092F907D092FA0770
:10FD8000E092FB07F092FC078091C80785FF3DC019
:10FD900029853A854B855C852D873E874F87588B13
:10FDA0002091F3063091F4064091F5065091F60645
:10FDB0006D817E818F8198850F946E09698B7A8B16
:10FDC0008B8B9C8B2091F7063091F8064091F906B9
:10FDD0005091FA0669817A818B819C810F946E091A
:10FDE000AE01475F5F4F4A01DE0115965D019E013E
:10FDF0002F5F3F4F6901ED84FE840F8518892989A3
:10FE00003A894B895C893FDE24C02091F706309106
:10FE1000F8064091F9065091FA0669817A818B8142
:10FE20009C810F946E0969837A838B839C832091D4
:10FE3000F3063091F4064091F5065091F6066D8177
:10FE40007E818F8198850F946E096D837E838F8369
:10FE500098872091270330912803409129035091DE
:10FE60002A0369817A818B819C810F947A0C20E02E
:10FE700030E040E05FE30F946E090F94E00A0F94C6
:10FE8000720A6093D5077093D6078093D707909333
:10FE9000D80720912B0330912C0340912D035091D2
:10FEA0002E036D817E818F8198850F947A0C20E0DE
:10FEB00030E040E05FE30F946E090F94E00A0F9486
:10FEC000720A6093D9077093DA078093DB079093E7
:10FED000DC0720912F033091300340913103509182
:10FEE000320369857A858B859C850F947A0C20E096
:10FEF00030E040E05FE30F946E090F94E00A0F9446
:10FF0000720A6093DD077093DE078093DF0790939A
:10FF1000E00720EF33E244E759E4C301B2010F9454
:10FF2000D2098823C1F08091EA0283FD14C0E091D8
:10FF30009003F091910320E030E046E153E462A9A0
:10FF400073A984A995A90F94060C18165CF18091E9
:10FF5000C70787FD27C020EF33E244E759E468A5CF
:10FF600079A58AA59BA50F94D209882361F088A55D
:10FF700099A5AAA5BBA58093030790930407A09316
:10FF80000507B093060741E061E081E00E94FCF2C2
:10FF9000811106C088E297E10E94A99F80E019C004
:10FFA00081E017C020913303309134034091350331
:10FFB00050913603C301B2010F947A0C0F94720A68
:10FFC0006093E1077093E2078093E3079093E4075F
:10FFD000C2CF64960FB6F894DEBF0FBECDBFDF91DF
:10FFE000CF911F910F91FF90EF90DF90CF90BF9036
:10FFF000AF909F908F907F906F905F904F900895FB
:020000021000EC
:100000004F925F926F927F928F929F92AF92BF9228
:10001000CF92DF92EF92FF920F931F93CF93DF93D4
:10002000CDB7DEB728970FB6F894DEBF0FBECDBFB1
:100030002B013C0129833A834B835C83ED82FE8252
:100040000F8318878501740120919D0730919E07C9
:1000500040919F075091A0070F947A0C4B015C01CF
:100060002091A1073091A2074091A3075091A407C6
:1000700069817A818B819C810F947A0C9B01AC0100
:10008000C501B4010F946E094B015C012091A507D5
:100090003091A6074091A7075091A8076D817E81F6
:1000A0008F8198850F947A0C9B01AC01C501B40136
:1000B0000F946E09F601608371838283938320918C
:1000C000A9073091AA074091AB075091AC07C30133
:1000D000B2010F947A0C4B015C012091AD07309175
:1000E000AE074091AF075091B00769817A818B814B
:1000F0009C810F947A0C9B01AC01C501B4010F9453
:100100006E094B015C012091B1073091B20740911B
:10011000B3075091B4076D817E818F8198850F94CC
:100120007A0C9B01AC01C501B4010F946E09F80172
:1001300060837183828393832091B5073091B607E2
:100140004091B7075091B807C301B2010F947A0CE0
:100150004B015C012091B9073091BA074091BB0770
:100160005091BC0769817A818B819C810F947A0CB4
:100170009B01AC01C501B4010F946E094B015C01F8
:100180002091BD073091BE074091BF075091C00735
:100190006D817E818F8198850F947A0C9B01AC01D3
:1001A000C501B4010F946E09F701608371838283E6
:1001B000938328960FB6F894DEBF0FBECDBFDF91B4
:1001C000CF911F910F91FF90EF90DF90CF90BF9054
:1001D000AF909F908F907F906F905F904F90089519
:1001E0003F924F925F926F927F928F929F92AF92C7
:1001F000BF92CF92DF92EF92FF920F931F93CF9314
:10020000DF9300D01F92CDB7DEB7382E6091FD0787
:100210007091FE078091FF07909100080F94A50A46
:100220002091410830914208409143085091440880
:100230000F947A0C2B013C016093F1077093F20745
:100240008093F3079093F40760910108709102087E
:1002500080910308909104080F94A50A2091450805
:100260003091460840914708509148080F947A0C05
:1002700069837A838B839C836093F5077093F60779
:100280008093F7079093F80760910508709106082E
:1002900080910708909108080F94A50A20914908B9
:1002A00030914A0840914B0850914C080F947A0CB9
:1002B0006093F9077093FA078093FB079093FC070C
:1002C0002091C80725FF15C049EF842E47E0942EE2
:1002D00055EFA52E57E0B52EE1EFCE2EE7E0DE2E4E
:1002E0007B018C0129813A814B815C81C301B20180
:1002F00087DE2091F7063091F8064091F90650917B
:10030000FA066091F1077091F2078091F3079091DE
:10031000F4070F946D092B013C016093F107709372
:10032000F2078093F3079093F4072091F30630913E
:10033000F4064091F5065091F6066091F50770912C
:10034000F6078091F7079091F8070F946D09609375
:10035000F5077093F6078093F7079093F80733201B
:1003600001F14092E5075092E6076092E70770922C
:10037000E8076093E9077093EA078093EB0790938F
:10038000EC078091F9079091FA07A091FB07B091D3
:10039000FC078093ED079093EE07A093EF07B093CF
:1003A000F0070F900F900F900F90DF91CF911F915A
:1003B0000F91FF90EF90DF90CF90BF90AF909F9004
:1003C0008F907F906F905F904F903F9008954F92E5
:1003D0005F926F927F928F929F92AF92BF92CF92D5
:1003E000DF92EF92FF920F931F93CF93DF932B0136
:1003F0003C0149015A01670178018091C70785FDD9
:1004000053C020E030E048EC52ECC701B6010F9435
:10041000060C87FD1DC02DEC3CEC4CE45DE36091C7
:100420000B0770910C0780910D0790910E070F94A8
:100430006E0920E030E040EA50E40F946E099B0121
:10044000AC01C1E0C701B6010F94D20918160CF433
:10045000C0E0A3019201C301B2010F947A0C6B01B9
:100460007C01A5019401C501B4010F947A0C9B0194
:10047000AC01C701B6010F946E09D1E020917B0752
:1004800030917C0740917D0750917E070F94D209EF
:1004900018160CF4D0E0CD2341F481E0A1DE80E910
:1004A00097E10E94511E01C0C1E08C2FDF91CF91D6
:1004B0001F910F91FF90EF90DF90CF90BF90AF9082
:1004C0009F908F907F906F905F904F9008952F92A4
:1004D0003F924F925F926F927F928F929F92AF92D4
:1004E000BF92CF92DF92EF92FF920F931F93CF9321
:1004F000DF93CDB7DEB760970FB6F894DEBF0FBEBF
:10050000CDBF1C0180910E08F1011081811169C0DD
:1005100013FF20C062857385848595850E94697468
:100520002091C9073091CA074091CB075091CC0761
:100530000F946D096093F1077093F2078093F307AE
:100540009093F4076093E5077093E6078093E707BD
:100550009093E80714FF21C0F101668577858089B3
:1005600091890E9469742091CD073091CE07409106
:10057000CF075091D0070F946D096093F5077093E2
:10058000F6078093F7079093F8076093E907709355
:10059000EA078093EB079093EC0715FF8BC0F101FE
:1005A00062897389848995890E9469742091D10731
:1005B0003091D2074091D3075091D4070F946D0921
:1005C0006093F9077093FA078093FB079093FC07F9
:1005D0006093ED077093EE078093EF079093F00719
:1005E00069C013FF21C0F1016285738584859585FB
:1005F0000E9469742091E5073091E6074091E70772
:100600005091E8070F946E096093E5077093E60731
:100610008093E7079093E8076093F1077093F207E0
:100620008093F3079093F40714FF21C0F1016685CE
:100630007785808991890E9469742091E9073091BA
:10064000EA074091EB075091EC070F946E09609315
:10065000E9077093EA078093EB079093EC076093A8
:10066000F5077093F6078093F7079093F80715FF47
:1006700021C0F10162897389848995890E94697416
:100680002091ED073091EE074091EF075091F00770
:100690000F946E096093ED077093EE078093EF0758
:1006A0009093F0076093F9077093FA078093FB0724
:1006B0009093FC078091C8074090ED075090EE079B
:1006C0006090EF077090F00785FF3BC02091F30624
:1006D0003091F4064091F5065091F6066091E907D5
:1006E0007091EA078091EB079091EC070F946E09E7
:1006F0006D877E878F87988B2091F7063091F8065B
:100700004091F9065091FA066091E5077091E6076D
:100710008091E7079091E8070F946E099E012F5F83
:100720003F4F4901AE014B5F5F4F5A01FE013996C1
:100730006F01830172012D853E854F855889A3D9AC
:1007400030C02091F7063091F8064091F90650919B
:10075000FA066091E5077091E6078091E7079091AE
:10076000E8070F946E0969877A878B879C872091A9
:10077000F3063091F4064091F5065091F60660912B
:10078000E9077091EA078091EB079091EC070F94CD
:100790006E096D837E838F83988749825A826B822C
:1007A0007C822091270330912803409129035091A6
:1007B0002A0369857A858B859C850F947A0C20E0C5
:1007C00030E040E05FE30F946E090F94E00A0F946D
:1007D000720A6093D5077093D6078093D7079093DA
:1007E000D80720912B0330912C0340912D03509179
:1007F0002E036D817E818F8198850F947A0C20E085
:1008000030E040E05FE30F946E090F94E00A0F942C
:10081000720A6093D9077093DA078093DB0790938D
:10082000DC0720912F033091300340913103509128
:10083000320369817A818B819C810F947A0C20E04C
:1008400030E040E05FE30F946E090F94E00A0F94EC
:10085000720A6093DD077093DE078093DF07909341
:10086000E007F1010081118106FF35C18091EA02A4
:1008700083FD31C1F101C688D788E08CF18C80906E
:10088000330390903403A0903503B0903603A50154
:100890009401C701B6010F947A0C0E9469740F94F9
:1008A000720A2B013C0180910E08E0919003F091B7
:1008B0009103811104C080910D088823B1F120E0DB
:1008C00030E046E153E462A973A984A995A90F9485
:1008D000D20987FF08C08091C70787FD04C0412C5B
:1008E000512C320115C0C701B6019F772091E50256
:1008F0003091E6024091E7025091E8020F947A0CA1
:1009000020E030E04AE754E40F94060C18163CF35C
:100910008091090890910A08A0910B08B0910C08E9
:10092000840D951DA61DB71DDEC020E030E046E118
:1009300053E462A973A984A995A90F94D20987FFEA
:1009400004C08091C70787FFD7C0809109089091A4
:100950000A08A0910B08B0910C08A3019201281B72
:10096000390B4A0B5B0BCA01B9010F94A50A9F779B
:100970002091E5023091E6024091E7025091E802B1
:100980000F947A0C6B017C0120E030E04AE754E4DC
:10099000C501B4010F947A0C9B01AC01C701B601EB
:1009A0000F94060C18160CF4A7C04092E107509261
:1009B000E2076092E3077092E40710FF3DC0809168
:1009C000510800910107109102078823C9F02FE711
:1009D00037EB4AE85BE3F101628D738D848D958D71
:1009E0000F947A0C6B017C01B801882777FD809504
:1009F000982F0F94A50A9B01AC01C701B60112C044
:100A0000B801882777FD8095982F0F94A50AF101EA
:100A1000228D338D448D558D0F947A0C2EE333EC5B
:100A20004EE259E30F947A0C609303077093040726
:100A30008093050790930607E090ED07F090EE078E
:100A40000091EF071091F0072091E9073091EA0734
:100A50004091EB075091EC076091E5077091E60734
:100A60008091E7079091E807B2DC811111C0809175
:100A7000E1079091E207A091E307B091E40780932A
:100A8000090890930A08A0930B08B0930C080AC0B9
:100A9000F101808191819C0128733327232BC9F4B4
:100AA00086FD02C080E031C04091E1075091E2072D
:100AB0006091E3077091E4078091090890910A081A
:100AC000A0910B08B0910C08481759076A077B07DB
:100AD00049F381E01AC08091090890910A08A09119
:100AE0000B08B0910C088093E1079093E207A09364
:100AF000E307B093E40761CF4092090850920A08D7
:100B000060920B0870920C0850CF60960FB6F89464
:100B1000DEBF0FBECDBFDF91CF911F910F91FF9030
:100B2000EF90DF90CF90BF90AF909F908F907F908D
:100B30006F905F904F903F902F9008954F925F92EB
:100B40006F927F92AF92BF92CF92DF92EF92FF921D
:100B50000F931F93CF93DF93CDB7DEB728970FB6D0
:100B6000F894DEBF0FBECDBF69837A838B839C83ED
:100B700029013A01ED82FE820F83188720EF33E2CC
:100B800044E759E40F94D209882311F12091F70624
:100B90003091F8064091F9065091FA0669817A8100
:100BA0008B819C810F946E0920912703309128033B
:100BB0004091290350912A030F947A0C0F94720AE2
:100BC0006093D5077093D6078093D7079093D80783
:100BD00020EF33E244E759E4C301B2010F94D20994
:100BE000882301F12091F3063091F4064091F50637
:100BF0005091F606C301B2010F946E0920912B03A8
:100C000030912C0340912D0350912E030F947A0CB8
:100C10000F94720A6093D9077093DA078093DB0709
:100C20009093DC0720EF33E244E759E46D817E8145
:100C30008F8198850F94D2098823C1F020912F03CA
:100C40003091300340913103509132036D817E81A8
:100C50008F8198850F947A0C0F94720A6093DD0748
:100C60007093DE078093DF079093E00720EF33E275
:100C700044E759E4C601B5010F94D2098823B1F0C5
:100C80002091330330913403409135035091360362
:100C9000C601B5010F947A0C0F94720A6093E107B4
:100CA0007093E2078093E3079093E40720EF33E229
:100CB00044E759E46A8D7B8D8C8D9D8D0F94D2090C
:100CC000882361F08A8D9B8DAC8DBD8D8093030749
:100CD00090930407A0930507B093060740E061E0F6
:100CE00081E00E94FCF2811106C082E597E10E943A
:100CF000A99F80E003C080E073DA81E028960FB6F8
:100D0000F894DEBF0FBECDBFDF91CF911F910F9141
:100D1000FF90EF90DF90CF90BF90AF907F906F905B
:100D20005F904F9008950E94431E80E059DA8091B1
:100D3000F1079091F207A091F307B091F407809327
:100D4000E4069093E506A093E606B093E70680914B
:100D5000F5079091F607A091F707B091F8078093F7
:100D6000E0069093E106A093E206B093E30680913B
:100D7000F9079091FA07A091FB07B091FC078093C7
:100D8000DC069093DD06A093DE06B093DF0660914B
:100D9000090870910A0880910B0890910C080F9433
:100DA000A50A20914D0830914E0840914F0850916E
:100DB00050080F947A0C6093D8067093D9068093EC
:100DC000DA069093DB068091030790910407A091C7
:100DD0000507B09106078093E1029093E202A09389
:100DE000E302B093E40208958F929F92AF92BF9274
:100DF000CF92DF92EF92FF920F931F93CF93DF93E7
:100E0000982EC62FD42FC22E20E030E0A901609189
:100E1000E1027091E2028091E3029091E4020F946A
:100E2000D20987FDA7C0911005C0C11103C0E1E040
:100E3000ED2701C0E0E0CC2049F0A090D806B090AA
:100E4000D906C090DA06D090DB0608C0F0EFAF2ECE
:100E5000F3E2BF2EF4E7CF2EF9E4DF2EE11102C05A
:100E6000DD23B9F05091DC064091DD063091DE06BD
:100E70002091DF06852F942FA32FB22F8093ED07AB
:100E80009093EE07A093EF07B093F007E11107C02E
:100E900004C050EF43E234E729E4CC23B9F0D09109
:100EA000E006C091E1067091E2066091E3068D2FA5
:100EB0009C2FA72FB62F8093E9079093EA07A09362
:100EC000EB07B093EC07E11107C004C0D0EFC3E219
:100ED00074E769E49920B1F08090E4069090E5060B
:100EE000F091E606E091E706C401AF2FBE2F809394
:100EF000E5079093E607A093E707B093E807B82DBE
:100F0000A92D04C0B0EFA3E2F4E7E9E41F930F9327
:100F1000FF92EF92E52EF42E032F122F2D2F3C2F50
:100F2000472F562F6B2F7A2F8F2F9E2F0E94337EA5
:100F30008091E1029091E202A091E302B091E4027B
:100F40008093030790930407A0930507B0930607C7
:100F50000F900F900F900F9080E0DF91CF911F9135
:100F60000F91FF90EF90DF90CF90BF90AF909F9048
:100F70008F9036C9DF91CF911F910F91FF90EF9025
:100F8000DF90CF90BF90AF909F908F9008959091F9
:100F9000C80795FB222720F9821791F0882311F0CA
:100FA000906201C09F7D9093C807882319F082E169
:100FB00090E202C08CEF9FE10E94B39F80E010C9D5
:100FC0000895AF92BF92CF92DF92EF92FF920F936C
:100FD0001F93CF93E82E062FF42EC091C807C5FBB0
:100FE000CC27C0F980E0D3DF9091C7079160909340
:100FF000C707EE2021F0002339F01F2D06C0011194
:1010000003C011E01F2501C010E040E06DE077E172
:1010100086E79AE00E94A6AB86E79AE00E94FAAEC5
:10102000111102C0FF2019F00E94B17A1FC0EE20FA
:1010300041F01092D5071092D6071092D707109260
:10104000D807002341F01092D9071092DA071092C6
:10105000DB071092DC0740E060E081E00E94FCF2D8
:10106000811104C085EE96E10E94A99FE0900B07D4
:10107000F0900C0700910D0710910E078091160358
:101080008F93809115038F93809114038F93809198
:1010900013038F93A0EFAA2EA3E2BA2EA4E7CA2EC1
:1010A000A9E4DA2E20E030E0A901CA01B9010E94CA
:1010B000337E81E095D81092DF0A8BED96E10E9495
:1010C000511E0F900F900F900F908C2FCF911F916A
:1010D0000F91FF90EF90DF90CF90BF90AF9057CFE0
:1010E0002F923F924F925F926F927F928F929F9238
:1010F000AF92BF92CF92DF92EF92FF920F931F9326
:10110000CF93DF93CDB7DEB72B970FB6F894DEBF42
:101110000FBECDBF6A874D834091F7065091F80608
:101120006091F9067091FA0649835A836B837C8338
:101130004090F3065090F4066090F5067090F60625
:10114000882309F4AEC0222321F08FE390E20E94AD
:101150002A96C090F907D090FA07E090FB07F0902C
:10116000FC0781EA93E00E942D1D9B01AC01C701A1
:10117000B6010F94060C18161CF5E090130310919D
:10118000140300911503F090160381EA93E00E9486
:101190002D1DFF920F931F93EF9210EFA12E13E2DC
:1011A000B12E14E7C12E19E4D12E7B018C01A601CA
:1011B0009501C601B501C2DC0F900F900F900F9002
:1011C00080E293E00E942D1DDC01CB01B05880939A
:1011D000F7069093F806A093F906B093FA0684E216
:1011E00093E00E942D1DDC01CB01B0588093F306E3
:1011F0009093F406A093F506B093F60688E493E086
:101200000E942D1DE62E172F082FF92EA301920103
:101210006091F3067091F4068091F5069091F606C0
:101220000F946D0920912B0330912C0340912D03D5
:1012300050912E030F947A0C0F94720A2B013C01EB
:1012400029813A814B815C816091F7067091F806A3
:101250008091F9069091FA060F946D092091270369
:10126000309128034091290350912A030F947A0C5E
:101270000F94720A21E02F932F93FF920F931F93E5
:10128000EF92A12CB12C6501E12CF12C8701A30177
:1012900092010E942CF80F900F900F900F900F90DA
:1012A0000F900E94431E20E030E040E251E4609144
:1012B0002F037091300380913103909132030F948A
:1012C0007A0C0F94720A6E837F8388879987609166
:1012D00005087091060880910708909108086983B5
:1012E0007A838B839C838091190890911A08A0912E
:1012F0001B08B0911C088093570790935807A09340
:101300005907B0935A071B86412C512C32017D811D
:10131000272E312C7B85872E992487FC909482146C
:1013200093040CF01DC1C0902B07D0902C07E090C7
:101330002D07F0902E0780911F0790912007A09114
:101340002107B0912207C81AD90AEA0AFB0ACC0C75
:10135000DD1CEE1CFF1C8FEF9FEFDC018093470725
:1013600090934807A0934907B0934A0780E293E01F
:101370000E942D1D84E293E00E942D1D8091C807DC
:1013800080648093C8070E9406240E9406240AE015
:1013900010E0959B38C08CE293E00E942D1DA701C0
:1013A0009601EE24FF248701E21AF30A040B150BC1
:1013B00031E03F933F939F938F937F936F93A12C43
:1013C000B12C650120E030E0A90160E070E0CB01C4
:1013D0000E942CF80F900F900F900F900F900F908D
:1013E0008091470790914807A0914907B0914A071B
:1013F000B7FF18C086ED9FE10E94BD9F812C912C04
:1014000030E82FEBFAC18EEC96E10E949C9F64E6D7
:1014100070E080E090E00F9438040150110909F069
:10142000B8CFB9CF8091C8078F7B8093C807009150
:101430005707109158072091590730915A0780910A
:10144000190890911A08A0911B08B0911C08B901C5
:10145000A801481B590B6A0B7B0BDB01CA014093A7
:101460004707509348076093490770934A07409194
:101470001108509112086091130870911408480FD8
:10148000591F6A1F7B1F40931108509312086093E5
:101490001308709314084091150850911608609134
:1014A000170870911808480F591F6A1F7B1F409337
:1014B0001508509316086093170870931808009346
:1014C000190810931A0820931B0830931C084091A8
:1014D0000508509106086091070870910808480FA8
:1014E000591F6A1F7B1F409305085093060860939D
:1014F00007087093080889819A81AB81BC81841B9D
:10150000950BA60BB70B480E591E6A1E7B1EC40115
:1015100001968215930504F58CE293E00E942D1D3F
:101520001F9251E05F939F938F937F936F93A12CB2
:10153000B12C6501EE80FF800885198520E030E040
:10154000A90160E070E0CB010E942CF80F900F9091
:101550000F900F900F900F906B856F5F6B87DACEB7
:10156000C301B2010F94A50A2091490830914A089D
:1015700040914B0850914C080F947A0C6B017C0100
:10158000AD816A2F70E080E090E00F94A30A9B0188
:10159000AC01C701B6010F94D9096B017C0188E247
:1015A00093E00E942D1D9B01AC01C701B6010F9471
:1015B0006E094B018E839D8322E0AB01BC018EEA54
:1015C00090E20E94D8A120E030E040EA52E4B40169
:1015D0008E819D810F947A0C20E030E048EC54E439
:1015E0000F946D09AB01BC0122E082E890E20E94F9
:1015F000D8A14091F1075091F2076091F3077091E3
:10160000F40722E08BE494E20E94D8A14091F50710
:101610005091F6076091F7077091F80722E087E490
:1016200094E20E949BA180E00E94F08088EC96E109
:101630000E94511E8CE293E00E942D1D9B0140915F
:101640000508509106086091070870910808E98024
:10165000FA800B811C81E41AF50A060B170B1F9206
:1016600041E04F939F938F933F932F93A12CB12CE5
:10167000650120E030E0A90160E070E0CB010E944C
:101680002CF80F900F900F900F900F900F90BA853D
:10169000BB2309F4B0C0C090F706D090F806E090E4
:1016A000F906F090FA062090F3063090F406409088
:1016B000F5065090F6068EE390E20E942A9660901E
:1016C0009003709091036114710409F444C0F30114
:1016D00081819281A381B4819C01AD016627772726
:1016E000CB01621B730B840B950B0F94A50A209101
:1016F00041083091420840914308509144080F94AA
:101700007A0C6093F7067093F8068093F90690932D
:10171000FA06F30185819681A781B0859C01AD0110
:1017200066277727CB01621B730B840B950B0F94F5
:10173000A50A2091450830914608409147085091EC
:1017400048080F947A0C6093F3067093F406809324
:10175000F5069093F60688E493E00E942D1D5B0148
:10176000182F092FA20191016091F3067091F406E0
:101770008091F5069091F6060F946D0920912B0348
:1017800030912C0340912D0350912E030F947A0C2D
:101790000F94720A2B013C01A70196016091F70694
:1017A0007091F8068091F9069091FA060F946D09F0
:1017B00020912703309128034091290350912A0357
:1017C0000F947A0C0F94720A21E02F932F930F93AA
:1017D0001F93BF92AF92A12CB12C6501E12CF12C8B
:1017E0008701A30192010E942CF80F900F900F9097
:1017F0000F900F900F903E812D81B401832F922F77
:101800002B960FB6F894DEBF0FBECDBFDF91CF9100
:101810001F910F91FF90EF90DF90CF90BF90AF900E
:101820009F908F907F906F905F904F903F902F9000
:10183000089540E050E060E87FE34093BD07509397
:10184000BE076093BF077093C0074093AD075093E6
:10185000AE076093AF077093B00740939D07509316
:101860009E0760939F077093A0071092B90710928C
:10187000BA071092BB071092BC071092B5071092DE
:10188000B6071092B7071092B8071092B1071092DE
:10189000B2071092B3071092B4071092A9071092E2
:1018A000AA071092AB071092AC071092A5071092EE
:1018B000A6071092A7071092A8071092A1071092EE
:1018C000A2071092A3071092A407811104C087E217
:1018D00090E20C94B39F089588E10FB6F89480933A
:1018E0006000109260000FBE8091C70780648093F3
:1018F000C70754985C9A389A399A3A9A80910A01A3
:10190000826080930A0180910A01816080930A01BC
:1019100080910A01846080930A010F9A179A0E9AA7
:10192000169A0D9A159A0A98129A0998119A3F9840
:10193000479A9D98A59A8091010180628093010148
:10194000809102018F7D809302018091010180646A
:1019500080930101809102018F7B8093020180912D
:101960000101806180930101809102018F7E80934B
:1019700002010E94B8210E94E22281E05ADF80E049
:1019800090E0A8E4B2E48093030790930407A09347
:101990000507B093060784E690E0909302078093D2
:1019A0000107909300078093FF061092ED071092B5
:1019B000EE071092EF071092F0071092E9071092CD
:1019C000EA071092EB071092EC071092E5071092CD
:1019D000E6071092E7071092E8071092900710921E
:1019E0008F071092821D1092831D1092841D1092F9
:1019F000851D80E090E0A0E0B2E48093FB06909328
:101A0000FC06A093FD06B093FE061092F30610921A
:101A1000F4061092F5061092F6061092F706109250
:101A2000F8061092F9061092FA0688E893E1A0E011
:101A3000B0E08093990790939A07A0939B07B09387
:101A40009C0781E08093E9021092ED061092EE0669
:101A50001092EF061092F0061092E9061092EA0634
:101A60001092EB061092EC068093C80780E090E09D
:101A7000AAE7B3E480931B0790931C07A0931D076C
:101A8000B0931E078093130790931407A093150734
:101A9000B093160780E090E8A5ECB3E480930B07C1
:101AA00090930C07A0930D07B0930E0710921707A1
:101AB000109218071092190710921A0710920F0728
:101AC0001092100710921107109212071092070738
:101AD000109208071092090710920A0780E090E020
:101AE000A0E1B3E48093770790937807A0937907F8
:101AF000B0937A071092E806109253081092520899
:101B00000E9425CF40913A0350913B0360913C03E2
:101B100070913D038AE39BE00E94ADDD82EB94E28D
:101B20000E949C9F86E79AE00E94D1AB0E94A5DAB2
:101B30000E947E4F0E943DD61092FD071092FE0734
:101B40001092FF07109200081092F1071092F2070E
:101B50001092F3071092F4071092010810920208F5
:101B600010920308109204081092F5071092F607DD
:101B70001092F7071092F8071092050810920608C5
:101B800010920708109208081092F9071092FA07AD
:101B90001092FB071092FC071092090810920A0895
:101BA00010920B0810920C081092FD071092FE077D
:101BB0001092FF07109200080E94E7740E942023F1
:101BC0000E942E230E9485DA61E178E08DEF97E094
:101BD0000E9418ED8AEF93E00F9444129091C6078B
:101BE000882311F0926001C09D7F9093C607682FF3
:101BF00070E085EC93E00E9481A088E197E10E946B
:101C0000511E80E00E94035082E299E00E94AC9A4B
